:100000000C944E180C947F180C947F180C947F1845
:100010000C947F180C947F180C947F180C947F1804
:100020000C947F180C947F180C947F180C947F18F4
:100030000C947F180C94F6C60C947F180C947F18BF
:100040000C947F180C9427A50C947F180C947F189F
:100050000C947F180C947F180C94622F0C94BCC2E3
:100060000C947F180C94F5A10C947F180C947F18B5
:100070000C947F180C947F180C947F180C947F18A4
:100080000C947F180C947F180C947F180C947F1894
:100090000C947F180C947F180C947F180C94EEBF6E
:1000A0000C947F180C947F180C947F180C947F1874
:1000B0000C947F180C947F180C947F180C947F1864
:1000C0000C947F180C947F180C947F180C947F1854
:1000D0000C947F180C947F180C947F180C947F1844
:1000E0000C947F18AF2FBD2FD92FE72F01300F3081
:1000F00029302D302F3033303B3040C145C14AC10B
:1001000054C1CDC15EC166C16EC178C182C18CC10E
:100110009BC1A5C1CDC1AFC1B9C1C3C1EBC1EEC1C6
:10012000E1C1E5C125C2F2C1F6C1FCC100C204C2F1
:100130000AC20EC212C225C218C21CC220C2084A7C
:10014000D73B3BCE016E84BCBFFDC12F3D6C7431EB
:100150009ABD56833DDA3D00C77F11BED9E4BB4C42
:100160003E916BAAAABE000000803F05A84CCDB20C
:10017000D44EB93836A9020C50B9918688083CA6ED
:10018000AAAA2ABE000000803F007C3C3E5E2B3DB8
:100190003F2F5B5D3B2C2A225C004572723A204D5A
:1001A000415854454D50204245440054656D70659A
:1001B000726174757265206865617465642062653A
:1001C00064207377697463686564206F66662E20A7
:1001D0004D415854454D502074726967676572658A
:1001E00064202121004572723A204D494E54454DFC
:1001F00050003A204578747275646572207377698F
:100200007463686564206F66662E204D494E5445C0
:100210004D502074726967676572656420210045DE
:1002200072723A204D415854454D50003A2045785D
:10023000747275646572207377697463686564208D
:100240006F66662E204D415854454D50207472699A
:10025000676765726564202100202D20496E7661F4
:100260006C6964206578747275646572206E756D52
:10027000626572202100504944204175746F747585
:100280006E652066696E69736865642120507574B7
:1002900020746865206C617374204B702C204B694E
:1002A00020616E64204B6420636F6E7374616E74A2
:1002B000732066726F6D2061626F766520696E745F
:1002C0006F20436F6E66696775726174696F6E2E19
:1002D0006800504944204175746F74756E652066DE
:1002E00061696C6564212074696D656F75740020A7
:1002F000403A006F6B20543A006F6B20423A005036
:100300004944204175746F74756E65206661696C2F
:100310006564212054656D70657261747572652025
:10032000746F6F206869676800204B643A20002072
:100330004B693A2000204B703A200020436C6173D7
:100340007369632050494420002054753A200020EE
:100350004B753A2000206D61783A2000206D696E5F
:100360003A200020643A200020626961733A20003C
:100370001000C90210012C01400122017001180176
:10038000B0010E01F00104015002FA00B002F000C9
:100390003003E600D003DC009004D2007005C800F2
:1003A000A006BE000008B400B009AA00D00BA0004F
:1003B000600E960060118C000015820020197800F4
:1003C000C01D6E00A0226400B0275A00902C50007F
:1003D00000314600E0343C0010383200903A2800EA
:1003E000603C1E00A03D1400803E0A00203F00003B
:1003F00070012C0190012701B0012201C0011D01F3
:10040000F00118011002130130020E01600209010F
:1004100090020401C002FF000003FA004003F5004F
:100420008003F000D003EB002004E6007004E1003C
:10043000E004DC004005D700C005D2004006CD0036
:10044000D006C8008007C3003008BE00F008B9001D
:10045000C009B400B00AAF00B00BAA00D00CA500D0
:10046000000EA000500F9B00C0109600501291008B
:1004700000148C00C0158700B0178200B0197D00F1
:10048000D01B7800001E730040206E00902269008F
:10049000F024640040275F0090295A00E02B5500AB
:1004A000102E500020304B0010324600E033410047
:1004B00090353C001037370070383200A0392D00DD
:1004C000B03A2800A03B2300603C1E00103D1900FC
:1004D000903D1400103E0F00703E0A00C03E050023
:1004E000003F0000686F77746F2E70727573613310
:1004F000642E637A00686F77746F2E707275736103
:1005000033642E636F6D00666F72756D2E70727539
:10051000736133642E637A00666F72756D2E70722C
:1005200075736133642E636F6D0070727573613320
:10053000642E637A00707275736133642E636F6D1D
:10054000005679626572206A617A796B6120202099
:1005500020202020200053656C656374206C616E40
:1005600067756167652020202020004365737469EA
:100570006E6100456E676C697368004572726F72D8
:1005800020696E206D656E75207374727563747565
:100590007265004572726F7220696E206D656E75AE
:1005A0002073747275637475726500446F7374613F
:1005B000766F76616E69205A0041646A757374695A
:1005C0006E67205A00426162797374657070696E5B
:1005D00067205900426162797374657070696E6753
:1005E000205900426162797374657070696E67208A
:1005F0005800426162797374657070696E67205843
:100600000020746F6F206C6F6E6720657874727550
:1006100073696F6E2070726576656E746564002014
:10062000746F6F206C6F6E67206578747275736974
:100630006F6E2070726576656E7465640020636FFE
:100640006C6420657874727573696F6E2070726562
:1006500076656E7465640020636F6C6420657874E1
:10066000727573696F6E2070726576656E746564FD
:1006700000656E6473746F7073206869743A20004B
:10068000656E6473746F7073206869743A200053E8
:100690007465707261746520746F6F206869676833
:1006A0003A2000537465707261746520746F6F2016
:1006B000686967683A200043616E6E6F7420656EEA
:1006C000746572207375626469723A200043616ECA
:1006D0006E6F7420656E74657220737562646972E2
:1006E0003A20006572726F722077726974696E6762
:1006F00020746F2066696C65006572726F72207776
:10070000726974696E6720746F2066696C65004E4B
:100710006F74205344207072696E74696E67004E66
:100720006F74205344207072696E74696E67005351
:1007300044207072696E74696E67206279746520F6
:10074000005344207072696E74696E672062797418
:1007500065200057726974696E6720746F2066693E
:100760006C653A200057726974696E6720746F2057
:1007700066696C653A200046696C652073656C6536
:10078000637465640046696C652073656C656374A9
:100790006564002053697A653A20002053697A65C0
:1007A0003A200046696C65206F70656E65643A207A
:1007B0000046696C65206F70656E65643A20006F55
:1007C00070656E206661696C65642C2046696C6595
:1007D0003A20006F70656E206661696C65642C203C
:1007E00046696C653A2000776F726B446972206FBE
:1007F00070656E206661696C656400776F726B442A
:100800006972206F70656E206661696C6564005363
:10081000442063617264206F6B00534420636172F3
:1008200064206F6B006F70656E526F6F742066612D
:10083000696C6564006F70656E526F6F74206661DD
:10084000696C656400766F6C756D652E696E697490
:10085000206661696C656400766F6C756D652E69E4
:100860006E6974206661696C656400534420696E2A
:100870006974206661696C00534420696E69742054
:100880006661696C0043616E6E6F74206F70656E97
:10089000207375626469720043616E6E6F74206FBD
:1008A00070656E2073756264697200486F74656E5E
:1008B00064206F6666736574733A00486F74656E82
:1008C00064206F6666736574733A006F70656E00BE
:1008D0006F70656E00545249474745524544005475
:1008E0005249474745524544005265706F727469DA
:1008F0006E6720656E6473746F70207374617475B5
:1009000073005265706F7274696E6720656E6473F0
:10091000746F7020737461747573007A5F6D6178A1
:100920003A20007A5F6D61783A20007A5F6D696ED7
:100930003A20007A5F6D696E3A2000795F6D6178C8
:100940003A2000795F6D61783A2000795F6D696EB9
:100950003A2000795F6D696E3A2000785F6D6178AA
:100960003A2000785F6D61783A2000785F6D696E9B
:100970003A2000785F6D696E3A2000496E76616CAE
:10098000696420657874727564657200496E766179
:100990006C69642065787472756465720041637473
:1009A0006976652045787472756465723A200041F5
:1009B00063746976652045787472756465723A204F
:1009C00000556E6B6E6F776E20636F6D6D616E6438
:1009D0003A202200556E6B6E6F776E20636F6D6DDF
:1009E000616E643A202200526573656E643A20009D
:1009F000526573656E643A20005072696E74657258
:100A00002073746F707065642064756520746F2046
:100A10006572726F72732E20466978207468652043
:100A20006572726F7220616E6420757365204D3936
:100A3000393920746F20726573746172742E2028A6
:100A400054656D706572617475726520697320728A
:100A5000657365742E205365742069742061667413
:100A600065722072657374617274696E67290050D3
:100A700072696E7465722073746F7070656420643F
:100A8000756520746F206572726F72732E204669CF
:100A90007820746865206572726F7220616E6420C0
:100AA000757365204D39393920746F207265737400
:100AB0006172742E202854656D7065726174757250
:100AC000652069732072657365742E2053657420E8
:100AD00069742061667465722072657374617274E2
:100AE000696E6729005072696E7465722068616C66
:100AF0007465642E206B696C6C28292063616C6CB2
:100B0000656421005072696E7465722068616C744E
:100B100065642E206B696C6C28292063616C6C65A0
:100B200064210020436F756E7420583A20002043E2
:100B30006F756E7420583A20004649524D57415205
:100B4000455F4E414D453A4D61726C696E2056319C
:100B50002E302E323B20537072696E7465722F678F
:100B600072626C206D617368757020666F722067A9
:100B7000656E36204649524D574152455F55524C9D
:100B80003A68747470733A2F2F6769746875622EAF
:100B9000636F6D2F707275736133642F507275734C
:100BA000612D69332D506C75732F2050524F544F67
:100BB000434F4C5F56455253494F4E3A312E3020E9
:100BC0004D414348494E455F545950453A5072751E
:100BD00073612069332045585452554445525F4350
:100BE0004F554E543A3120555549443A3030303003
:100BF000303030302D303030302D303030302D30FE
:100C00003030302D303030303030303030303030E7
:100C10000A004649524D574152455F4E414D453AB3
:100C20004D61726C696E2056312E302E323B20534E
:100C30007072696E7465722F6772626C206D617379
:100C400068757020666F722067656E36204649525F
:100C50004D574152455F55524C3A68747470733A1F
:100C60002F2F6769746875622E636F6D2F707275B0
:100C7000736133642F50727573612D69332D506C1D
:100C800075732F2050524F544F434F4C5F5645526F
:100C900053494F4E3A312E30204D414348494E453D
:100CA0005F545950453A507275736120693320453D
:100CB000585452554445525F434F554E543A312093
:100CC000555549443A30303030303030302D3030A6
:100CD00030302D303030302D303030302D3030301D
:100CE0003030303030303030300A00426564204FD0
:100CF0004B2E0042656420646F6E652E005A616859
:100D0000726976616E69206265642E2E2E004265DE
:100D1000642048656174696E672E005A6168726963
:100D200076616E69204F4B2E0048656174696E676D
:100D300020646F6E652E005A6168726976616E6913
:100D40002E2E2E0048656174696E672E2E2E004D82
:100D500031303920496E76616C696420657874722F
:100D60007564657220004D31303920496E76616CB2
:100D7000696420657874727564657220004E6F2016
:100D8000746865726D6973746F7273202D206E6F55
:100D90002074656D7065726174757265004E6F20A8
:100DA000746865726D6973746F7273202D206E6F35
:100DB0002074656D7065726174757265004D3232B4
:100DC0003120496E76616C6964206578747275644F
:100DD000657220004D32323120496E76616C696453
:100DE00020657874727564657220004D3231382048
:100DF000496E76616C696420657874727564657299
:100E000020004D32313820496E76616C696420656E
:100E10007874727564657220004D32303020496EEE
:100E200076616C69642065787472756465722000FF
:100E30004D32303020496E76616C6964206578747B
:100E4000727564657220004D31303520496E7661CF
:100E50006C696420657874727564657220004D3128
:100E6000303520496E76616C6964206578747275DE
:100E700064657220004D31303420496E76616C69B2
:100E80006420657874727564657220004D31303469
:100E900020496E76616C696420657874727564654A
:100EA000722000456E642066696C65206C697374FD
:100EB00000456E642066696C65206C69737400423D
:100EC0006567696E2066696C65206C6973740042A1
:100ED0006567696E2066696C65206C69737400448F
:100EE0006F6E65207072696E74696E672066696CDA
:100EF0006500446F6E65207072696E74696E67205C
:100F000066696C65004E6F204C696E65204E756D8C
:100F1000626572207769746820636865636B7375B6
:100F20006D2C204C617374204C696E653A20004E24
:100F30006F204C696E65204E756D62657220776911
:100F4000746820636865636B73756D2C204C6173E6
:100F500074204C696E653A20004E6F2043686563CB
:100F60006B73756D2077697468206C696E65206E8F
:100F7000756D6265722C204C617374204C696E65CE
:100F80003A20004E6F20436865636B73756D207760
:100F9000697468206C696E65206E756D6265722C6F
:100FA000204C617374204C696E653A20006368655B
:100FB000636B73756D206D69736D617463682C204C
:100FC0004C617374204C696E653A200063686563F8
:100FD0006B73756D206D69736D617463682C204C43
:100FE000617374204C696E653A20004C696E65200F
:100FF0004E756D626572206973206E6F74204C614E
:101000007374204C696E65204E756D6265722B316C
:101010002C204C617374204C696E653A20004C6939
:101020006E65204E756D626572206973206E6F74F7
:10103000204C617374204C696E65204E756D62653D
:10104000722B312C204C617374204C696E653A20F0
:1010500000446F6E6520736176696E672066696C07
:10106000652E00446F6E6520736176696E67206639
:10107000696C652E006F6B006F6B002020506C61F7
:101080006E6E657242756666657242797465733A12
:1010900020002020506C616E6E6572427566666538
:1010A0007242797465733A20002046726565204D5E
:1010B000656D6F72793A20002046726565204D6536
:1010C0006D6F72793A2000204C6173742055706402
:1010D000617465643A2000204C617374205570641B
:1010E000617465643A2000207C20417574686F72D9
:1010F0003A2000207C20417574686F723A200020ED
:10110000536F667477617265205265736574002051
:10111000536F667477617265205265736574002041
:101120005761746368646F6720526573657400204B
:101130005761746368646F6720526573657400203B
:1011400042726F776E206F757420526573657400FC
:101150002042726F776E206F7574205265736574CC
:10116000002045787465726E616C205265736574F9
:10117000002045787465726E616C205265736574E9
:1011800000506F776572557000506F7765725570BB
:1011900000656E717565696E67202200656E7175F8
:1011A00065696E672022002070726F2070726F6A0E
:1011B0006576656E69207A6D656E0020666F7220B7
:1011C00074616B652065666665637400526573744F
:1011D000617274756A7465207469736B61726E757F
:1011E000005265626F6F7420746865207072696E5A
:1011F000746572004D6F6420205B7679732E2076C3
:10120000796B6F6E5D004D6F6465205B6869676820
:1012100020706F7765725D004D6F64202020202064
:1012200020205B74696368795D004D6F64652020E0
:101230002020205B73696C656E745D0056796D6566
:101240006E612066696C616D656E7475210043681E
:10125000616E67696E672066696C616D656E742189
:1012600000566C6F7A74652066696C616D656E748A
:1012700000496E736572742066696C616D656E7489
:10128000004120737469736B6E65746520746C61C2
:101290006369746B6F00416E6420707265737320B4
:1012A000746865206B6E6F62005A6D656E612075A3
:1012B000737065736E6121004368616E67652073AA
:1012C000756363657373210043697374656E692088
:1012D0006261727679004C6F6164696E6720636F3A
:1012E0006C6F720050726F73696D2063656B656A15
:1012F000746500506C656173652077616974005A8C
:1013000061766164656E692066696C616D656E7495
:1013100075004C6F6164696E672066696C616D650C
:101320006E74004261727661206E656E6920636939
:1013300073746100436F6C6F72206E6F7420636C06
:101340006561720046696C616D656E74206E657AC8
:1013500061766564656E0046696C616D656E7420CA
:101360006E6F74206C6F61646564004E65004E6F33
:1013700000416E6F005965730056796D656E61208E
:101380006F6B3F004368616E67656420636F7272C4
:101390006563746C793F00506F64706F72610053C5
:1013A0007570706F72740050726564656872656AFA
:1013B000746520747279736B75210050726568656D
:1013C000617420746865206E6F7A7A6C65210043C1
:1013D000485942413A004552524F523A00526563D1
:1013E0007472616374005265637472616374005A4D
:1013F00061766573742066696C616D656E74004C0E
:101400006F61642066696C616D656E740056796AFF
:101410006D6F75742066696C616D656E7400556ED4
:101420006C6F61642066696C616D656E74005072EA
:101430006564656872657600507265686561740000
:101440004E6173746176656E690053657474696E7C
:101450006773004B616C6962726F766174205A0029
:1014600043616C696272617465205A004175746FE2
:1014700020646F6C61646974205A203F0041757468
:101480006F2061646A757374205A203F00456E6452
:1014900073746F702061626F727400456E64737450
:1014A0006F702061626F727400446F6C6164656E6E
:1014B00069206F7379205A004C6976652061646AEF
:1014C000757374205A004261627973746570205993
:1014D00000426162797374657020590042616279DB
:1014E000737465702058004261627973746570206E
:1014F00058005A204F6666736574005A204F66661E
:1015000073657400486F6D6520582F5920626566B9
:101510006F7265205A00486F6D6520582F59206200
:1015200065666F7265205A005A2070726F6265207E
:101530006F75742E20626564005A2070726F626548
:10154000206F75742E206265640056796D656E6932
:1015500074205344004368616E67652053442063E0
:1015600061726400496E69632E20534400496E69BC
:10157000742E20534420636172640056796D656E49
:1015800069742066696C616D656E74004368616E94
:1015900067652066696C616D656E74004175746F76
:1015A000526574722E004175746F526574722E000C
:1015B000556E52657420205600556E526574202079
:1015C00056005320556E5265742B6D6D0053205597
:1015D0006E5265742B6D6D00556E526574202B6DC7
:1015E0006D00556E526574202B6D6D00486F702034
:1015F0006D6D00486F70206D6D005265747261638F
:101600007420205600526574726163742020560065
:10161000537761702052652E6D6D00537761702095
:1016200052652E6D6D0052657472616374206D6D2C
:101630000052657472616374206D6D0053544F5095
:101640005045442E200053544F505045442E200006
:101650004B494C4C45442E20004B494C4C45442EA4
:1016600020004E6F206D6F76652E004E6F206D6FDF
:1016700076652E005469736B2070726572757365A0
:101680006E005072696E742061626F7274656400DE
:101690004F626E6F76656E69207469736B75005268
:1016A0006573756D696E67207072696E740057613D
:1016B000697420666F7220757365722E2E2E005726
:1016C00061697420666F7220757365722E2E2E000C
:1016D000536C6565702E2E2E00536C6565702E2E32
:1016E0002E005A61646E61205344206B61727461F4
:1016F000004E6F2053442063617264005469736B21
:10170000207A205344005072696E742066726F6DA7
:10171000205344005A61737461766974207469734C
:101720006B0053746F70207072696E7400506F6B31
:101730007261636F76617400526573756D652070B8
:1017400072696E7400506F7A617374617669742087
:101750007469736B005061757365207072696E7483
:10176000004C616469740054756E65005072697054
:1017700072617661005072657061726500496E66D3
:101780006F726D61636500496E666F207363726589
:10179000656E004F626E6F766974005265667265A1
:1017A0007368004F626E6F76697420767963686F34
:1017B0007A6900526573746F7265206661696C7333
:1017C00061666500556C6F7A69742070616D65742F
:1017D000004C6F6164206D656D6F72790053746F9A
:1017E0007265206D656D6F72790053746F7265203C
:1017F0006D656D6F7279004C434420636F6E747237
:10180000617374004C434420636F6E74726173742F
:101810000046696C2E204469612E20330046696CB5
:101820002E204469612E20330046696C2E204469C5
:10183000612E20320046696C2E204469612E2032D0
:101840000046696C2E204469612E20310046696C87
:101850002E204469612E2031004520696E206D6D77
:1018600033004520696E206D6D330046696C616DF3
:10187000656E740046696C616D656E7400506F68CA
:101880007962004D6F74696F6E005465706C6F748F
:10189000610054656D7065726174757265004573A1
:1018A000746570732F6D6D004573746570732F6D63
:1018B0006D005A73746570732F6D6D005A73746583
:1018C00070732F6D6D005973746570732F6D6D009B
:1018D0005973746570732F6D6D00587374657073F0
:1018E0002F6D6D005873746570732F6D6D00412DF1
:1018F0007265747261637400412D72657472616304
:101900007400416D61782000416D6178200056546B
:10191000726176206D696E005654726176206D6931
:101920006E00566D696E00566D696E00650065004B
:101930007A007A007900790078007800566D617835
:101940002000566D6178200056652D6A65726B0027
:1019500056652D6A65726B00567A2D6A65726B004A
:10196000567A2D6A65726B005678792D6A65726BAE
:10197000005678792D6A65726B00416363656C006F
:10198000416363656C005049442D43005049442D28
:1019900043005049442D44005049442D44005049CF
:1019A000442D49005049442D49005049442D5000D0
:1019B0005049442D50004F6666004F6666004F6EDA
:1019C00020004F6E20004175746F74656D7000418A
:1019D00075746F74656D7000200220466163740039
:1019E00020022046616374002002204D61780020AF
:1019F00002204D6178002002204D696E00200220F7
:101A00004D696E004B6F6E74726F6C6100436F6E48
:101A100074726F6C00507275746F6B203200466C7C
:101A20006F77203200507275746F6B203100466CF6
:101A30006F77203100507275746F6B203000466CE8
:101A40006F77203000507275746F6B00466C6F7743
:101A500000527963686C6F73742076656E742E0023
:101A600046616E207370656564004265640042657E
:101A70006400547279736B6133004E6F7A7A6C65CF
:101A80003300547279736B6132004E6F7A7A6C65F1
:101A90003200547279736B61004E6F7A7A6C650014
:101AA000527963686C6F737400537065656400509D
:101AB0006F73756E6F7574206F2031306D6D004DD2
:101AC0006F76652031306D6D00506F73756E6F7578
:101AD00074206F20316D6D004D6F766520316D6D16
:101AE00000506F73756E6F7574206F20302E316DDE
:101AF0006D004D6F766520302E316D6D0045787428
:101B000072756465723300457874727564657233FA
:101B10000045787472756465723200457874727528
:101B20006465723200457874727564657200457838
:101B300074727564657200506F73756E6F75742082
:101B40005A004D6F7665205A00506F73756E6F7531
:101B5000742059004D6F7665205900506F73756E73
:101B60006F75742058004D6F7665205800506F7364
:101B7000756E6F7574206F7375004D6F766520619B
:101B8000786973005265747261637400526574728F
:101B9000616374004578747275646F766174004592
:101BA000787472756465005A61706E6F7574207A0E
:101BB00064726F6A0053776974636820706F776529
:101BC00072206F6666005679706E6F7574207A6445
:101BD000726F6A0053776974636820706F776572FB
:101BE000206F6E005A63686C6164697400436F6FA4
:101BF0006C646F776E0050726564656872657620FC
:101C000041425320636F6E6600507265686561746F
:101C10002041425320636F6E6600507265646568B0
:101C200072657620414253204265640050726568B7
:101C300065617420414253204265640050726564BE
:101C400065687265762041425320416C6C00507289
:101C500065686561742041425320416C6C0050728C
:101C60006564656872657620414253203300507286
:101C70006568656174204142532033005072656489
:101C80006568726576204142532032005072656863
:101C9000656174204142532032005072656465686A
:101CA000726576204142532031005072656865614B
:101CB000742041425320310050726564656872653A
:101CC000762041425300507265686561742041423C
:101CD000530050726564656872657620504C4120EF
:101CE000636F6E66005072656865617420504C4188
:101CF00020636F6E66005072656465687265762059
:101D0000504C4120426564005072656865617420E2
:101D1000504C41204265640050726564656872658C
:101D20007620504C4120416C6C00507265686561B2
:101D30007420504C4120416C6C00507265646568A1
:101D400072657620504C41203300507265686561A1
:101D50007420504C41203300507265646568726590
:101D60007620504C412032005072656865617420C5
:101D7000504C41203200507265646568726576206F
:101D8000504C412031005072656865617420504CA0
:101D90004120310050726564656872657620504C50
:101DA00041005072656865617420504C41004E617D
:101DB0007374617620706F636174656B0053657432
:101DC000206F726967696E004E617374617620706E
:101DD0006F636174656B20686F6D65005365742077
:101DE000686F6D65206F6666736574730041757406
:101DF0006F20686F6D65004175746F20686F6D6549
:101E0000005679706E6F7574206D6F746F72790003
:101E100044697361626C6520737465707065727378
:101E2000004175746F7374617274004175746F73DF
:101E30007461727400486C61766E69206E616269CB
:101E4000646B61004D61696E004B61727461207654
:101E5000796A6D75746100436172642072656D6F9B
:101E6000766564004B6172746120766C6F7A656E82
:101E700061004361726420696E7365727465640009
:101E80005072757361206933207072697072617667
:101E9000656E6100507275736120693320726561EF
:101EA00064792E004D383420582059205A2045009E
:101EB0004D3234004D3233202573006175746F2527
:101EC000692E67000A002F000A002E0044656C6529
:101ED00074696F6E206661696C65642C2046696C5C
:101EE000653A200046696C652064656C65746564BC
:101EF0003A002E002E002E002E004E6F77206672C4
:101F00006573682066696C653A20004E6F772064BF
:101F10006F696E672066696C653A20002220706FD9
:101F200073002220706172656E743A22005355422C
:101F3000524F5554494E452043414C4C20746172D8
:101F40006765743A2200747279696E6720746F2035
:101F500063616C6C207375622D67636F64652066C6
:101F6000696C6573207769746820746F6F206D6188
:101F70006E79206C6576656C732E204D4158206C0F
:101F80006576656C2069733A000000211042206379
:101F9000308440A550C660E770088129914AA16B42
:101FA000B18CC1ADD1CEE1EFF131121002733252DA
:101FB00022B5529442F772D662399318837BB35A92
:101FC000A3BDD39CC3FFF3DEE362244334200401AA
:101FD00014E664C774A44485546AA54BB5288509E2
:101FE00095EEE5CFF5ACC58DD5533672261116307A
:101FF00006D776F6669556B4465BB77AA719973832
:1020000087DFF7FEE79DD7BCC7C448E5588668A7B9
:10201000784008611802282338CCC9EDD98EE9AF81
:10202000F9488969990AA92BB9F55AD44AB77A9619
:102030006A711A500A333A122AFDDBDCCBBFFB9ED1
:10204000EB799B588B3BBB1AABA66C877CE44CC5E9
:102050005C222C033C600C411CAEED8FFDECCDCD21
:10206000DD2AAD0BBD688D499D977EB66ED55EF4B9
:102070004E133E322E511E700E9FFFBEEFDDDFFC71
:10208000CF1BBF3AAF599F788F8891A981CAB1EB16
:10209000A10CD12DC14EF16FE18010A100C230E33F
:1020A000200450254046706760B9839893FBA3DAFB
:1020B000B33DC31CD37FE35EF3B1029012F322D28F
:1020C000323542145277625672EAB5CBA5A895898B
:1020D000856EF54FE52CD50DC5E234C324A01481DF
:1020E000046674476424540544DBA7FAB79987B89B
:1020F000975FE77EF71DC73CD7D326F2369106B02F
:102100001657667676154634564CD96DC90EF92F9A
:10211000E9C899E9898AB9ABA9445865480678277E
:1021200068C018E1088238A3287DCB5CDB3FEB1E3A
:10213000FBF98BD89BBBAB9ABB754A545A376A16CE
:102140007AF10AD01AB32A923A2EFD0FED6CDD4DCA
:10215000CDAABD8BADE89DC98D267C076C645C451E
:102160004CA23C832CE01CC10C1FEF3EFF5DCF7CDA
:10217000DF9BAFBABFD98FF89F176E367E554E746E
:102180005E932EB23ED10EF01E22004D3232302030
:1021900053256900203A2000004C414E472053450A
:1021A0004C20464F52434544002200205A3A00201A
:1021B000593A0020453A00205A3A0020593A00582E
:1021C0003A0020002E0020423A0020453A00543ABE
:1021D0000020573A0020453A00543A002042403A45
:1021E0000020403A00202F003A00205400202F0009
:1021F00020423A00202F006F6B20543A00256920BE
:102200006D696E2C2025692073656300256920683F
:102210006F757273202569206D696E757465730022
:102220004D313130004D3239004665622031392060
:102230003230313600436F6D70696C65643A20004E
:10224000286E6F6E652C2064656661756C74206302
:102250006F6E666967290046656220313920323029
:1022600031362031373A34363A323900737461727C
:10227000740022002200FFFFFF0000A0400000A029
:10228000400000004000005643000046431FC54880
:102290004300000000000000001F856B3E00005658
:1022A00043000046430000494300000000000000D6
:1022B000001F856B3E6563686F3A004572726F72EE
:1022C0003A00473120453430204631303000473124
:1022D000204537302046343030004D383300473108
:1022E00020452D38302046343030004D3833002D15
:1022F0002D3A2D2D002D2D2D0053440001200001DD
:1023000020004D36303000464C4558202D202032DC
:1023100033302F35300050502020202D20203235F2
:10232000342F3130300048495053202D2020323294
:10233000302F3130300050455420202D20203234B1
:10234000302F393000504C4120202D2020323130A8
:102350002F35300041425320202D20203235352F9B
:10236000313030004D3834004D3834205820592059
:102370005A2045004D3234004D3233202573005829
:102380000059005A004578747275646572004732CE
:1023900038004D383400473238205A004533442D38
:1023A00076360052414D426F2D31306100312D376C
:1023B000356D6D002D2D2D2D2D2D2D2D2D2D2D2DF2
:1023C000004669726D77617265202D20322E322EA3
:1023D000330048617264636F6465642044656661BC
:1023E000756C742053657474696E6773204C6F61EB
:1023F0006465640046696C616D656E742073657414
:1024000074696E67733A2044697361626C65640035
:102410002020204D32303020440046696C616D65CB
:102420006E742073657474696E67733A002020209F
:102430004D3230392053004175746F2D52657472DE
:102440006163743A20533D3020746F206469736176
:10245000626C652C203120746F20696E7465727017
:1024600072657420657874727564652D6F6E6C7911
:10247000206D6F766573206173207265747261637D
:102480007473206F72207265636F7665726965730D
:10249000002046002020204D323038205300526565
:1024A000636F7665723A20533D4578747261206C93
:1024B000656E67746820286D6D2920463A537065F3
:1024C000656420286D6D2F6D2900205A002046007C
:1024D0002020204D323037205300526574726163E2
:1024E000743A20533D4C656E67746820286D6D29E1
:1024F00020463A537065656420286D6D2F6D292044
:102500005A3A205A4C69667420286D6D290020447F
:10251000002049002020204D333031205000504908
:10252000442073657474696E67733A00205A002002
:10253000590020204D323036205800486F6D6520FC
:102540006F666673657420286D6D293A002045001A
:10255000205A0020580020420020540020204D32F4
:102560003035205300416476616E63656420766186
:10257000726961626C65733A20533D4D696E2066E5
:102580006565647261746520286D6D2F73292C2038
:10259000543D4D696E2074726176656C2066656588
:1025A000647261746520286D6D2F73292C20423D63
:1025B0006D696E696D756D207365676D656E7420EC
:1025C00074696D6520286D73292C20583D6D6178E4
:1025D000696D756D205859206A65726B20286D6D84
:1025E0002F73292C20205A3D6D6178696D756D20FF
:1025F0005A206A65726B20286D6D2F73292C20205C
:10260000453D6D6178696D756D2045206A65726B19
:1026100020286D6D2F73290020540020204D32306A
:1026200034205300416363656C65726174696F6E39
:102630003A20533D616363656C65726174696F6EC6
:102640002C20543D7265747261637420616363650C
:102650006C65726174696F6E00204500205A00201D
:10266000590020204D3230312058004D6178696D7D
:10267000756D20416363656C65726174696F6E206E
:10268000286D6D2F7332293A00204500205A002012
:10269000590020204D3230332058004D6178696D4B
:1026A000756D2066656564726174657320286D6D53
:1026B0002F73293A00204500205A0020590020207D
:1026C0004D39322058005374657073207065722044
:1026D000756E69743A0045303A20005A3A20005924
:1026E0003A2000583A20004D53312C4D533220509F
:1026F000696E730A005A00205A3A00590020593A6C
:1027000000580020583A0024F4D43050C38E20C220
:10271000A24017828B7011127A910D816CD90AA890
:1027200061E108C7586607615143061E4B5D05C14C
:1027300045A7041A411104093D980371393103403A
:1027400036DB0265339102D4305402802E1D0263C1
:102750002CEE01752AC501B028A001102781018F38
:102760002564012B244B01E0223401AC211F018D93
:10277000200D01801FFC00841EED00971DDF00B8B6
:102780001CD200E61BC600201BBC00641AB200B2BB
:1027900019A8000A19A0006A189900D117910040E1
:1027A000178B00B516840031167E00B31579003AF8
:1027B000157300C7146F0058146A00EE1366008882
:1027C00013630025135E00C7125B006C12570015DF
:1027D000125400C111510070114F0021114B00D64D
:1027E0001049008D1047004610440002104200C0FE
:1027F0000F4000800F3E00420F3C00060F3B00CB15
:102800000E3800930E37005C0E3500270E3400F3AF
:102810000D3200C10D3100900D3000600D2E0032E0
:102820000D2D00050D2C00D90C2B00AE0C290085B8
:102830000C29005C0C2700350C27000E0C2600E844
:102840000B2400C40B2400A00B23007D0B23005A93
:102850000B2100390B2100180B2000F80A1F00D9AA
:102860000A1E00BB0A1E009D0A1D00800A1D00638F
:102870000A1C00470A1B002C0A1B00110A1A00F749
:10288000091A00DD091900C4091900AB09190092E1
:102890000917007B091800630917004C0916003658
:1028A000091600200916000A091500F5081500E0B0
:1028B000081400CC081400B8081400A408140090F0
:1028C0000813007D0812006B081300580812004618
:1028D0000812003408110023081100120811000129
:1028E000081100F0071000E0071000D0071000C02A
:1028F000071000B0070F00A107100091070E00831A
:10290000070F0074070F0065070E0057070E0049F8
:10291000070E003B070D002E070E0020070D0013C9
:10292000070D0006070D00F9060C00ED060D00E08E
:10293000060C00D4060C00C8060C00BC060C00B047
:10294000060C00A4060B0099060C008D060B0082F5
:10295000060B0077060B006C060B0061060A005799
:10296000060B004C060A0042060A0038060A002E32
:10297000060A0024060A001A060A001006090007C3
:10298000060A00FD050900F4050900EB050900E24F
:10299000050900D9050900D0050900C7050900BED1
:1029A000050900B5050800AD050800A50509009C4E
:1029B000050800940508008C050800840508007CC3
:1029C000050800740508006C050700650508005D32
:1029D000050700560508004E05070047050700409B
:1029E00005080038050700310507002A0507002300
:1029F0000507001C050600160507000F050700085F
:102A000005060002050700FB040600F5040700EEBA
:102A1000040600E8040600E2040700DB040600D513
:102A2000040600CF040600C9040600C3040600BD66
:102A3000040600B7040600B1040500AC040600A6B5
:102A4000040600A00405009B040600950405009000
:102A50000406008A04050085040500800406007A47
:102A600004050075040500700405006B040500668C
:102A7000040500610405005C0405005704050052CC
:102A80000405004D04050048040500430405003E0C
:102A90000404003A04050035040500300404002C49
:102AA00004050027040400230405001E0404001A82
:102AB00004040016040500110404000D04040009B8
:102AC0000405000404040000040400FC030400F8EE
:102AD000030400F4030400F0030400EC030400E822
:102AE000030400E4030400E0030400DC030400D852
:102AF000030400D4030400D0030400CC030400C882
:102B0000030300C503030024F404D9201BC40C5C98
:102B10000E9804C4095F0265077101F405F900FB12
:102B200004B30048048700C103690058035500033B
:102B3000034500BE023A008402310053022A0029F4
:102B400002250004022000E4011C00C8011900AFA6
:102B50000117009801140084011300710110006135
:102B600001100051010E0043010D0036010B002B36
:102B7000010B0020010B00150109000C01090003E5
:102B8000010800FB000800F3000800EB000700E468
:102B9000000600DE000600D8000600D2000600CCC9
:102BA000000500C7000500C2000500BD000400B913
:102BB000000400B5000400B1000400AD000400A949
:102BC000000400A5000300A20003009F0004009B76
:102BD000000300980003009500020093000300909A
:102BE0000003008D0002008B0003008800020086B5
:102BF00000020084000300810002007F0002007DCB
:102C00000002007B000200790002007700010076DC
:102C10000002007400020072000100710002006FE7
:102C20000002006D0001006C0002006A00010069F2
:102C300000020067000100660001006500010064F9
:102C40000002006200010061000100600001005FFD
:102C50000002005D0001005C0001005B0001005A01
:102C60000001005900010058000100570001005602
:102C70000001005500010054000100530000005302
:102C80000001005200010051000100500001004FFE
:102C90000001004E0000004E0001004D0001004CFC
:102CA0000001004B0000004B0001004A00010049F8
:102CB00000010048000000480001004700010046F4
:102CC00000000046000100450000004500010044EE
:102CD00000010043000000430001004200000042E8
:102CE0000001004100000041000100400001003FE0
:102CF0000000003F0001003E0000003E0001003DDA
:102D00000000003D0001003C0000003C0000003CD1
:102D10000001003B0000003B0001003A0000003AC7
:102D200000010039000000390001003800000038BF
:102D300000000038000100370000003700010036B5
:102D400000000036000000360001003500000035AC
:102D500000000035000100340000003400000034A1
:102D60000001003300000033000000330001003296
:102D7000000000320000003200010031000000318C
:102D80000000003100010030000000300000003081
:102D90000001002F0000002F0000002F0000002F76
:102DA0000001002E0000002E0000002E0001002D6A
:102DB0000000002D0000002D0000002D0001002C5F
:102DC0000000002C0000002C0000002C0001002B53
:102DD0000000002B0000002B0000002B0001002A47
:102DE0000000002A0000002A0000002A000100293B
:102DF000000000290000002900000029000000292F
:102E00000001002800000028000000280000002821
:102E10000000002800010027000000270000002714
:102E20000000002700000027000100260000002607
:102E300000000026000000260000002600010025FA
:102E400000000025000000250000002500000025EE
:102E500000000025000100240000002400000024E0
:102E600000000024000000240001002300000023D3
:102E700000000023000000230000002300000023C6
:102E800000000023000100220000002200000022B8
:102E900000000022000000220000002200010021AA
:102EA000000000210000002100000021000000219E
:102EB000000000210000002100010020000000208F
:102EC0000000002000000020000000200000002082
:102ED00000000020000000200001001F0000001F73
:102EE0000000001F0000001F0000001F0000001F66
:102EF0000000001F0001001E0000001E0000001E58
:102F00000000001E0000000000090A02080B0C0D62
:102F1000070603040100000000000000000000009C
:102F200000000000000000000000000000000000A1
:102F300000000011100F0000000000000000000061
:102F40000000000000000000000000000000000081
:102F5000000000000000000000000000000102105E
:102F600020200808102040102040800201020108A3
:102F70000402010102040810204080804020100853
:102F800004020180040201804020100804020108AC
:102F9000040201010204081020408001020408100C
:102FA0002040801008040880102040044080102039
:102FB0004004800505050507050808080802020207
:102FC000020A0A08080404040401010101010101C4
:102FD000010303030303030303040707070C0C0C9B
:102FE0000C0C0C0C0C020202020606060606060673
:102FF000060B0B0B0B0B0B0B0B07070A0A0A0A0A33
:103000000A05050504040408080000200023002622
:103010000029002C002F00320000010000030106EF
:1030200001090100002200250028002B002E00319C
:1030300000340002010000050108010B010000211D
:1030400000240027002A002D003000330001010079
:1030500000040107010A01024E414E494E495459EC
:10306000494E46CDCCCC3D0AD7233C17B7D1387753
:10307000CC2B329595E6241FB14F0A000020410069
:1030800000C84200401C4620BCBE4CCA1B0E5AAEB3
:10309000C59D74007C72EF8CC2BF807211241FBE6C
:1030A000CFEFD1E2DEBFCDBF00E00CBF17E0A0E064
:1030B000B2E0EAE4F6EA01E00BBF02C007900D922D
:1030C000A23FB107D9F727E1A2EFB7E001C01D92F7
:1030D000A730B207E1F710E3CAE9D0E300E006C089
:1030E00022970109FE010BBF0E94ADCCC439D10764
:1030F00080E00807A9F70E94C6C30C9414D30C946F
:103100000000CF93DF93EC019C012C5F3F4F41E027
:1031100050E060E070E0898D9A8D0E94232388231F
:1031200099F04D895E896F89788D452B462B472B09
:1031300059F44C815D816E817F814D8B5E8B6F8BED
:10314000788F998190689983DF91CF910895CF927C
:10315000DF92EF92FF920F931F93CF93DF93EC01D7
:1031600089899A89AB89BC89803E9F4FAF41B1055F
:1031700010F080E06BC0CE01C4DF8823D1F30E9441
:103180003721182F8823A9F3E98DFA8DCC80DD80B3
:10319000EE80FF8032E0C31AD108E108F10805840F
:1031A00004C0CC0CDD1CEE1CFF1C0A94D2F78685F3
:1031B0009785A089B189C80ED91EEA1EFB1E81E041
:1031C0008093F807C092FB09D092FC09E092FD09B8
:1031D000F092FE0980E092E0EBEFF7E0DF019C0166
:1031E0001D9221503040E1F701E0E98DFA8D848194
:1031F000081790F42BEF37E0B701A601400F511DDF
:10320000611D711D8091F9079091FA070E94F246A5
:103210008823E1F00F5FE9CFC12C82E0D82EE12CAA
:10322000F12C058404C0CC0CDD1CEE1CFF1C0A94A0
:10323000D2F749895A896B897C894C0D5D1D6E1DB9
:103240007F1D498B5A8B6B8B7C8B812FDF91CF91AC
:103250001F910F91FF90EF90DF90CF900895CF9343
:10326000DF93EC0141E0611101C040E06C857D8598
:103270008E859F850E947721882341F0888920E2EE
:10328000829FC00111248550984F02C080E090E0D9
:10329000DF91CF91089530E020E04EE2DC015C91B7
:1032A000503271F0383029F4FB01E20FF11D4083F8
:1032B0002F5FFB01E20FF11DDC015C9150832F5F5A
:1032C0003F5F01963B3051F7FB01E20FF11D108289
:1032D0000895CF93DF93EB01FC012381211102C0FC
:1032E00080E00EC02250223020F48FE288831982C1
:1032F00006C060E0B4DF009799F3BE01CCDF81E047
:10330000DF91CF910895FB012BE030E23193215002
:10331000E9F7DC0190E027E03A2FEB2F8D91811146
:103320000AC0DA013C931196EC9381E0FB01908195
:10333000903239F525C08F32A1F38E3219F0EAE8C8
:10334000F1E008C02A30E1F098E02AE0E5CF3196BC
:103350003817B1F034913111FACF291788F03FEDC9
:10336000380F3E3568F431E0390FFB01E90FF11DEC
:103370009FE9980F9A3108F480528083932FCCCF25
:1033800080E008950F931F93CF93DF93EC018B019F
:103390008B81882311F080E042C0FB018789803156
:1033A00039F18032C1F783E08B83F801428D538D70
:1033B000648D758D4D8B5E8B6F8B788F9E012F5E2C
:1033C0003F4FC8010E942E22882329F31A8F098FAC
:1033D00081E089831C821D821E821F8218861986C5
:1033E0001A861B861C861D861E861F86188A17C095
:1033F00082E08B831D8A1E8A1F8A188EFB01408DF6
:10340000518D60E070E095E0440F551F661F771FF7
:103410009A95D1F7498B5A8B6B8B7C8BD7CFDF91E9
:10342000CF911F910F9108952F923F924F925F92EB
:103430006F927F928F929F92AF92BF92CF92DF92C4
:10344000EF92FF920F931F93CF93DF93EC015B01F9
:103450006A018B81811103C08FEF9FEFC7C0898103
:1034600080FFFACF49895A896B897C89888599853B
:10347000AA85BB852601612C712C8A019B01081B42
:10348000190B2A0B3B0B401651066206730618F007
:103490006A01C81AD90A76013E0124E0620E711C45
:1034A000E114F10409F476C0488559856A857B8565
:1034B0004A0181E098222B811A012B01E9E0569400
:1034C000479437942794EA95D1F7898D9A8DFC011A
:1034D000223049F4628D738D848D958D620D731D3C
:1034E000841D951D3CC0148111501221811491043A
:1034F000C1F4111116C0452B462B472B49F48D8979
:103500009E89AF89B88D8C839D83AE83BF8309C0AC
:103510004C815D816E817F81930121D7882309F4DD
:103520009BCFE98DFA8D6C817D818E819F81625068
:10353000710981099109058404C0660F771F881FEE
:10354000991F0A94D2F72685378540895189620FE1
:10355000731F841F951F610F711D811D911D20E038
:1035600032E02819390987012E153F0508F4890131
:103570000115F2E01F0769F52091FB093091FC0964
:103580004091FD095091FE09621773078407950762
:1035900019F41FC0C6012AC09501AB01BC0180917E
:1035A000F9079091FA070E947D46882309F454CFC9
:1035B000A00EB11E88859985AA85BB85800F911FB5
:1035C000A11DB11D88879987AA87BB87E01AF10AD8
:1035D00067CF40E08CD6882309F43ECFB401655014
:1035E000784FA801C5010E94D3CFE2CFDF91CF91E0
:1035F0001F910F91FF90EF90DF90CF90BF90AF9011
:103600009F908F907F906F905F904F903F902F9002
:103610000895CF93DF931F92CDB7DEB741E050E01E
:10362000BE016F5F7F4F00DF019719F4898190E041
:1036300002C08FEF9FEF0F90DF91CF910895CF924F
:10364000DF92EF92FF920F931F93CF93DF936C0162
:10365000EB017A01FC018381823060F000851185E5
:10366000228533850F71112722273327012B022B47
:10367000032B11F08FEF5CC04115510511F0F701DC
:1036800010821DE040E250E0BE01C601CDDE803276
:10369000910539F021E0892B09F420E0822F8195F2
:1036A00047C028812223C1F0253E61F32E3251F319
:1036B0003B853F733F3061F4E114F10449F04A8DDA
:1036C0005B8D452B29F42F713FEF320F343030F0F2
:1036D0002B8523FDD7CF2CC080E02AC030E02150BD
:1036E0003109129FC001139F900D1124F701E80FBB
:1036F000F91F298120832B8121832D8122832F8112
:103700002383298524832E852583288926832A8956
:1037100027832C8920872E892187288D22872C8D2D
:1037200023872E8D2487288126FFD2CF1586D0CFE0
:10373000DF91CF911F910F91FF90EF90DF90CF908D
:1037400008951F93CF93DF93EC018B81823018F49F
:1037500080E090E023C0488559856A857B85A5E097
:103760007695679557954795AA95D1F7142F1F70B1
:10377000CE014FDF97FDECCF488559856A857B8563
:10378000415E5F4F6F4F7F4F488759876A877B87BE
:1037900020E2129FC00111248550984FDF91CF91F4
:1037A0001F9108954F925F926F927F92AF92BF9256
:1037B000CF92DF92EF92FF920F931F93CF93DF93FD
:1037C000EC016A017B012B81222349F089899A89C6
:1037D000AB89BC8984179507A607B70710F480E06A
:1037E0006BC0223009F463C0C114D104E104F104B8
:1037F00049F41C821D821E821F82188619861A8631
:103800001B8659C088859985AA85BB85E98DFA8D67
:10381000E585F0E03996AC01BD01415051096109DF
:1038200071090E2E04C076956795579547950A94B1
:10383000D2F797018601015011092109310904C00D
:103840003695279517950795EA95D2F7041715072A
:103850002607370720F0892B8A2B8B2B49F48D897B
:103860009E89AF89B88D8C839D83AE83BF8304C04E
:10387000041B150B260B370B280139015E0184E070
:10388000A80EB11C411451046104710481F04C81F3
:103890005D816E817F819501898D9A8D60D591E0E2
:1038A000491A5108610871088111ECCF05C0C8861A
:1038B000D986EA86FB8681E0DF91CF911F910F9137
:1038C000FF90EF90DF90CF90BF90AF907F906F9080
:1038D0005F904F9008950F931F93CF93DF93EC0168
:1038E0008B818823D1F1898187FF32C061E0CE01CD
:1038F000B6DC8C01009789F1FC018081853E69F17D
:103900008B81823040F449895A896B897C89448F44
:10391000558F668F778F4D895E896F89788DF80115
:10392000538F428F758B648BE091F207F091F30710
:10393000309759F0B8016A5E7F4FC80148961995D3
:10394000F801808D918D938B828B89818F7789830C
:10395000DF91CF911F910F918AC481E0888380E02D
:10396000DF91CF911F910F910895CF93DF93EC01D9
:10397000B2DF1B82DF91CF910895FC0123812111D9
:10398000F4CF08954F925F926F927F92AF92BF9261
:10399000CF92DF92EF92FF920F931F93CF93DF931B
:1039A00000D01F92CDB7DEB75C016A017B01FC013C
:1039B00083818130E9F4818181FF1AC0F501818919
:1039C0009289A389B48984179507A607B70780F061
:1039D000892B8A2B8B2B09F472C0F501408451840A
:1039E00062847384B701A601C501DCDE811102C0C7
:1039F00080E066C0F501818D928DC114D104E1048F
:103A0000F10469F4458956896789708D25D7882323
:103A100079F3F501158A168A178A108E37C0F501D9
:103A200044815581668177819E012F5F3F4F97D4F6
:103A30008823F1F249815A816B817C81F501818D66
:103A4000928DFC012789203139F4483FFFEF5F0751
:103A500061057105D8F407C0483F2FEF5207620790
:103A60002FE0720798F4F8D6882309F4C1CFF50146
:103A700044815581668177810FEF1FEF2FEF3FE083
:103A8000818D928D51D5882309F4B2CFF501C18A79
:103A9000D28AE38AF48A818180688183C5011BDF31
:103AA000882309F4A5CFB701A6014C145D046E0468
:103AB0007F0410F4B301A201C50174DE01C081E0EE
:103AC0000F900F900F900F90DF91CF911F910F915A
:103AD000FF90EF90DF90CF90BF90AF907F906F906E
:103AE0005F904F900895FF920F931F93CF93DF93B2
:103AF000EC01F42E80E2689FF0011124E550F84FAC
:103B00008385817121F0842F827109F04EC08091EC
:103B1000FB099091FC09A091FD09B091FE098C87E9
:103B20009D87AE87BF87688B4489558960E070E0C8
:103B3000BA0155274427028D138D20E030E0402B39
:103B4000512B622B732B4D8B5E8B6F8B788F838504
:103B5000887151F4048D158D268D378D098B1A8B44
:103B60002B8B3C8B81E00BC08031F9F49E012F5EE2
:103B70003F4F898D9A8D72D48823B9F084E08B836E
:103B80008F2D8F7089831C821D821E821F82188652
:103B900019861A861B86F4FE0BC040E050E0BA017D
:103BA000CE01F0DE811104C011C01B8280E00EC086
:103BB000F5FE0BC049895A896B897C89CE01DF915A
:103BC000CF911F910F91FF90EDCD81E0DF91CF91CB
:103BD0001F910F91FF900895AF92BF92CF92DF9205
:103BE000EF92FF920F931F93CF93DF937C01EB0132
:103BF0006A01B22E898D9A8DF701928F818F40E0F4
:103C000050E0BA01CE01CEDDA12C088519852A85A8
:103C10003B8589899A89AB89BC89081719072A07C6
:103C20003B07A0F585E036952795179507958A956A
:103C3000D1F70F70CE0185DD009709F481C0FC013A
:103C40002081222311F0253EB9F4A1100EC040912D
:103C5000FB095091FC096091FD097091FE09F70183
:103C60004487558766877787008BFC018081AA246B
:103C7000A3948111CACF0AC04BE050E0BC01C60139
:103C80000E94C6CF892B09F0C0CF58C08B2D8274FB
:103C9000823409F055C0AA2049F0F701008961E09B
:103CA000C701DDDAEC01009769F44AC08B818230EC
:103CB00009F446C0CE014BDA882309F441C0CBEFAA
:103CC000D7E000E080E2FE0111928A95E9F78BE0EF
:103CD000F601DE0101900D928A95E1F7E091F2077D
:103CE000F091F307309739F0BE01625F7F4FCE014C
:103CF0004096199508C081E298E2998B888B80E004
:103D000098E09F878E87888999899B8B8A8B998F6A
:103D1000888F8E859F859F8B8E8BA9D2882381F07B
:103D20004B2D602FC701DF91CF911F910F91FF9015
:103D3000EF90DF90CF90BF90AF90D5CEB7FEF0CF91
:103D400080E0DF91CF911F910F91FF90EF90DF9076
:103D5000CF90BF90AF9008953F924F925F926F9235
:103D60007F928F929F92AF92BF92CF92DF92EF920B
:103D7000FF920F931F93CF93DF93CDB7DEB7C3545A
:103D8000D1090FB6F894DEBF0FBECDBF5C016B0149
:103D900024965FAF4EAF2497522E1C8E1F8E198231
:103DA0001C826115710511F410E073C0FC01838160
:103DB0008111FACF2496EEADFFAD249780818F322A
:103DC00011F076011DC02496EEADFFAD24978081E1
:103DD0008F3231F431962496FFAFEEAF2497F3CFB4
:103DE000F60183818250823060F3F601618D728D1D
:103DF000CE010196C7DA8823B9F2CE0101967C0183
:103E00008E01045E1F4F3801FE0131964F01402E96
:103E1000312E19C08823A9F121E0AE01495C5F4F22
:103E2000B701C801D9DE882309F4BECFEC14FD0424
:103E300011F0C7019ADD0615170501F1942D832DA8
:103E40007801092F182FAE014E5B5F4FBE01695CF0
:103E50007F4F24968EAD9FAD249755DA882309F4C1
:103E6000A3CF2496EEADFFAD249780818F3291F6DB
:103E700031962496FFAFEEAF2497F3CF982D892D7E
:103E8000DFCF252DAE01495C5F4FB701C501A4DE30
:103E9000182FCE01019671DDCE014C966EDD812F7B
:103EA000CD5BDF4F0FB6F894DEBF0FBECDBFDF9105
:103EB000CF911F910F91FF90EF90DF90CF90BF9027
:103EC000AF909F908F907F906F905F904F903F90BA
:103ED0000895CF93DF93EC0140E050E0BA0152DD4A
:103EE000882361F061E0CE01BAD9009739F025EE60
:103EF000FC0120831B82DF91CF91B9C180E0DF916B
:103F0000CF9108951F93CF93DF93CDB7DEB76B9713
:103F10000FB6F894DEBF0FBECDBFAB0119821C8275
:103F200022E0BC01CE01019617DF182F882321F073
:103F3000CE010196CEDF182FCE0101961EDD812F16
:103F40006B960FB6F894DEBF0FBECDBFDF91CF9159
:103F50001F9108952F923F924F925F926F927F929E
:103F60008F929F92AF92BF92CF92DF92EF92FF9289
:103F70000F931F93CF93DF9300D01F921F92CDB763
:103F8000DEB78C015B013A01DC0113968C9113972B
:103F90008130C1F411968C9181FF14C082FF18C04A
:103FA000F801418952896389748980859185A28548
:103FB000B38584179507A607B70751F0C801F2DB50
:103FC000811106C081E0F80180838FEF9FEF37C138
:103FD000630183C0D80159968D919C915A97FC0139
:103FE000F481F1501A012B0169E0569447943794FB
:103FF00027946A95D1F7F221FD834A0121E09222AC
:10400000FF2309F476C080E092E0881999097601CF
:104010008C159D0508F47C01D8015996ED91FC9111
:104020005A9714962D903D904D905C901797B2E062
:104030002B1A310841085108058404C0220C331C96
:10404000441C551C0A94D2F786859785A089B189AE
:10405000280E391E4A1E5B1EED812E0E311C411C9E
:10406000511CE114F2E0FF0609F089C08091FB09C0
:104070009091FC09A091FD09B091FE09821593056C
:10408000A405B50569F41092F8078FEF9FEFDC01E6
:104090008093FB099093FC09A093FD09B093FE095E
:1040A0009501B201A1018091F9079091FA070E9450
:1040B000F246882309F486CFF80180859185A28590
:1040C000B3858E0D9F1DA11DB11D80879187A2878D
:1040D000B387AE0CBF1CCE18DF08D80118964D91DF
:1040E0005D916D917C911B97C114D10409F072CF41
:1040F0007AC08114910409F086CF14964D915D9198
:104100006D917C911797411551056105710559F421
:1041100055968D919D910D90BC91A02D0097A10574
:10412000B10539F520C09E012F5F3F4F18D188237C
:1041300009F448CF89819A81AB81BC81F801218D36
:10414000328DF9012789203139F4883FFFEF9F072D
:10415000A105B10540F40DC0883F2FEF9207A207DB
:104160002FE0B20730F0C8010E94811881114BCFB7
:1041700029CFF80184839583A683B78344CF811424
:10418000910411F5D80118964D915D916D917C9136
:104190001B9751968D919D910D90BC91A02D481724
:1041A00059076A077B0780F062D0882309F40ACF99
:1041B00081E08093F8072092FB093092FC0940923D
:1041C000FD095092FE0907C041E0C201B1018FD044
:1041D000882309F4F7CEA701B501C4018550984F93
:1041E0000E94D3CF69CF51968D919D910D90BC9136
:1041F000A02DF801218184179507A607B70738F489
:10420000418B528B638B748B206821830CC080910F
:10421000F2079091F307892B31F06114710419F0C2
:104220002068F8012183D80111968C9183FD02C08A
:10423000C30105C0C8014FDB8111FACFC3CE0F9077
:104240000F900F900F900F90DF91CF911F910F91D2
:10425000FF90EF90DF90CF90BF90AF909F908F90A6
:104260007F906F905F904F903F902F900895CF93E5
:104270008091F8078823B9F14091FB095091FC091E
:104280006091FD097091FE092BEF37E08091F907ED
:104290009091FA070E94F246C82F811102C0C0E037
:1042A00023C04091F4075091F5076091F607709193
:1042B000F707411551056105710591F02BEF37E0C6
:1042C0008091F9079091FA070E94F246882339F30A
:1042D0001092F4071092F5071092F6071092F70764
:1042E0001092F80701C0C1E08C2FCF910895CF92B2
:1042F000DF92EF92FF92CF936B017C01C42F8091EC
:10430000FB099091FC09A091FD09B091FE098C1563
:104310009D05AE05BF05C9F0AADF811102C080E08E
:1043200018C02BEF37E0B701A6018091F9079091F3
:10433000FA070E947D46882391F3C092FB09D09230
:10434000FC09E092FD09F092FE0981E0C111809321
:10435000F807CF91FF90EF90DF90CF9008958F9264
:104360009F92AF92BF92CF92DF92EF92FF920F9304
:104370001F93CF93DF93EC016A017B01890189854B
:104380009A85AB85BC850196A11DB11D8417950743
:10439000A607B70710F480E054C08F89803129F454
:1043A0009927872F762F652F0BC08032A1F7CB017D
:1043B000BA0127E096958795779567952A95D1F765
:1043C0008B889C88AD88BE88680D791D8A1D9B1DD1
:1043D0008090FB099090FC09A090FD09B090FE0927
:1043E000681579058A059B0581F48F89803191F4E0
:1043F000DD24EE24FF24F601EE0FFF1FE550F84FF9
:1044000080819181A0E0B0E016C040E070DF8111B2
:10441000ECCFC1CFE894C7F8DD24EE24FF24F601E9
:10442000EE0FFF1FEE0FFF1FE550F84F80819181C7
:10443000A281B381BF70F80180839183A283B3838B
:1044400081E0DF91CF911F910F91FF90EF90DF906E
:10445000CF90BF90AF909F908F9008954F925F92B2
:104460006F927F92AF92BF92CF92DF92EF92FF92C4
:104470000F931F93CF93DF9300D01F92CDB7DEB77A
:104480008C0149835A836B837C835901C12CD12CC5
:104490007601412C42E0542E612C712C49815A81C5
:1044A0006B817C819E012F5F3F4FC80158DF8823BD
:1044B00041F1D301C201F801058404C0880F991F9E
:1044C000AA1FBB1F0A94D2F7C80ED91EEA1EFB1EF4
:1044D00049815A816B817C818789803139F481E0FF
:1044E000483F5F4F6105710538F4D8CF81E0483F00
:1044F0005F4F6F4F7F4090F2F501C082D182E28220
:10450000F3820F900F900F900F90DF91CF911F913A
:104510000F91FF90EF90DF90CF90BF90AF907F9082
:104520006F905F904F9008954F925F926F927F923D
:104530008F929F92AF92BF92CF92DF92EF92FF92B3
:104540000F931F93CF93DF93EC014A015B01280186
:104550003901423051056105710508F462C0498591
:104560005A856B857C854F5F5F4F6F4F7F4F481536
:1045700059056A057B0508F454C08F89803129F4F8
:10458000FF24EB2CDA2CC92C0CC0803209F049C076
:104590007501640177E0F694E794D794C7947A950F
:1045A000D1F74B895C896D897E89C40ED51EE61EC4
:1045B000F71E41E0C701B6019ADE882391F19F8979
:1045C000903159F49924AA24BB24F401EE0FFF1F63
:1045D000E550F84F5182408210C0E89487F8992442
:1045E000AA24BB24F401EE0FFF1FEE0FFF1FE550BE
:1045F000F84F40825182628273829A89923090F0A1
:104600004D815E816F8178854C0D5D1D6E1D7F1D16
:104610004093F4075093F5076093F6077093F707FC
:1046200001C080E0DF91CF911F910F91FF90EF903B
:10463000DF90CF90BF90AF909F908F907F906F90C2
:104640005F904F9008952F923F924F925F926F929A
:104650007F928F929F92AF92BF92CF92DF92EF9212
:10466000FF920F931F93CF93DF93CDB7DEB72F97B2
:104670000FB6F894DEBF0FBECDBF1C014C875D871F
:104680006E877F873B872A87DC0119960D911D91E4
:104690002D913C911C970F5F1F4F2F4F3F4F0D8364
:1046A0001E832F833887EA85FB8580809180A280D6
:1046B000B38081149104A104B10431F0FFEF8F1A8B
:1046C0009F0AAF0ABF0A10C0DC018D909D90AD908B
:1046D000BC90B1E0B9870C851D852E853F850130E2
:1046E00011052105310509F0198675016401412C78
:1046F000512C3201F10181859285A385B48548163C
:1047000059066A067B0608F04EC00D811E812F8176
:1047100038850C151D052E053F0550F4F2E0CF2E0F
:10472000D12CE12CF12CA2E08A2E912CA12CB12CC1
:104730009E012F5F3F4FB701A601C10110DE882304
:1047400091F149815A816B817C81D701C601019623
:10475000A11DB11D452B462B472B19F04C015D01C6
:104760000FC0AC01BD01481959096A097B090C85C4
:104770001D852E853F85401751076207730741F05D
:104780001FEF411A510A610A710A6C017D01B2CF13
:104790000FEF1FEF2FEF3FE0B701A601C101C4DE0D
:1047A0008D83811113C01D823DC02601370121E098
:1047B000421A51086108710897018601B301A201EC
:1047C000C101B2DE882379F3730162018C149D0468
:1047D000AE04BF0450F3AA85BB854D915D916D91E8
:1047E0007C914115510561057105A9F4EA85FB85A8
:1047F00080829182A282B382F985FF2399F00FEF24
:10480000801A900AA00AB00AD1018D929D92AD92B1
:10481000BC92139707C095018401C10185DE811107
:10482000E5CFC1CF8D812F960FB6F894DEBF0FBEB6
:10483000CDBFDF91CF911F910F91FF90EF90DF904F
:10484000CF90BF90AF909F908F907F906F905F9030
:104850004F903F902F900895AF92BF92CF92DF92EA
:10486000EF92FF920F931F93CF93DF9300D01F928D
:10487000CDB7DEB75C016A017B0182E090E0A0E089
:10488000B0E0F50180839183A283B3839E012F5F03
:104890003F4FB701A601C50162DD811102C080E072
:1048A00023C000E010E09801B701A601C5013CDE7D
:1048B0008823A9F3C980DA80EB80FC80F501878921
:1048C000803149F481E0F8EFCF16FFEFDF06E10415
:1048D000F10450F4DBCF81E098EFC9169FEFD906C1
:1048E000E9069FE0F90690F20F900F900F900F905D
:1048F000DF91CF911F910F91FF90EF90DF90CF90BC
:10490000BF90AF9008957F928F929F92AF92BF9287
:10491000CF92DF92EF92FF920F931F93CF93DF938B
:10492000EC01142F7093FA076093F9071F8A82E055
:1049300090E0A0E0B0E088839983AA83BB831092C3
:10494000F8071092F4071092F5071092F6071092EC
:10495000F7078FEF9FEFDC018093FB099093FC0931
:10496000A093FD09B093FE09442349F1453008F0B6
:10497000DEC040E060E070E0CB01B9DC882309F4E0
:10498000D6C020E1129FF0011124E755F64F808137
:104990008F7709F0CCC084859585A685B785843648
:1049A0009105A105B10508F4C2C0C084D184E28498
:1049B000F384C114D104E104F10421F4B8C0C12C82
:1049C000D12C760140E0C701B60191DC782E882316
:1049D00009F4ADC0809106089091070881159240B6
:1049E00009F0A5C030910B08332309F4A0C08091D1
:1049F000090890910A08892B09F499C020910808A8
:104A0000222309F494C03A8B2C831D8630E041E0C8
:104A100050E06D85062FCA01062E02C0880F991F2F
:104A20000A94E2F72817390731F081E0860F8D8765
:104A3000683078F37CC0209111083091120821155C
:104A4000310519F040E050E008C020911F08309176
:104A5000200840912108509122082D833E834F83E6
:104A600058878091090890910A0846015701880EDD
:104A7000991EA11CB11C8B8A9C8AAD8ABE8AE091CA
:104A80000C08F0910D08F98FE88FA0910B08B0E0A9
:104A90000E949DCC680D791D8A1D9B1D6A8F7B8F9E
:104AA0008C8F9D8FB5E0EE0FFF1FBA95E1F7E150B7
:104AB000FE4FEF2FFF27E695DC01CB018E0F9F1FE6
:104AC000A11DB11D8E879F87A88BB98B80900E0882
:104AD00090900F088114910419F0A12CB12C08C0FA
:104AE00080901B0890901C08A0901D08B0901E0894
:104AF000A7019601281B390B4A0B5B0BDA01C90190
:104B0000880D991DAA1DBB1D04C0B695A795979544
:104B100087950A95D2F789879A87AB87BC87853FA7
:104B20003FE09307A105B10520F48CE08F8B712C39
:104B300015C0853F9F4FA105B10510F480E10DC060
:104B40008091270890912808A0912908B0912A08FF
:104B50008A8F9B8FAC8FBD8F80E28F8B872DDF91EB
:104B6000CF911F910F91FF90EF90DF90CF90BF906A
:104B7000AF909F908F907F9008954F925F926F9229
:104B80007F928F929F92AF92BF92CF92DF92EF92DD
:104B9000FF920F931F93CF93DF932C0124EF33E009
:104BA00081E090E0F90145915491441655060CF0CE
:104BB00062C0AC0141505109DA01AA0FBB1FAA0F14
:104BC000BB1FAE50BC4FFD0165917491440F551F42
:104BD000440F551F40515C4FFA0165907490FC01E1
:104BE000EE0FFF1FEE0FFF1FEE50FC4FA590B4908D
:104BF000FD0105911491F901C591D491FA018590B7
:104C00009490882777FD8095982F0E9417C96B0193
:104C10007C01B20166197709882777FD8095982F66
:104C20000E9417C92B013C01B501601B710B88273D
:104C300077FD8095982F0E9417C99B01AC01C30195
:104C4000B2010E944ACB2B013C01BE0168197909CF
:104C5000882777FD8095982F0E9417C99B01AC018A
:104C6000C301B2010E947CC89B01AC01C701B6011F
:104C70000E949CC711C001962C5F3F4F8D33910558
:104C800009F090CFE2EEF4E065917491882777FD0A
:104C90008095982F0E9417C9DF91CF911F910F9196
:104CA000FF90EF90DF90CF90BF90AF909F908F904C
:104CB0007F906F905F904F9008954F925F926F92A8
:104CC0007F928F929F92AF92BF92CF92DF92EF929C
:104CD000FF920F931F93CF93DF932C01662371F103
:104CE000EBEBF2E28491882341F09091C00095FFB4
:104CF000FCCF8093C6003196F5CF70E04AE050E0DB
:104D000085EE9FE00E944AA3E9E5F2E084918823C2
:104D100041F09091C00095FFFCCF8093C600319682
:104D2000F5CF8091C00085FFFCCF8AE08093C6005C
:104D30000E94E45060E070E0CB017EC024E733E0E5
:104D400081E090E0F90145915491441655060CF02C
:104D500062C0AC0141505109DA01AA0FBB1FAA0F72
:104D6000BB1FAE58BC4FFD0165917491440F551F98
:104D7000440F551F40595C4FFA0165907490FC0137
:104D8000EE0FFF1FEE0FFF1FEE58FC4FA590B490E3
:104D9000FD0105911491F901C591D491FA01859015
:104DA0009490882777FD8095982F0E9417C96B01F2
:104DB0007C01B20166197709882777FD8095982FC5
:104DC0000E9417C92B013C01B501601B710B88279C
:104DD00077FD8095982F0E9417C99B01AC01C301F4
:104DE000B2010E944ACB2B013C01BE01681979092E
:104DF000882777FD8095982F0E9417C99B01AC01E9
:104E0000C301B2010E947CC89B01AC01C701B6017D
:104E10000E949CC711C001962C5F3F4F80329105C4
:104E200009F090CFEEEEF3E065917491882777FD5D
:104E30008095982F0E9417C9DF91CF911F910F91F4
:104E4000FF90EF90DF90CF90BF90AF909F908F90AA
:104E50007F906F905F904F90089560E08091540A2A
:104E60009091550A2ADF6093500A7093510A8093FB
:104E7000520A9093530A80914E0A90914F0A7DDE18
:104E800060934A0A70934B0A80934C0A90934D0AA0
:104E90008FB7F8941092420A8FBF089520911402A0
:104EA00030911502409116025091170260E070E0B7
:104EB0008FE793E40E947CC86093220A7093230AD0
:104EC0008093240A9093250A089597FF03C0809148
:104ED000490A04C0FC01E45EF54F808190E008952A
:104EE000CF93DF93D82FC62FC19561E00E9426C2D1
:104EF0006C2F8D2F0E945FC26C2F70E08D2FDF9181
:104F0000CF910C941CC1CF93C1E020E030E048E485
:104F100052E46091500A7091510A8091520A909126
:104F2000530A0E9478CA18160CF0C0E06C2F88E073
:104F300090E0CF91D5CF2F923F924F925F926F9298
:104F40007F928F929F92AF92BF92CF92DF92EF9219
:104F5000FF920F931F93CF93DF93CDB7DEB72897C0
:104F60000FB6F894DEBF0FBECDBF8091420A8823F2
:104F700009F4F8C172DF8090500A9090510AA09015
:104F8000520AB090530A0091580A1091590AB80178
:104F9000882777FD8095982F0E9417C9A501940155
:104FA0000E949BC76B017C0160932A0A70932B0AB5
:104FB00080932C0A90932D0A20E030E040E251E4E7
:104FC0000E9478CA181624F481E08093210AF7C061
:104FD00020E030E040E251ECC701B6010E9475C804
:104FE00087FD02C0012B21F481E08093210A0CC1CE
:104FF0008091210A882351F010923E0A10923F0AB4
:105000001092400A1092410A1092210A209118022F
:105010003091190240911A0250911B02C701B6014A
:105020000E944ACB69837A838B839C836093360A80
:105030007093370A8093380A9093390A20913E0A78
:1050400030913F0A4091400A5091410AC701B60190
:105050000E949CC72B013C012090260A3090270A11
:105060001091280A0091290A9101412F502F0E9486
:1050700075C887FD14C02090220A3090230A109131
:10508000240A0091250A9101412F502FB201C3013A
:105090000E9478CA18161CF01201162D072DC101A6
:1050A000A12FB02F80933E0A90933F0AA093400A0D
:1050B000B093410A209114023091150240911602DA
:1050C00050911702B101812F902F0E944ACB6D831E
:1050D0007E838F8398876093320A7093330A80931C
:1050E000340A9093350A20913A0A30913B0A409154
:1050F0003C0A50913D0AC501B4010E949BC7209112
:1051000010023091110240911202509113020E943C
:105110004ACB20ED3CEC4CE45DE30E944ACB2B01F2
:105120003C0123E333E343E75FE360912E0A709190
:105130002F0A8091300A9091310A0E944ACB9B013C
:10514000AC01C301B2010E949CC72B013C016093DA
:105150002E0A70932F0A8093300A9093310A2D8182
:105160003E814F81588569817A818B819C810E9423
:105170009CC7A30192010E949BC72B013C0120E028
:1051800030E04FE753E40E9478CA20E030E0A90104
:105190001816E4F4C701B6010E9478CA18167CF408
:1051A000A7019601B101812F902F0E949BC76093A8
:1051B0003E0A70933F0A8093400A9093410A412C23
:1051C000512C9FE7692E93E4792E21C0C301B201CF
:1051D0000E9475C887FF1BC020E030E0A901C7010D
:1051E000B6010E9475C887FF0FC0A7019601B101E3
:1051F000812F902F0E949BC760933E0A70933F0AB5
:105200008093400A9093410A412C512C32018092A4
:105210003A0A90923B0AA0923C0AB0923D0A6091F1
:10522000140A7091150A882777FD8095982F0E949F
:1052300017C99B01AC01C501B4010E9478CA1816B8
:10524000DCF46091080270910902882777FD80954F
:10525000982F0E9417C99B01AC01C501B4010E949F
:1052600075C887FF09C0C301B2010E94E4C87595E3
:10527000679560931C0A02C010921C0A0E9406C324
:105280000091180A1091190A20911A0A30911B0AEC
:10529000601B710B820B930B653C79408105910576
:1052A00058F031DE0E9406C36093180A7093190A01
:1052B00080931A0A90931B0A0E9406C300911D0A4C
:1052C00010911E0A20911F0A3091200A601B710B59
:1052D000820B930B683873418105910508F442C035
:1052E0000E9406C360931D0A70931E0A80931F0AD2
:1052F0009093200AC0904A0AD0904B0AE0904C0A42
:10530000F0904D0A20E030E040E751E4C701B601DB
:105310000E9478CA18161CF520E030E046E153E4FC
:10532000C701B6010E9475C887FF19C06091560A6F
:105330007091570A882777FD8095982F0E9417C98A
:105340009B01AC01C701B6010E9478CA87FD03C06A
:105350001092490A07C08FE78093490A03C0109250
:10536000490AA59828960FB6F894DEBF0FBECDBFA8
:10537000DF91CF911F910F91FF90EF90DF90CF9031
:10538000BF90AF909F908F907F906F905F904F9065
:105390003F902F900895CF93DF931092260A10929A
:1053A000270A1092280A1092290A2091140230919B
:1053B0001502409116025091170260E070E08FE7ED
:1053C00093E40E947CC86093220A7093230A80931E
:1053D000240A9093250A6D9A80910101806180933F
:1053E00001019D9A8091010188608093010187ED00
:1053F00080937A0010927E0010927D0080917E0052
:10540000816080937E0080917E00826080937E0028
:1054100080917E00846080937E0080E888BD8091CA
:105420006E00846080936E006AEF70E080E090E030
:105430000E9435C38FE090E09093150A8093140A80
:1054400060E080910A0290910B0237DC20E030E0AE
:1054500040E751E40E9475C887FF0AC080910A02A4
:1054600090910B02409790930B0280930A02E8CF31
:1054700086E391E0909309028093080260E08091B6
:10548000160A9091170A19DC20E030E04BE953E44A
:105490000E9478CA181654F48091160A9091170A3F
:1054A00040969093170A8093160AE8CFC091120A8B
:1054B000D091130ACE0161DB20E030E046E153E4F5
:1054C0000E9478CA181634F46096D093130AC093D9
:1054D000120AECCFDF91CF91089508951092590AE6
:1054E0001092580A1092570A1092560A10921C0AEB
:1054F00075981092570A1092560A1092490AA59868
:1055000008952F923F924F925F926F927F928F9267
:105510009F92AF92BF92CF92DF92EF92FF920F9342
:105520001F93CF93DF93CDB7DEB7AE970FB6F89446
:10553000DEBF0FBECDBF6B8F7C8F8D8F292E5A871C
:1055400049873CA72BA70E9406C36F8F78A389A326
:105550009AA30E9406C36FA378A789A79AA7298553
:105560003A85121613061CF0E4EAF6E017C0E7EBE2
:10557000F6E08191882339F09091C00095FFFCCF2F
:105580008093C600F6CF8091C00085FFFCCF1BC280
:105590009091C00095FFFCCF8093C600819181114E
:1055A000F7CF8091C00085FFFCCF8AE08093C600D2
:1055B00095DF49855A858FE7452B99F18093490AF4
:1055C0008F8D98A1A9A1BAA1898B9A8BAB8BBC8B2B
:1055D0008D879E87AF87B88B1D8290E4988FACE152
:1055E000A98FB6E4BA8F1DA61D8A1E8A1F8A2FE7CF
:1055F00030E040E050E029833A834B835C83EFE75F
:105600004E2E512C612C712C1BA21CA21DA21EA27D
:1056100031E03E8F1C861B86312C00E010E01EA678
:1056200005C080931C0ACCCF0E9485848091420AD9
:10563000882309F4F6C011DC49855A85452B51F0C1
:1056400030904A0A00914B0A10914C0A50914D0A31
:105650005EA709C03090500A0091510A1091520A79
:105660008091530A8EA7232D302F412F5EA56DA563
:105670007D898E899F890E9478CA18162CF03DA6D4
:105680000D8B1E8B9EA59F8B232D302F412F5EA54A
:105690006D81788D898D9A8D0E9475C887FD05C0B2
:1056A0003D82088F198FAEA5AA8F0E9406C32FA135
:1056B00038A549A55AA5621B730B840B950B653C55
:1056C00079408105910538F01EDC0E9406C36FA366
:1056D00078A789A79AA74E8D442309F44FC02B8D34
:1056E0003C8D4D8D522D632D702F812F9EA50E94D4
:1056F00078CA18160CF095C00E9406C329893A8909
:105700004B895C89621B730B840B950B6938734161
:105710008105910508F485C0D301C20129813A8130
:105720004B815C81821B930BA40BB50B49855A8579
:10573000B595A79597958795452B19F08093490ABC
:1057400002C080931C0A0E9406C36D877E878F87E4
:10575000988BDC01CB0129893A894B895C89821BB2
:10576000930BA40BB50B8BA39CA3ADA3BEA33B8D46
:105770003DA74C8D4D8B5D8D5E8B2F8A2B8D3C8D87
:105780004D8D522D632D702F812F9EA50E9475C8BF
:1057900087FFEEC20E9406C32D853E854F8558893E
:1057A000621B730B840B950B69387341810591055E
:1057B00008F4DEC20E9406C3698B7A8B8B8B9C8BAC
:1057C000DC01CB012D853E854F855889821B930BCB
:1057D000A40BB50B4B855C85452B09F010C1898165
:1057E0009A81AB81BC81840D951DA61DB71D2985AD
:1057F0003A85B595A79597958795232B09F4B5C25A
:105800008093490A4B855C854F5F5F4F5C874B8770
:105810005B8D5D838C8D888F9D8D998F2A8EA1E005
:10582000AE8F20E030E040EA51E46B8D7C8D8D8DB1
:10583000922D0E949CC79B01AC01632D702F812F7C
:105840009EA50E9478CA181694F4EFEFF2E08491B6
:10585000882341F09091C00095FFFCCF8093C60053
:105860003196F5CF8091C00085FFFCCFACC00E947F
:1058700006C32F8D38A149A15AA1621B730B840B5B
:10588000950B613D77408105910508F44FC049852E
:105890005A85452B81F0E090490AF12CE9EFF2E0BE
:1058A00084918823C1F09091C00095FFFCCF809334
:1058B000C6003196F5CFE0901C0AF12CE3EFF2E040
:1058C0008491882341F09091C00095FFFCCF809394
:1058D000C6003196F5CF22E030E0432D502F612FE6
:1058E0007EA585EE9FE00E9420A4EFEEF2E0849179
:1058F000882341F09091C00095FFFCCF8093C600B3
:105900003196F5CF4AE050E0B70185EE9FE00E9466
:105910004AA38091C00085FFFCCF8AE08093C60037
:105920000E9406C36F8F78A389A39AA30E9406C31F
:105930006B017C010E9406C389889A88AB88BC8869
:105940002D853E854F855889820E931EA41EB51E57
:10595000C818D908EA08FB08C60ED71EE81EF91EAB
:1059600031E8C3163FE4D30632E1E306F10490F0D8
:10597000E2EDF2E08491882341F09091C00095FF20
:10598000FCCF8093C6003196F5CF8091C00085FF93
:10599000FCCF19C04B855C858BA59CA5841795070A
:1059A0000CF042CEE6E7F2E08491882341F090913A
:1059B000C00095FFFCCF8093C6003196F5CF809153
:1059C000C00085FFFCCF8AE08093C600AE960FB67C
:1059D000F894DEBF0FBECDBFDF91CF911F910F9125
:1059E000FF90EF90DF90CF90BF90AF909F908F90FF
:1059F0007F906F905F904F903F902F9008958BA075
:105A00009CA0ADA0BEA0880E991EAA1EBB1E2BA1F5
:105A10003CA14DA15EA1281B390B4A0B5B0BCA01AF
:105A2000B90129813A814B815C810E9410CCA5018A
:105A300094010E9475CC240D351D461D571D24313F
:105A400031054105510504F129013A013CEE4316A7
:105A50005104610471042CF06BEE462E512C612C24
:105A6000712C40E84416510461047104DCF08EEF9F
:105A700090E0A0E0B0E084199509A609B7098983F0
:105A80009A83AB83BC8312C054E1452E512C612C08
:105A9000712C24E130E040E050E029833A834B83CD
:105AA0005C8304C049825A826B827C82E8E6F3E020
:105AB0008491882341F09091C00095FFFCCF8093A2
:105AC000C6003196F5CF2AE030E0B301A20185EEA1
:105AD0009FE00E941FA3E3E6F3E08491882341F056
:105AE0009091C00095FFFCCF8093C6003196F5CF12
:105AF0002AE030E049815A816B817C8185EE9FE00C
:105B00000E941FA3ECE5F3E08491882341F090917B
:105B1000C00095FFFCCF8093C6003196F5CF22E000
:105B200030E04D81588D698D7A8D85EE9FE00E9421
:105B300020A4E5E5F3E08491882341F09091C00032
:105B400095FFFCCF8093C6003196F5CF22E030E080
:105B50004DA55D896E897F8985EE9FE00E9420A416
:105B60008091C00085FFFCCF8AE08093C6002B8522
:105B70003C85233031050CF432CE69817A818B81EA
:105B80009C810E9417C920E030E040E850E40E9468
:105B90004ACB6B017C012D81388D498D5A8D6DA5C5
:105BA0007D898E899F890E949BC720ED3FE049E453
:105BB00050E40E944ACB20E030E040E05FE30E94E6
:105BC0004ACB9B01AC01C701B6010E947CC86B01A6
:105BD0007C01C501B4010E9417C920E030E04AE70A
:105BE00054E40E947CC84B015C01EFE4F3E0849133
:105BF000882341F09091C00095FFFCCF8093C600B0
:105C00003196F5CF22E030E0B701A60185EE9FE0A6
:105C10000E9420A4E9E4F3E08491882341F090916C
:105C2000C00095FFFCCF8093C6003196F5CF22E0EF
:105C300030E0B501A40185EE9FE00E9420A4809190
:105C4000C00085FFFCCF8AE08093C6002AE939E9CD
:105C500049E15FE3C701B6010E944ACB6B017C01B9
:105C60009B01AC010E949CC7A50194010E947CC8C5
:105C70006D837E838F839887A5019401C701B60148
:105C80000E944ACB20E030E040E05EE30E944ACB35
:105C90004B015C01EBE3F3E08491882341F09091A8
:105CA000C00095FFFCCF8093C6003196F5CF809160
:105CB000C00085FFFCCF8AE08093C600E5E3F3E0F7
:105CC0008491882341F09091C00095FFFCCF809390
:105CD000C6003196F5CF22E030E0B701A60185EE8F
:105CE0009FE00E9420A48091C00085FFFCCF8AE045
:105CF0008093C600EFE2F3E08491882341F0909115
:105D0000C00095FFFCCF8093C6003196F5CF22E00E
:105D100030E04D815E816F81788585EE9FE00E9445
:105D200020A48091C00085FFFCCF8AE08093C6004C
:105D3000E9E2F3E08491882341F09091C00095FF5F
:105D4000FCCF8093C6003196F5CF22E030E0B5015C
:105D5000A40185EE9FE00E9420A48091C00085FFF1
:105D6000FCCF8AE08093C6003ACD80931C0A4ACDCE
:105D70001E8E57CDCF93C82FB1DB0E9433568111B1
:105D800034C0EBEBF2E29491992341F08091C00092
:105D900085FFFCCF9093C6003196F5CF6C2F70E055
:105DA0004AE050E085EE9FE00E944AA38091C00047
:105DB00085FFFCCF8AE08093C600ECE2F2E084919C
:105DC000882341F09091C00095FFFCCF8093C600DE
:105DD0003196F5CF8091C00085FFFCCF8AE080939B
:105DE000C6008FE192E00E94F683CF910C94DB55C0
:105DF000CF93C82F73DB0E943356811134C0EBEB75
:105E0000F2E29491992341F08091C00085FFFCCF8C
:105E10009093C6003196F5CF6C2F70E04AE050E0C9
:105E200085EE9FE00E944AA38091C00085FFFCCFD1
:105E30008AE08093C600E2EFF1E08491882341F08C
:105E40009091C00095FFFCCF8093C6003196F5CFAE
:105E50008091C00085FFFCCF8AE08093C60085EE6C
:105E600091E00E94F683CF910C94DB55A5980E9497
:105E70003356811125C0EBEBF2E28491882341F087
:105E80009091C00095FFFCCF8093C6003196F5CF6E
:105E9000EBEAF1E08491882341F09091C00095FFF6
:105EA000FCCF8093C6003196F5CF8091C00085FF6E
:105EB000FCCF8AE08093C6008AE991E00E94F683D5
:105EC0000C94DB551F920F920FB60F9211240BB654
:105ED0000F920F931F932F933F934F935F936F9363
:105EE0007F938F939F93AF93BF93CF93DF93EF9362
:105EF000FF9380910702811112C080911C0A809348
:105F0000110A882311F0759A01C075988091490A89
:105F10008093100A882311F0A59A01C0A59890914A
:105F2000110A80910702981708F475989091100A49
:105F300080910702981708F4A598809107028F5F57
:105F40008F77809307028091060290E08B30910555
:105F500008F093C0FC01EE58FF4F0C9491CC1092C6
:105F60007B0080E480937C0080917A008064809341
:105F70007A000E94FF8381E019C02091780030915F
:105F8000790080910C0A90910D0AA0910E0AB091AF
:105F90000F0A820F931FA11DB11D80930C0A9093CD
:105FA0000D0AA0930E0AB0930F0A82E080930602B6
:105FB00064C010927B0082E480937C0080917A0020
:105FC000806480937A000E94FF8383E0EFCF20916A
:105FD0007800309179008091080A9091090AA09187
:105FE0000A0AB0910B0A820F931FA11DB11D809365
:105FF000080A9093090AA0930A0AB0930B0A84E056
:10600000D5CF10927B0081E480937C0080917A0050
:10601000806480937A000E94FF8385E0C7CF20913F
:106020007800309179008091040A9091050AA0913E
:10603000060AB091070A820F931FA11DB11D80931C
:10604000040A9093050AA093060AB093070A86E013
:10605000ADCF0E94FF8387E0A9CF88E0A7CF0E9441
:10606000FF8389E0A3CF109206028091030A8F5F1D
:106070008093030A02C0109206028091030A8031C5
:1060800008F463C08091420A811110C080910C0A0B
:1060900090910D0A9093550A8093540A8091080AB2
:1060A0009091090A90934F0A80934E0A81E0809361
:1060B000420A1092030A10920C0A10920D0A1092D2
:1060C0000E0A10920F0A1092040A1092050A1092FA
:1060D000060A1092070A1092FF091092000A109205
:1060E000010A1092020A1092080A1092090A1092EC
:1060F0000A0A10920B0A2091540A3091550A809195
:10610000160A9091170A8217930714F080E032DE86
:106110002091540A3091550A80910A0290910B0205
:106120002817390714F080E063DE20914E0A309181
:106130004F0A8091120A9091130A821793072CF04C
:106140001092570A1092560A91DE00E010E0E80122
:10615000CC0FDD1FCD5BD54F8881998118161906AC
:1061600044F461E0802F0E9436AD888199810197C7
:1061700009C0892B49F060E0802F0E9436AD8881EC
:1061800099810196998388830F5F1F4F0330110512
:10619000F1F6FF91EF91DF91CF91BF91AF919F9178
:1061A0008F917F916F915F914F913F912F911F91AF
:1061B0000F910F900BBE0F900FBE0F901F90189570
:1061C0002CEA35EC47E25EE30C944ACB2CEA35EC42
:1061D00047E25EE30C947CC82CEA35EC47E25EE3D0
:1061E0000C947CC82CEA35EC47E25EE30C944ACB75
:1061F000CF93DF93EC0160E08E810E945FC281E06B
:1062000090E00E9459C361E08E810E945FC281E0EC
:1062100090E00E9459C360E08E810E945FC284E6D4
:1062200090E0DF91CF910C9459C3CF92DF92EF921F
:10623000FF920F931F93CF93DF937C01C0E0D0E0D8
:10624000C62ED12C87010C0F1D1F61E0F80187813C
:106250000E9426C2B6010C2E02C0759567950A945D
:10626000E2F76170F80187810E945FC22196C43015
:10627000D10541F7C701DF91CF911F910F91FF9099
:10628000EF90DF90CF90B4CFCF92DF92EF92FF925A
:106290000F931F93CF93DF937C01C0E0D0E0C62E15
:1062A000D12C87010C0F1D1F61E0F80187810E942E
:1062B00026C2B6010C2E02C0759567950A94E2F7C6
:1062C0006170F80187810E945FC22196C830D105B4
:1062D00041F7C701DF91CF911F910F91FF90EF9090
:1062E000DF90CF9085CF1F93CF93DF93EC01162FD4
:1062F000642F8C810E945FC28D818F3F19F060E016
:106300000E945FC28F85612F84FF05C0CE01DF919F
:10631000CF911F91B9CF70E084E0759567958A950C
:10632000E1F7CE0182DF612FCE01DF91CF911F9186
:106330007CCF40E0D8CF61E0FCDF80E496E00C94B5
:1063400059C362E0F6DF80E496E00C9459C3CF9322
:10635000DF93CDB7DEB728970FB6F894DEBF0FBE38
:10636000CDBF28E0EFE1F6E0DE01119601900D923D
:106370002A95E1F7FC012389421710F04FEF420FF5
:10638000FE013196E40FF11DE40FF11D2081260F6F
:106390002068622F28960FB6F894DEBF0FBECDBFDF
:1063A000DF91CF91C6CFFC016089262F2460208B1E
:1063B0006C60BFCFCF93DF93EC01423018F08F8534
:1063C00088608F874B8B1C8A222329F0413019F477
:1063D0008F8584608F8780E593EC0E9459C360E0CD
:1063E0008C810E945FC260E08E810E945FC28D81BD
:1063F0008F3F19F060E00E945FC26F8564FD19C095
:1064000063E0CE0112DF84E991E10E9459C363E0A9
:10641000CE010BDF84E991E10E9459C363E0CE0114
:1064200004DF86E990E00E9459C362E0CE01FDDE00
:1064300013C06062CE017DDF84E991E10E9459C3FF
:106440006F856062CE0175DF86E990E00E9459C3D6
:106450006F856062CE016DDF6F856062CE0169DF9E
:106460008CE390E00E9459C384E0888BCE019BDFCF
:106470008CE390E00E9459C3CE015DDF88EB9BE086
:106480000E9459C382E0898B66E0CE0152DF8CE323
:1064900090E0DF91CF910C9459C36F927F928F92CD
:1064A000AF92CF92EF920F931F93CF93DF93CDB71D
:1064B000DEB73C01162F842F5E854F853889998978
:1064C000F301848325830683E782C086A1868286C2
:1064D000538744873587968761E00E9426C2F3017F
:1064E00085818F3F19F061E00E9426C261E0F301CF
:1064F00086810E9426C2112319F0F301178603C07A
:1065000080E1F301878720E041E060E1C301DF9192
:10651000CF911F910F91EF90CF90AF908F907F9080
:106520006F9048CF8F92AF92CF92EF920F93DC0192
:1065300013961C921E921297E5EEF6E0ED93FC93F3
:106540001F921F921F921F928C2CAE2CC02EE22EF7
:10655000042F2FEF462F61E0A0DF0F900F900F90D8
:106560000F900F91EF90CF90AF908F900895CF93B1
:10657000DF93EC01423018F08F8588608F874B8B5A
:106580001C8A222329F0413019F48F8584608F877B
:1065900080E593EC0E9459C360E08C810E945FC249
:1065A00060E08E810E945FC28D818F3F19F060E0B4
:1065B0000E945FC26F8564FD19C063E0CE0135DEC5
:1065C00084E991E10E9459C363E0CE012EDE84E9A3
:1065D00091E10E9459C363E0CE0127DE86E990E095
:1065E0000E9459C362E0CE0120DE13C06062CE017A
:1065F000A0DE84E991E10E9459C36F856062CE01FB
:1066000098DE86E990E00E9459C36F856062CE01F2
:1066100090DE6F856062CE018CDE8CE390E00E949C
:1066200059C384E0888BCE01BEDE8CE390E00E94EB
:1066300059C3CE0186DE80E496E00E9459C382E011
:10664000898B66E0CE0175DE8CE390E00E9459C331
:1066500040E068E0CE017BDE60EC77E0CE010E9496
:1066600093C741E068E0CE0172DE60EC77E0CE01D6
:106670000E9493C742E066E0CE0169DE6EEB77E0F0
:10668000CE01DF91CF910C9493C7CF92DF92EF921E
:10669000FF920F931F93CF93DF931F921F92CDB75B
:1066A000DEB78C01677088E0689FB00111246064D8
:1066B000C80149835A833DDE4981C42E5A81D52EB3
:1066C000E12CF12CD6016D916D01D801ED91FC9179
:1066D0000190F081E02DC8011995BFEFEB1AFB0A7C
:1066E000E8E0EE16F10471F70F900F90DF91CF9173
:1066F0001F910F91FF90EF90DF90CF90089541E0B0
:10670000F2DD81E090E008950F931F93CF93DF9324
:10671000EC018B0144E150E0BC018AE59AE00E9463
:106720009DCFCE010E947CCF992744E150E0481BC9
:10673000590BB801865A954F0E949DCF8AE59AE081
:10674000DF91CF911F910F910895AF92BF92CF9299
:10675000DF92EF92FF920F931F93CF93DF93EC01A1
:106760005B017A01690144E150E0BC018AE59AE0ED
:106770000E949DCFCE010E947CCFEC01DD2704E179
:1067800010E0A8014C1B5D0BB501CE01865A954F58
:106790000E949DCFC5010E947CCFC80FD91FDD2765
:1067A000A8014C1B5D0BB701CE01865A954F0E9484
:1067B0009DCFC7010E947CCF8C0F9D1F9927A801F8
:1067C000481B590BB601865A954F0E949DCF8AE50A
:1067D0009AE0DF91CF911F910F91FF90EF90DF90A2
:1067E000CF90BF90AF9008952F923F924F925F92BB
:1067F0006F927F928F929F92AF92BF92CF92DF92D1
:10680000EF92FF920F931F93CF93DF93CDB7DEB735
:10681000CF54D1090FB6F894DEBF0FBECDBF1C0117
:106820007E8F6D8F4A012FAB09AF2896EFAE289768
:106830002C96ACAEBDAECEAEDFAE2C9734E0239F2F
:1068400050011124FC01EA0DFB1D80819181A28180
:10685000B381898F9A8FAB8FBC8FDA01AA0DBB1DD4
:10686000BCAFABAF4D905D906D907C90A301920159
:10687000698D7A8D8B8D9C8D0E949CC721966CAF03
:106880007DAF8EAF9FAF2197B4E00B9F80011124A5
:10689000F101E00FF11F20813181428153812F8F5F
:1068A00038A349A35AA3A401400F511F23965FAFF9
:1068B0004EAF2397DA01CD90DD90ED90FC90A701CB
:1068C00096016F8D78A189A19AA10E949CC72796F5
:1068D0006CAF7DAF8EAF9FAF27972896EFAD28970F
:1068E000B4E0EB9FC0011124F101E80FF91F2081F2
:1068F0003181428153812BA33CA34DA35EA3ED8D37
:10690000FE8DE80FF91F60817181828193810E9461
:106910009BC76FA378A789A79AA7AD8DBE8D1C963C
:106920008D919D910D90BC91A02D60968CAF9DAFE7
:10693000AEAFBFAF6097D1011C962D913D914D91A7
:106940005C911F972BA73CA74DA75EA7A3019201BF
:1069500050582D8B3E8B4F8B588FD701C601B058A6
:10696000898B9A8BAB8BBC8BED8DFE8DEA0DFB1D5D
:1069700020813181428153812FA738AB49AB5AAB7B
:1069800021962CAD3DAD4EAD5FAD21976FA578A999
:1069900089A99AA90E949BC76B017C01ED8DFE8D90
:1069A000E00FF11F80819181A281B3818BAB9CAB01
:1069B000ADABBEAB27962CAD3DAD4EAD5FAD2797D1
:1069C000BC01CD010E949BC74B015C01A701960150
:1069D0006D897E898F89988D0E944ACB2B013C015D
:1069E000A501940169897A898B899C890E944ACB87
:1069F0009B01AC01C301B2010E949CC72B013C0169
:106A0000A50194016D897E898F89988D0E944ACB5A
:106A10004B015C01A701960169897A898B899C8960
:106A20000E944ACB9B01AC01C501B4010E949BC7E7
:106A3000A30192010E940FC86B017C0120E030E0AD
:106A4000A9010E9475C887FF0AC02BED3FE049EC01
:106A500050E4C701B6010E949CC76B017C01AA9655
:106A60008FADAA97882351F02BED3FE049EC50E41D
:106A7000C701B6010E949BC76B017C012FA538A9F5
:106A800049A95AA9698D7A8D8B8D9C8D0E9475C8F4
:106A900081111FC02BA93CA94DA95EA96F8D78A1BA
:106AA00089A19AA10E9475C8811113C020E030E02D
:106AB000A901C701B6010E9475C881110AC02BED5A
:106AC0003FE049EC50E4C701B6010E949CC76B014E
:106AD0007C01A9962CAD3DAD4EAD5FADA997C70128
:106AE000B6010E944ACB2FA138A549A55AA55F77C8
:106AF0000E9485CA4B015C012FE632E143E85AE36C
:106B00000E9475C887FDC8C1C501B4010E9452C961
:106B10000E94E9C87A8F698FDB01AB2B21F4E1E099
:106B2000F0E0FA8FE98F298D3A8DB90180E090E08D
:106B30000E9415C94B015C019B01AC01C701B60164
:106B40000E947CC82B013C01A50194016FA178A58E
:106B500089A59AA50E947CC86FA778AB89AB9AAB30
:106B60002BA53CA54DA55EA560966CAD7DAD8EAD0B
:106B70009FAD60970E949BC7A50194010E947CC8AD
:106B80006BAB7CAB8DAB9EAB20E030E040E05FE3D5
:106B9000C301B2010E944ACBA30192010E944ACBD9
:106BA0009B01AC0160E070E080E89FE30E949BC71E
:106BB0006FA378A789A79AA7CE010196FC01289612
:106BC0004FAD289734E0439FE00DF11D11242BA118
:106BD0003CA14DA15EA120833183428353832BA529
:106BE0003CA54DA55EA52D873E874F87588BB12CC0
:106BF00041E050E058A34F8F1C01BFA9A4E0BA9F09
:106C0000800D911D112498AF8FAB910159AD44E0D7
:106C1000549F200D311D11243AAF29AFFCA7EBA7DB
:106C20004F8D58A1898D9A8D4817590708F01AC1C0
:106C300088E18B150CF444C02FA138A549A55AA5AD
:106C400069897A898B899C890E944ACB6B017C0176
:106C5000A30192016D897E898F89988D0E944ACB0C
:106C6000A70196010E949CC7A62E172F982E892E49
:106C70002FA138A549A55AA56D897E898F89988D40
:106C80000E944ACB6B017C01A301920169897A8938
:106C90008B899C890E944ACB9B01AC01C701B6013C
:106CA0000E949BC76D8B7E8B8F8B988FB3948A2DA0
:106CB000912FA92DB82D898B9A8BAB8BBC8B6CC077
:106CC000AF8DB8A1BD0180E090E00E9415C9A3017D
:106CD00092010E944ACB6B017C010E9479C8698BAA
:106CE0007A8B8B8B9C8BC701B6010E94ADCB4B017D
:106CF0005C01EBADFCADC080D180E280F380F7FA9F
:106D0000F094F7F8F0942396AEADBFAD23972D9194
:106D10003D914D915C912BA33CA34DA35EA329898A
:106D20003A894B895C89C701B6010E944ACB6D8BB9
:106D30007E8B8F8B988FA50194016BA17CA18DA177
:106D40009EA10E944ACB9B01AC016D897E898F89EF
:106D5000988D0E949CC76D8B7E8B8F8B988FA50121
:106D60009401C701B6010E944ACB6B017C012989BD
:106D70003A894B895C896BA17CA18DA19EA10E945F
:106D80004ACB9B01AC01C701B6010E949BC7698B2E
:106D90007A8B8B8B9C8BB12C2D893E894F89588D9A
:106DA00021966CAD7DAD8EAD9FAD21970E949CC7A5
:106DB000EFA9F8AD608371838283938329893A892F
:106DC0004B895C8927966CAD7DAD8EAD9FAD2797C5
:106DD0000E949CC7A9ADBAAD6D937D938D939C9392
:106DE00013972FA538A949A95AA9EBA5FCA560813D
:106DF0007181828193810E949CC7ABA5BCA56D93D4
:106E00007D938D939C9313972BA93CA94DA95EA9C3
:106E10006D857E858F8598890E949CC76D877E874A
:106E20008F87988BC1010E942C4DFE01E659FF4FC0
:106E30006F012C96ECACFDAC0EAD1FAD2C979E01F6
:106E4000235F3F4FAE01475F5F4FBE016B5F7F4FD8
:106E5000C1010E9431B42F8D38A12F5F3F4F38A35D
:106E60002F8FDECE2D8D3E8D245F3F4F4D8D5E8D5D
:106E7000485F5F4F6D8D7E8D6C5F7F4FDE01A65941
:106E8000BF4F6D012C96ECACFDAC0EAD1FAD2C9739
:106E90008D8D9E8D0E9431B4C15BDF4F0FB6F8948B
:106EA000DEBF0FBECDBFDF91CF911F910F91FF903D
:106EB000EF90DF90CF90BF90AF909F908F907F909A
:106EC0006F905F904F903F902F900895FC01148237
:106ED0001782138212828DED97E09183808308954B
:106EE0002DED37E0FC01318320832781222319F027
:106EF00004960C94B51C0895CF92DF92EF92FF9206
:106F00000F931F93CF93DF93EC01875B9F4FDEDFDF
:106F1000CE0186599F4FDADF7E0129E8E20EF11C8F
:106F200087016E0131E4C31A3EEFD30AC801CEDFF8
:106F3000015E1F4F0C151D05C9F7FE01EF53FE4FF3
:106F400089E1818314823596178ACE018C519E4F38
:106F5000BDDFFE01EB56FD4F1082118212821382BB
:106F6000389610821182128213821A821B82188232
:106F700019826E0187E6C81A8DEFD80AF6011082D1
:106F8000118212821382F80111821082FE01ED5FDC
:106F9000FD4F108286E391E0F7019C011192215090
:106FA0003040E1F7FE01EF55FD4F81E08083C95B82
:106FB000DF4F198218820E9406C368577C4E8F4F9C
:106FC0009F4FF6016083718382839383DF91CF911A
:106FD0001F910F91FF90EF90DF90CF900895FC01EB
:106FE00020E03EE2DB014C91403241F0283011F4C8
:106FF00030833196DB014C91408331962F5F6F5F78
:107000007F4F2B3079F7108208952F923F924F9245
:107010005F926F927F928F929F92AF92BF92CF9228
:10702000DF92EF92FF920F931F93CF93DF93CDB731
:10703000DEB7CA58D1090FB6F894DEBF0FBECDBF78
:107040008C016B017A014901CA57DF4F1882C6587B
:10705000D04084E0E80EF11C180191E1290E311CAA
:10706000F801EA5BFF4FC957DF4FF983E883C75840
:10707000D0403801FEE56F1AFDEF7F0A58018CE51C
:10708000A81A8DEFB80A90E4492E512C4C0E5D1EC3
:1070900094E0490E511CA101BE016F5F7F4FC701F3
:1070A0000E941F1B18160CF04AC12C85322F387114
:1070B000303109F0ACC0F3018081918101970297D2
:1070C00008F4A5C0BE016F5F7F4FCE0187589F4F68
:1070D00086DFA0961FAEA097F6018081811107C0C0
:1070E00069EE76E0CE01815A9F4F0E94F6CFB6013D
:1070F000CE01815A9F4F0E94F6CFBE0167587F4F45
:10710000CE01815A9F4F0E94F6CF69EE76E0CE0104
:10711000815A9F4F0E94F6CFCE01805C9F4FD6DEF2
:1071200021E0AE0147585F4FB701C2010E94AC1E7B
:10713000811147C0F30180819181892B09F041C001
:10714000E5EBF2E28491882341F09091C00095FF35
:10715000FCCF8093C6003196F5CFE0917A0CF0E039
:10716000EE0FFF1FE45EFD4F0190F081E02DEA5726
:10717000FE4F0190F081E02D8191882339F09091AC
:10718000C00095FFFCCF8093C600F6CF8091C00071
:1071900085FFFCCF8AE08093C600FE01E758FF4FD1
:1071A0008191882339F09091C00095FFFCCF8093A6
:1071B000C600F6CF8091C00085FFFCCF8AE08093A7
:1071C000C6008BE1FE01EC5BFF4FDE01959601905E
:1071D0000D928A95E1F724968EAD9FAD24979CA3DE
:1071E0008BA38DED97E09AA389A320E030E0AE0158
:1071F0004F5D5F4FBE01615A7F4FC80106DFCE0170
:1072000081966EDECE01805C9F4F6ADE44CF89811D
:10721000882309F494C08E3209F43DCF8F3509F4E8
:107220003ACFF80181898E3209F435CF8F3509F4D0
:1072300032CF23FD30CF81E0303109F080E0C957F3
:10724000DF4FE881F981C758D0408083811108C0A1
:107250008985873409F01FCF8A858E3709F41BCFC3
:1072600098012C5F3F4FBE016F5F7F4FC901C75729
:10727000DF4F2883C958D040C657DF4F3883CA58DC
:10728000D040ADDEF30180819181C757DF4F288167
:10729000C958D040C657DF4F3881CA58D0400097F0
:1072A000F1F4F6018191882339F09091C00095FFA7
:1072B000FCCF8093C600F6CFF9018191882339F085
:1072C0009091C00095FFFCCF8093C600F6CF8091CF
:1072D000C00085FFFCCF8AE08093C600DCCE813001
:1072E000910539F4F5018081918101969183808324
:1072F000D2CE029709F0CFCE8114910439F0B901B2
:10730000C4010E94E3CF892B71F419C0CA57DF4F23
:10731000F881C658D0402F2F30E0F501808191814F
:107320002817390761F0CA57DF4FF881C658D04097
:10733000FF5FCA57DF4FF883C658D040ACCEC65760
:10734000DF4F0FB6F894DEBF0FBECDBFDF91CF91F8
:107350001F910F91FF90EF90DF90CF90BF90AF9073
:107360009F908F907F906F905F904F903F902F9065
:1073700008950F931F93CF93DF93CDB7DEB76F9729
:107380000FB6F894DEBF0FBECDBF8C01FC01EE55E9
:10739000FD4F1182108240E050E0BA01835B9F4FA5
:1073A0000E94D21BC801875B9F4F2BE1FC013496E2
:1073B000DE01159601900D922A95E1F7FC0182817C
:1073C00093819C838B838DED97E09A83898320E062
:1073D00030E0AE014F5F5F4F64EC77E0C80115DE2F
:1073E000CE0101967DDD6F960FB6F894DEBF0FBE1D
:1073F000CDBFDF91CF911F910F9108952BE1FB013C
:107400003496DC01149601900D922A95E1F7FB0168
:1074100022813381FC01338322830895EF92FF920E
:107420000F931F93CF93DF93EC011B82FC01E05B72
:10743000FF4F8081882329F0CE01835B9F4F0E94FC
:10744000B51C7E018FE3E81A8EEFF80A45E360E091
:10745000C7010E94CA4581112CC0E5EBF2E284917C
:10746000882341F09091C00095FFFCCF8093C60027
:107470003196F5CFE0917A0CF0E0EE0FFF1FE45E5D
:10748000FD4F0190F081E02DE857FE4F0190F08113
:10749000E02D8491882341F09091C00095FFFCCFAE
:1074A0008093C6003196F5CF8091C00085FFFCCF58
:1074B0009EC08E010A531E4F41E0B701C8010E94D1
:1074C0008324811133C040E0B701C8010E948324A6
:1074D00081112CC0EBEBF2E28491882341F0909172
:1074E000C00095FFFCCF8093C6003196F5CFE091A8
:1074F0007A0CF0E0EE0FFF1FE45EFD4F0190F0818B
:10750000E02DE657FE4F0190F081E02D8491882315
:1075100041F09091C00095FFFCCF8093C60031965A
:10752000F5CF8091C00085FFFCCF61C0B801CE01CE
:10753000835B9F4F0E94C21981112CC0EBEBF2E2DA
:107540008491882341F09091C00095FFFCCF8093F7
:10755000C6003196F5CFE0917A0CF0E0EE0FFF1FF8
:10756000E45EFD4F0190F081E02DE457FE4F019065
:10757000F081E02D8491882341F09091C00095FF27
:10758000FCCF8093C6003196F5CF8091C00085FF77
:10759000FCCF2DC081E08B83E5EBF2E28491882360
:1075A00041F09091C00095FFFCCF8093C6003196CA
:1075B000F5CFE0917A0CF0E0EE0FFF1FE45EFD4F97
:1075C0000190F081E02DE257FE4F0190F081E02D17
:1075D0008491882341F09091C00095FFFCCF809367
:1075E000C6003196F5CF8091C00085FFFCCF8AE0C0
:1075F0008093C6008E01075B1F4FB801CE018659EC
:107600009F4FFCDEC859DF4F19830883DF91CF916C
:107610001F910F91FF90EF900895FC011282138249
:107620000895FC012381222311F021E02283089593
:10763000FC012281211112820895AF92BF92CF9254
:10764000DF92EF92FF920F931F93CF93DF931F92DE
:10765000CDB7DEB78C018FE2FB0181935F01D12CA6
:1076600041E07801F1E4EF1AFEEFFF0A6FE1C62E68
:107670002D2D30E0F7018081918128173907D8F44A
:10768000C29EC001C39E900D112483579F4FB50128
:10769000800F911F49830E946919C50149815C01CE
:1076A0000196F5012081222321F04D3810F44F5F1F
:1076B000F6CFD394DDCF47FD11C0B501C801885185
:1076C0009E4F0F90DF91CF911F910F91FF90EF9000
:1076D000DF90CF90BF90AF900C946919F5011082A4
:1076E0000F90DF91CF911F910F91FF90EF90DF905E
:1076F000CF90BF90AF9008953F924F925F926F925C
:107700007F928F929F92AF92BF92CF92DF92EF9231
:10771000FF920F931F93CF93DF93CDB7DEB7AC9754
:107720000FB6F894DEBF0FBECDBF7C015B01FC013C
:107730008381882309F408C1C70188519E4F0E94A4
:10774000B51CF7011282CE0101966C01BFDB270147
:1077500098E6490E511CC701875B9F4FF201918348
:107760008083F50180818F3209F084C06FE270E080
:10777000C5010E9401D08C010F5F1F4F7AE0372EA8
:107780000115110509F47CC06FE270E0C8010E9488
:1077900001D04C01009709F474C00817190708F0CC
:1077A00070C03C01601A710AA301B801CE01809635
:1077B0000E942AD0E0E2F0E0EC0FFD1FE60DF71D7D
:1077C0001082FE01B0968191882339F09091C0001B
:1077D00095FFFCCF8093C600F6CF8091C00085FF57
:1077E000FCCF3092C600F201608171816115710594
:1077F00019F06C5F7F4F02C060E070E021E0AE01E5
:10780000405E5F4FCE0105960E94AC1E81112BC0D9
:10781000EBEEF6E08491882341F09091C00095FF53
:10782000FCCF8093C6003196F5CFFE01B0968191D2
:10783000882339F09091C00095FFFCCF8093C6005B
:10784000F6CFE2EFFEE18491882341F09091C000F1
:1078500095FFFCCF8093C6003196F5CF8091C00094
:1078600085FFFCCF6CC0F201D182C08284010F5F22
:107870001F4F86CFC70186599F4FF20191838083A6
:107880008501F20180819181009711F0049602C078
:1078900080E090E0B8010E94821F882339F1E4EE75
:1078A000FEE18491882341F09091C00095FFFCCFC8
:1078B0008093C6003196F5CFF8018191882339F085
:1078C0009091C00095FFFCCF8093C600F6CF8091C9
:1078D000C00085FFFCCF8AE08093C600F701E35625
:1078E000FD4F10821182128213822CC0ECECFEE15B
:1078F0008491882341F09091C00095FFFCCF809344
:10790000C6003196F5CFF8018191882339F0909126
:10791000C00095FFFCCF8093C600F6CFEAECFEE1F5
:107920008491882341F09091C00095FFFCCF809313
:10793000C6003196F5CF8091C00085FFFCCF8AE06C
:107940008093C600C601CCDAAC960FB6F894DEBFC1
:107950000FBECDBFDF91CF911F910F91FF90EF90A0
:10796000DF90CF90BF90AF909F908F907F906F905F
:107970005F904F903F9008958F929F92AF92BF92E9
:10798000CF92DF92EF92FF92CF93DF931F92CDB70A
:10799000DEB77C01FC018281882309F4BCC07196AA
:1079A0008191882339F09091C00095FFFCCF80939E
:1079B000C600F6CFE8ECFEE18491882341F0909177
:1079C000C00095FFFCCF8093C6003196F5CFE091C3
:1079D0007A0CF0E0EE0FFF1FE45EFD4F0190F081A6
:1079E000E02DE456FE4F0190F081E02D8491882334
:1079F00041F09091C00095FFFCCF8093C600319676
:107A0000F5CFF701E356FD4F4081518162817381CB
:107A10002AE030E085EE9FE00E9476A3E6ECFEE1EE
:107A20008491882341F09091C00095FFFCCF809312
:107A3000C6003196F5CFF701EB56FD4F40815181DD
:107A4000628173812AE030E085EE9FE00E9476A398
:107A50008091C00085FFFCCF8AE08093C6000E9421
:107A600006C3E0E6CE2EEAEEDE2EE12CF12CA701D5
:107A700096010E9453CC49015A016091770A709196
:107A8000780A8091790A90917A0AA70196010E945A
:107A900053CC821A930AC4016CE370E00E942CCC90
:107AA0006983CE0101960E947385FC012191CF016B
:107AB000222339F03091C00035FFFCCF2093C6005F
:107AC000F4CF40E050E06AE385EE9FE00E942EA3F1
:107AD000C4016CE370E00E942CCC8983CE01019636
:107AE0000E947385FC012191CF01222339F030914E
:107AF000C00035FFFCCF2093C600F4CFE4ECFEE1DC
:107B000084918823E1F09091C00095FFFCCF809391
:107B1000C6003196F5CFEFEFF6E08491882341F06F
:107B20009091C00095FFFCCF8093C6003196F5CFB1
:107B30008091C00085FFFCCF8AE08093C6000F9043
:107B4000DF91CF91FF90EF90DF90CF90BF90AF90FB
:107B50009F908F900895AF92BF92CF92DF92EF9255
:107B6000FF920F931F93CF93DF935C01EB01FB0117
:107B700001900020E9F78F0101501109061B170B36
:107B80006C01F8E1CF1AFEEFDF0AF60110826EE415
:107B900070E0CE010E9401D07C01009729F4F80129
:107BA0003197EC0FFD1F0DC060E270E00E9401D024
:107BB000EC0121966AE270E0C7010E9401D0FC014D
:107BC00031978DE081838AE082831382BE01C501F3
:107BD0008C519E4F0E9433A4F6018081882371F15D
:107BE000EBEBF2E28491882341F09091C00095FF85
:107BF000FCCF8093C6003196F5CFE0917A0CF0E08F
:107C0000EE0FFF1FE45EFD4F0190F081E02DE05686
:107C1000FE4F0190F081E02D8491882341F09091F6
:107C2000C00095FFFCCF8093C6003196F5CF8091C0
:107C3000C00085FFFCCF8AE08093C600DF91CF9122
:107C40001F910F91FF90EF90DF90CF90BF90AF907A
:107C500008952F923F924F925F926F927F928F92F0
:107C60009F92AF92BF92CF92DF92EF92FF920F93CB
:107C70001F93CF93DF93CDB7DEB7CC55D1090FB6A5
:107C8000F894DEBF0FBECDBF4C018C010F551D4FC8
:107C9000662339F0F8011082F401838181111DC03F
:107CA00015C0F8018081882309F4AFC0F401E756BC
:107CB000FD4FC080D180E280F3800E9406C3C616CB
:107CC000D706E806F90608F4A0C0E4CFC401A6DB95
:107CD000F4018381882309F498C07401F7E4EF0E5E
:107CE000F11CF70181818F9380818F938BEB9EE153
:107CF0009F938F938E01015C1F4F1F930F930E94E0
:107D000039D00F900F900F900F900F900F90B12CD3
:107D1000F80101900020E9F73197E01BF10BBE1646
:107D200084F46801CB0CD11CB7FCDA94F601808195
:107D3000992787FD90950E946DCFF6018083B394BB
:107D4000E7CFFDE48F0E911C40E050E0BA01C40182
:107D50000E94D21B512CCE0101966C0184EB682E3F
:107D60008EE1782E5E0191E2A90EB11C40E050E058
:107D7000B601C4010E941F1B1816DCF5412CF60148
:107D800001900020E9F73197EC19FD094E1674F4C3
:107D90001601240C311C47FC3A94F101808190E0DB
:107DA0000E946DCFF10180834394E9CF8A858E379D
:107DB000E9F245E050E0B801C6010E941CD0892BD1
:107DC000A9F61F930F937F926F92BF92AF920E947A
:107DD00039D0C5010E94CB4880EB9EE10E944B49FF
:107DE0000F900F900F900F900F900F905524539479
:107DF000BDCF511004C08FEF9FEFF70104C0F70112
:107E000080819181019691838083C45ADF4F0FB6A0
:107E1000F894DEBF0FBECDBFDF91CF911F910F91C0
:107E2000FF90EF90DF90CF90BF90AF909F908F909A
:107E30007F906F905F904F903F902F9008950F9399
:107E40001F93CF93DF93EC018C0108511E4FC801A3
:107E50000E946B1CC8010E94B51C18821982DF9118
:107E6000CF911F910F910895CF92DF92EF92FF92E1
:107E70000F931F93CF93DF93CDB7DEB76F970FB6F6
:107E8000F894DEBF0FBECDBF8C016A017C0188E68D
:107E9000E80EF11CC80186599F4FF701918380833A
:107EA000E65CFD4F22E030E031832083329671831F
:107EB000608340E050E0BA0104960E94D21BF701B3
:107EC000808191812BE1FC013496DE0115960190B1
:107ED0000D922A95E1F7FC01828193819C838B832B
:107EE0008DED97E09A8389839601AE014F5F5F4FD6
:107EF00064EC77E0C80189D8CE0101960E94703702
:107F00006F960FB6F894DEBF0FBECDBFDF91CF9155
:107F10001F910F91FF90EF90DF90CF9008952F92D7
:107F20003F924F925F926F927F928F929F92AF9209
:107F3000BF92CF92DF92EF92FF920F931F93CF9356
:107F4000DF93CDB7DEB7AC970FB6F894DEBF0FBEA8
:107F5000CDBF8C016B01342EDC0113968C918823EC
:107F600009F449C3F801E551FE4F8081882309F4E3
:107F7000F5C02111C1C07801BDEFEB1AFB0AF70172
:107F80008081882361F1EBEBF2E28491882341F058
:107F90009091C00095FFFCCF8093C6003196F5CF3D
:107FA000E6E4FFE18491882341F09091C00095FFC1
:107FB000FCCF8093C6003196F5CF4AE050E061E0F7
:107FC00070E085EE9FE00E944AA38091C00085FF8B
:107FD000FCCF8AE08093C6000E94E4500CC3E5EB1E
:107FE000F2E28491882341F09091C00095FFFCCF8C
:107FF0008093C6003196F5CFEDE2FFE184918823AE
:1080000041F09091C00095FFFCCF8093C60031965F
:10801000F5CFF6018191882339F09091C00095FF4A
:10802000FCCF8093C600F6CFE2E2FFE18491882383
:1080300041F09091C00095FFFCCF8093C60031962F
:10804000F5CFD7018C91FDE8BF2EB801B89E600D29
:10805000711D1124685F7D4FC801EFDAF70180813F
:10806000F801B89EE00DF11D1124E85FFD4F8191EC
:10807000882339F09091C00095FFFCCF8093C60013
:10808000F6CFECE1FFE18491882341F09091C000AC
:1080900095FFFCCF8093C6003196F5CF5801F3E6EB
:1080A000AF1AFDEFBF0AD5014D915D916D917C91A5
:1080B0002AE030E085EE9FE00E9476A38091C00028
:1080C00085FFFCCF8AE08093C600F7012081F8018C
:1080D00084E0289FE00DF11D1124EC5FFD4FD501D8
:1080E0004D915D916D917C91408351836283738347
:1080F0002F5FF70120832CC0E5EBF2E28491882307
:1081000041F09091C00095FFFCCF8093C60031965E
:10811000F5CFEBE0FFE18491882341F09091C0001E
:1081200095FFFCCF8093C6003196F5CFF601819183
:10813000882339F09091C00095FFFCCF8093C60052
:10814000F6CF8091C00085FFFCCF8AE08093C60007
:10815000C80188519E4F0E94B51C30C0F801ED5FE8
:10816000FD4F1082E5EBF2E28491882341F090917B
:10817000C00095FFFCCF8093C6003196F5CFEAEFA3
:10818000FEE18491882341F09091C00095FFFCCFDF
:108190008093C6003196F5CFF6018191882339F09E
:1081A0009091C00095FFFCCF8093C600F6CF8091E0
:1081B000C00085FFFCCF8AE08093C600D8011296EC
:1081C0001C92FE0131965F01CF010E9466372801A3
:1081D000F8E64F0E511CC801875B9F4FD2018D936B
:1081E0009C93F60180818F3209F091C06FE270E0BC
:1081F000C6010E9401D001967C01EAE02E2EE11416
:10820000F10409F48AC06FE270E0C7010E9401D056
:108210004C01009709F482C0E816F90608F07EC008
:108220003C016E187F08A301B701CE0180960E9421
:108230002AD0E0E2F0E0EC0FFD1FE60DF71D108202
:10824000FE01B0968191882339F09091C00095FF8E
:10825000FCCF8093C600F6CF8091C00085FFFCCF95
:108260002092C600D2016D917C916115710519F0C3
:108270006C5F7F4F02C060E070E021E0AE01405EC5
:108280005F4FCE0105960E94AC1E811138C0E0916F
:108290007A0CF0E0EE0FFF1FE45EFD4F0190F081DD
:1082A000E02DEE56FE4F0190F081E02D8491882361
:1082B00041F09091C00095FFFCCF8093C6003196AD
:1082C000F5CFFE01B0968191882339F09091C000DE
:1082D00095FFFCCF8093C600F6CFE8EFFEE18491D6
:1082E000882341F09091C00095FFFCCF8093C60099
:1082F0003196F5CF8091C00085FFFCCF43C1F201DC
:10830000B182A0827401FFEFEF1AFF0A78CFC80193
:1083100086599F4FD2018D939C937601F801E851C5
:10832000FE4F4F01332009F4E5C0D2016D917C91DD
:108330006115710519F06C5F7F4F02C060E070E05D
:1083400021E0A701C4010E94AC1E20917A0C882371
:1083500009F49AC0F40181899289A389B489F8014A
:10836000EB56FD4F80839183A283B383E22FF0E02D
:10837000EE0FFF1FE45EFD4F0190F081E02DEC5603
:10838000FE4F0190F081E02D8491D801AB56BD4F96
:10839000882349F09091C00095FFFCCF8093C600E0
:1083A00031968491F5CFF7018191882339F090912E
:1083B000C00095FFFCCF8093C600F6CFE0917A0C09
:1083C000F0E0EE0FFF1FE45EFD4F0190F081E02D25
:1083D000EA56FE4F0190F081E02D8491882341F010
:1083E0009091C00095FFFCCF8093C6003196F5CFE9
:1083F0004D915D916D917C912AE030E085EE9FE09A
:108400000E9476A38091C00085FFFCCF8AE0809314
:10841000C600F801E356FD4F1082118212821382CA
:10842000E0917A0CF0E0EE0FFF1FE45EFD4F01904B
:10843000F081E02DE856FE4F0190F081E02D84910F
:10844000882341F09091C00095FFFCCF8093C60037
:108450003196F5CF8091C00085FFFCCF8AE08093F4
:10846000C600A70160E070E0C801FEDCD8015196AB
:108470008C91882319F0C801419601C0C7010E9460
:10848000B9838CE097E0B2C0E22FF0E0EE0FFF1F5F
:10849000E45EFD4F0190F081E02DEE56FE4F01901D
:1084A000F081E02D8491882341F09091C00095FFE8
:1084B000FCCF8093C6003196F5CFF70181918823D8
:1084C00039F09091C00095FFFCCF8093C600F6CFA5
:1084D000E6EFFEE18491882341F09091C00095FF82
:1084E000FCCF8093C6003196F5CF8091C00085FF08
:1084F000FCCF48C0F201608171816115710519F0EE
:108500006C5F7F4F02C060E070E026E5A701C40108
:108510000E94AC1E81113AC0E0917A0CF0E0EE0F9F
:10852000FF1FE45EFD4F0190F081E02DEE56FE4FFF
:108530000190F081E02D8491882341F09091C0005A
:1085400095FFFCCF8093C6003196F5CFF70181915E
:10855000882339F09091C00095FFFCCF8093C6002E
:10856000F6CFE4EFFEE18491882341F09091C000C2
:1085700095FFFCCF8093C6003196F5CF8091C00067
:1085800085FFFCCF8AE08093C60032C081E0D8012D
:108590008C93E0917A0CF0E0EE0FFF1FE45EFD4F4C
:1085A0000190F081E02DE656FE4F0190F081E02D24
:1085B0008491882341F09091C00095FFFCCF809377
:1085C000C6003196F5CFF6018191882339F090915C
:1085D000C00095FFFCCF8093C600F6CF8091C0000D
:1085E00085FFFCCF8AE08093C600C7010E94B98353
:1085F000C5010E947037AC960FB6F894DEBF0FBE6F
:10860000CDBFDF91CF911F910F91FF90EF90DF9041
:10861000CF90BF90AF909F908F907F906F905F9022
:108620004F903F902F90089521E0FC01218340E07E
:1086300076CCCF92DF92EF92FF920F931F93CF935E
:10864000DF93CDB7DEB76F970FB6F894DEBF0FBEDE
:10865000CDBF8C016C0128E6C20ED11C86599F4FFC
:10866000F60191838083E65CFD4F21E030E03183A9
:1086700020837801FCE5EF1AFDEFFF0AF701118274
:10868000108240E050E0BA0104960E94D21BF6012D
:10869000808191812BE1FC013496DE0115960190D9
:1086A0000D922A95E1F7FC01828193819C838B8353
:1086B0008DED97E09A83898320E030E0AE014F5F33
:1086C0005F4F64EC77E0C8010E940538CE01019647
:1086D0000E947037F701808191816F960FB6F894F0
:1086E000DEBF0FBECDBFDF91CF911F910F91FF90E5
:1086F000EF90DF90CF900895AF92BF92CF92DF922C
:10870000EF92FF920F931F93CF93DF93CDB7DEB716
:108710006F970FB6F894DEBF0FBECDBF8C017B0103
:10872000CE0101960E946637F801EF58FF4F808115
:108730006801811104C029E4C20ED11C03C08AE67D
:10874000C80ED11C21E0A701B6016C5F7F4FCE019E
:1087500005960E94AC1E81113AC0E5EBF2E28491CD
:10876000882341F09091C00095FFFCCF8093C60014
:108770003196F5CFE0917A0CF0E0EE0FFF1FE45E4A
:10878000FD4F0190F081E02DEE55FE4F0190F081FC
:10879000E02D8491882341F09091C00095FFFCCF9B
:1087A0008093C6003196F5CFF7018191882339F087
:1087B0009091C00095FFFCCF8093C600F6CF8091CA
:1087C000C00085FFFCCF8AE08093C60036C0F80168
:1087D000E154FE4F808191818A30910530F59C01F2
:1087E0002F5F3F4F318320832FE1289F7001299F06
:1087F000F00C112429E8E20EF11CE00EF11E5C01E0
:10880000B701C7014F960E94FE3981E0A81AB1084E
:108810002FE1E21AF1088FEFA816B80689F7B60122
:10882000C80187579F4F0E94FE39BE016F5F7F4F7F
:10883000C80186599F4F0E94FE39CE0101960E94C1
:1088400070376F960FB6F894DEBF0FBECDBFDF91C5
:10885000CF911F910F91FF90EF90DF90CF90BF903D
:10886000AF900895EF92FF920F931F93CF93DF93F2
:10887000EC01C154DE4F2881398121153105F9F011
:1088800021503109398328838C0107571F4FB801C4
:1088900086599F4F0E94FE39C80100E010E07C011C
:1088A0002FE1E20EF11C288139810217130738F4F9
:1088B0000F5F1F4FB7010E94FE39C701F0CFDF9154
:1088C000CF911F910F91FF90EF900895EF92FF923B
:1088D0000F931F93CF93DF93EC010E949EAC8E0108
:1088E0000D5F1D4FF80180819E0128513E4F790197
:1088F0008823A1F1C9010E94B51CF8018081815033
:108900008083BE01FDE88F9F600D711D1124685F9B
:108910007D4F21E041E0CE0102DBF8018081FE01C4
:1089200024E0829FE00DF11D1124EC5FFD4F40819A
:10893000518162817381FE01E356FD4F4083518373
:1089400062837383C7010E94D21BCE01DF91CF9156
:108950001F910F91FF90EF900C94113B0E9414AD6A
:10896000C7010E94B51C1A8284EA9EE1DF91CF9173
:108970001F910F91FF90EF908EC48FEF8EBD0DB4BD
:1089800007FEFDCF8EB508958EBD0DB407FEFDCF59
:10899000089561E0FC0180810C945FC2FC0122819A
:1089A000322F306A36953CBD20FD06C031E02630BE
:1089B00009F430E0232F01C020E02DBD60E0FC0170
:1089C00080810C945FC2CF92DF92EF92FF920F935F
:1089D0001F93CF93DF93EC018B017A010E9406C3B2
:1089E0006B01CBDF8B838F3F49F40E9406C36C1968
:1089F0007D096D327140A8F381E144C08E3F11F0D2
:108A00008FE040C0E114F104D9F0C70101972FEFC6
:108A10002EBDF8014FEF9F01201B310B281739079E
:108A200038F40DB407FEFDCF2EB521934EBDF3CF24
:108A30000DB407FEFDCF2EB5F801E80FF91F208316
:108A4000D801E00EF11EC12CD12CAE15BF0579F076
:108A50008D91ED2DFF27E827EE0FFF1FE757F04E12
:108A600085919491DC2CCC24C826D926EECF85DFC5
:108A7000082F10E0102F002780DF082BC016D1062A
:108A800031F080E28983CE0184DF80E003C0CE0133
:108A900080DF81E0DF91CF911F910F91FF90EF90E8
:108AA000DF90CF9008950F931F93CF93DF93EB0147
:108AB0000E9406C38B0161DF8F3F49F00E9406C30D
:108AC000601B710B6C177D07B0F380E001C081E083
:108AD000DF91CF911F910F910895CF92DF92FF9276
:108AE0000F931F93CF93DF9300D01F92CDB7DEB7C4
:108AF0006C01F62E29833A834B835C834FDF6CE253
:108B000071E0C601D0DF8F2D80643EDF08E110E008
:108B10005C814B813A812981DA01C901002E04C0B0
:108B2000B695A795979587950A94D2F729833A83A6
:108B30004B835C8329DF0850110929813A814B81DD
:108B40005C81083F8FEF180739F7FF2029F0E8E034
:108B5000FE1621F08FEF03C085E901C087E814DF1E
:108B6000FCE0FF1201C009DF10E007DFF60183839C
:108B700087FF04C01F3F11F01F5FF7CF0F900F90CA
:108B80000F900F90DF91CF911F910F91FF90DF9089
:108B9000CF900895BF92CF92DF92EF92FF920F9302
:108BA0001F93CF93DF93EC01B62E1C82198248836A
:108BB0000E9406C38B0161E088810E9426C2CE011B
:108BC000E8DE60E082E30E9426C261E083E30E9467
:108BD00026C261E084E30E9426C261E085E30E9430
:108BE00026C261E085E30E945FC285E08A8382E558
:108BF0008CBD1DBC6AE0F62E8FEFC6DEFA94E1F75D
:108C000020E030E0A90160E0CE0167DFF82E8B8321
:108C100081E0F81649F00E9406C3601B710B613DAC
:108C2000774070F381E046C02AEA31E040E050E04E
:108C300068E0CE0152DF82FF02C0FC820CC054E02B
:108C4000F52E9BDE8B83FA94E1F78A3A11F082E0ED
:108C500031C082E08C838C81823031F4C12CD12CE4
:108C6000E12C40E4F42E03C0C12CD12C760120E08D
:108C700030E0A90167E3CE0130DFA701960169E288
:108C8000CE012BDF8B83882349F00E9406C3601B33
:108C9000710B613D774058F38AE00CC08C818230C3
:108CA000B1F420E030E0A9016AE3CE0116DF8823A9
:108CB00029F088E08983CE016CDE14C05EDE807C02
:108CC000803C11F483E08C8358DE57DE56DECE0103
:108CD00060DE86E08B1518F488E1898303C0BA82D0
:108CE00081E001C080E0DF91CF911F910F91FF9053
:108CF000EF90DF90CF90BF900895AF92BF92CF9248
:108D0000DF92EF92FF920F931F93CF93DF93EC01CB
:108D10006A017B0189018C81833039F0F9E0CC0C48
:108D2000DD1CEE1CFF1CFA95D1F773E0B72EE4E0D2
:108D3000AE2EBA94A701960161E1CE01CEDE882362
:108D400011F0A98207C040E052E0B801CE013BDE3D
:108D500081110EC0CE01BB2049F01BDE20E030E0C7
:108D6000A9016CE0CE01B9DE1982E3CF12DE80E00A
:108D7000DF91CF911F910F91FF90EF90DF90CF90F7
:108D8000BF90AF900895CF93DF93EC016EBD20E0CC
:108D900030E00DB407FEFDCFFA01E20FF31F808132
:108DA0008EBD0DB407FEFDCF81818EBD2E5F3F4F7E
:108DB000211582E0380769F70DB407FEFDCF8FEF6C
:108DC000E3DD8FEFE1DDD9DD8B838F71853031F00D
:108DD00083E18983CE01DDDD80E001C081E0DF91A8
:108DE000CF9108950F931F93CF93DF93EC018901E7
:108DF0008C81833039F0B9E0440F551F661F771F0F
:108E0000BA95D1F79A01AB0168E1CE0166DE8823FD
:108E100011F086E01EC0A8016EEFCE01B4DF8823FA
:108E2000C9F068E572E0CE013EDE182F811102C064
:108E300087E10FC020E030E0A9016DE0CE014DDEFA
:108E4000811106C09ADD811103C0CE01A2DD05C0EB
:108E500086E18983CE019DDD10E0812FDF91CF91E6
:108E60001F910F910895FC016591759185919491E1
:108E700008952F923F924F925F926F927F928F92BE
:108E80009F92AF92BF92CF92DF92EF92FF920F9399
:108E90001F93CF93DF9300D000D0CDB7DEB71C0176
:108EA000FC01EA58FD4D14919C01220F331F220F43
:108EB000331F3E832D832759334F4901F901108217
:108EC00011821282138225E73CE041E75CE06DE607
:108ED0007CE089E69CE00E9413BE8D819E818B57C9
:108EE0009D4DC1DF6B017C01612F772767FD709578
:108EF000872F972F0E9417C92B013C012D813E819E
:108F00002C5C334F590120E030E040EC5FE3C701B7
:108F1000B6010E944ACBA30192010E944ACBF501FF
:108F200060837183828393832D813E8121523A4FE6
:108F30003C832B83F90160817181828193816093ED
:108F4000A1057093A2058093A3059093A40520E04A
:108F500030E040E752E40E947CC825E5C22E2CE0B8
:108F6000D22E7B018C0120E43CE04CE35CE068E322
:108F70007CE084E39CE00E9431B40E949EACF4014A
:108F8000108211821282138225E73CE041E75CE007
:108F90006DE67CE089E69CE00E9413BE2D813E8157
:108FA00027583D4D3A832983C9015DDF9058A301BD
:108FB00092010E944ACBF50160837183828393837F
:108FC00020E030E040E752E46091A1057091A205F5
:108FD0008091A3059091A4050E947CC87B018C011F
:108FE00020E43CE04CE35CE068E37CE084E39CE06C
:108FF0000E9431B40E949EAC89819A8134DF9B012A
:10900000AC010E949CC7A30192010E944ACBF501CA
:10901000608371838283938320E030E040E05FE3EC
:10902000EB81FC8160817181828193810E944ACBB6
:109030006093A1057093A2058093A3059093A40566
:1090400020E030E040E752E40E947CC87B018C01C4
:1090500020E43CE04CE35CE068E37CE084E39CE0FB
:109060000E9431B40E949EAC8D819E818F569D4D91
:10907000FADE0D811E81035A134FF80120813181E0
:10908000428153810E949CC7F40160837183828373
:1090900093838D819E8187559D4DE5DE2D813E8197
:1090A0002D533A4F7901F80120813181428153815A
:1090B0000E949CC7F70160837183828393838D81B3
:1090C0009E8183569D4DCFDE2D813E8129543A4F9E
:1090D0007901F80120813181428153810E949CC72E
:1090E000F7016083718382839383F401808191818E
:1090F000A281B381F50180839183A283B38310920F
:10910000A1051092A2051092A3051092A4050E9439
:1091100017A5F101E65AF34F81E0808326960FB63A
:10912000F894DEBF0FBECDBFDF91CF911F910F919D
:10913000FF90EF90DF90CF90BF90AF909F908F9077
:109140007F906F905F904F903F902F900895FC011B
:109150002491222341F03091C00035FFFCCF2093B1
:10916000C6000196F4CF22E030E085EE9FE00C943B
:1091700020A4FC012491222341F03091C00035FF4E
:10918000FCCF2093C6000196F4CF2AE030E085EEB4
:109190009FE00C9476A32091890A30918A0A2430AA
:1091A00031050CF077C040918B0A50918C0A60E633
:1091B000649F9001659F300D1124BC01C9018D563B
:1091C000954F0E9415D0E5EBF2E28491882341F09F
:1091D0009091C00095FFFCCF8093C6003196F5CFEB
:1091E000E0917A0CF0E0EE0FFF1FE45EFD4F01907E
:1091F000F081E02DEA5DFE4F0190F081E02D849139
:10920000882341F09091C00095FFFCCF8093C60069
:109210003196F5CF80918B0A90918C0A20E6289F99
:10922000F001299FF00D1124ED56F54F819188230F
:1092300039F09091C00095FFFCCF8093C600F6CF27
:10924000E4E7F2E28491882341F09091C00095FF19
:10925000FCCF8093C6003196F5CF8091C00085FF8A
:10926000FCCF8AE08093C60080918B0A90918C0A93
:10927000019664E070E00E9440CC90938C0A809349
:109280008B0A8091890A90918A0A019690938A0AA2
:109290008093890A08952091890A30918A0A24309E
:1092A00031050CF077C040918B0A50918C0A60E632
:1092B000649F9001659F300D1124BC01C9018D563A
:1092C000954F0E9475CFE5EBF2E28491882341F03F
:1092D0009091C00095FFFCCF8093C6003196F5CFEA
:1092E000E0917A0CF0E0EE0FFF1FE45EFD4F01907D
:1092F000F081E02DEA5DFE4F0190F081E02D849138
:10930000882341F09091C00095FFFCCF8093C60068
:109310003196F5CF80918B0A90918C0A20E6289F98
:10932000F001299FF00D1124ED56F54F819188230E
:1093300039F09091C00095FFFCCF8093C600F6CF26
:10934000E2E7F2E28491882341F09091C00095FF1A
:10935000FCCF8093C6003196F5CF8091C00085FF89
:10936000FCCF8AE08093C60080918B0A90918C0A92
:10937000019664E070E00E9440CC90938C0A809348
:109380008B0A8091890A90918A0A019690938A0AA1
:109390008093890A08959B9AA3980895FCDF40E082
:1093A00052EC61E070E085EE9FE00E942EA2ECE6B8
:1093B000F2E28491882341F09091C00095FFFCCFA8
:1093C0008093C6003196F5CF8091C00085FFFCCF19
:1093D0008AE08093C60025EB32E2F901849188236C
:1093E00041F09091C00095FFFCCF8093C60031966C
:1093F000F5CF84B780FF20C0A0917A0CB0E0AA0F0F
:10940000BB1FA45EBD4FED91FC91E85DFE4F019046
:10941000F081E02D9491992341F04091C00045FFE7
:10942000FCCF9093C6003196F5CF9091C00095FF88
:10943000FCCF9AE09093C60081FF20C0A0917A0CE7
:10944000B0E0AA0FBB1FA45EBD4FED91FC91E65D9D
:10945000FE4F0190F081E02D9491992341F04091CD
:10946000C00045FFFCCF9093C6003196F5CF909198
:10947000C00095FFFCCF9AE09093C60082FF20C009
:10948000A0917A0CB0E0AA0FBB1FA45EBD4FED9176
:10949000FC91E45DFE4F0190F081E02D94919923C1
:1094A00041F04091C00045FFFCCF9093C60031963B
:1094B000F5CF9091C00095FFFCCF9AE09093C60045
:1094C00083FF20C0A0917A0CB0E0AA0FBB1FA45E5E
:1094D000BD4FED91FC91E25DFE4F0190F081E02DDA
:1094E0009491992341F04091C00045FFFCCF9093A7
:1094F000C6003196F5CF9091C00095FFFCCF9AE061
:109500009093C60085FF20C0A0917A0CB0E0AA0F0E
:10951000BB1FA45EBD4FED91FC91E05DFE4F01903D
:10952000F081E02D8491882341F09091C00095FF57
:10953000FCCF8093C6003196F5CF8091C00085FFA7
:10954000FCCF8AE08093C60014BEE1E2F7E084918C
:10955000882341F09091C00095FFFCCF8093C60016
:109560003196F5CFE8E2F7E08491882341F09091BD
:10957000C00095FFFCCF8093C6003196F5CF809157
:10958000C00085FFFCCF8AE08093C600F90184917A
:10959000E5EBF2E2882349F09091C00095FFFCCF03
:1095A0008093C60031968491F5CFA0917A0CB0E0FB
:1095B000AA0FBB1FA45EBD4FED91FC91EC5CFE4F6A
:1095C0000190F081E02D8491882341F09091C000BA
:1095D00095FFFCCF8093C6003196F5CFE7E5F2E228
:1095E0008491882341F09091C00095FFFCCF809337
:1095F000C6003196F5CFA0917A0CB0E0AA0FBB1F40
:10960000A45EBD4FED91FC91EE5CFE4F0190F081A8
:10961000E02D4491442341F05091C00055FFFCCF10
:109620004093C6003196F5CFE0E4F2E284918823BE
:1096300041F09091C00095FFFCCF8093C600319619
:10964000F5CF8091C00085FFFCCF8AE08093C600F3
:10965000E5E3F2E28491882341F09091C00095FF08
:10966000FCCF8093C6003196F5CFE9E2F2E2849117
:10967000882341F09091C00095FFFCCF8093C600F5
:109680003196F5CF8091C00085FFFCCF8AE08093B2
:10969000C600F9012491E5EBF2E2222349F0809122
:1096A000C00085FFFCCF2093C60031962491F5CFF2
:1096B000E0917A0CF0E0EE0FFF1FE45EFD4F0190A9
:1096C000F081E02DEA5CFE4F0190F081E02D849165
:1096D000882341F09091C00095FFFCCF8093C60095
:1096E0003196F5CF0E9412B04AE050E0BC0185EE01
:1096F0009FE00E944AA3E0917A0CF0E0EE0FFF1F7A
:10970000E45EFD4F0190F081E02DE85CFE4F01909A
:10971000F081E02D8491882341F09091C00095FF65
:10972000FCCF8093C6003196F5CF4AE050E060ED63
:1097300074E085EE9FE00E944AA38091C00085FFFF
:10974000FCCF8AE08093C60010928F0A1092900A94
:109750001092910A1092920A0E9451A00E94239C9A
:109760000E94CB290E94E1B30E9400AF0E9459845D
:10977000489913C0FFEF23ED80E3F1502040804073
:10978000E1F700C00000489911C06A9A729A0E94DD
:109790009483489BFECF729808959FEFE3EDF0E32A
:1097A0009150E040F040E1F700C000000895809142
:1097B000830A9091840A60E070E001960C94CCCC0E
:1097C0008091830A9091840A4AE050E060E070E062
:1097D00001960C9434CE682F772767FD7095209101
:1097E0008D0A30918E0A40E6429FC001439F900D42
:1097F00011248D56954F0E9401D09093840A809336
:10980000830A21E0892B09F420E0822F08950E9429
:1098100006C360937F0A7093800A8093810A9093B5
:10982000820A08950E9406C360937F0A7093800A9B
:109830008093810A9093820AE0918D0AF0918E0ABA
:10984000E157F54F8081811121C0E0917A0CF0E061
:10985000EE0FFF1FE45EFD4F0190F081E02DE65C0E
:10986000FE4F0190F081E02D8491882341F090918A
:10987000C00095FFFCCF8093C6003196F5CF809154
:10988000C00085FFFCCF8AE08093C600089585EE76
:109890009FE00E9480A2E0917A0CF0E0EE0FFF1FA3
:1098A000E45EFD4F0190F081E02DE659FE4F0190FE
:1098B000F081E02D8491882341F09091C00095FFC4
:1098C000FCCF8093C6003196F5CF4091180C509193
:1098D000190C60911A0C70911B0C4F5F5F4F6F4F0A
:1098E0007F4F2AE030E085EE9FE00E941FA3809129
:1098F000C00085FFFCCF8AE08093C60093CF8F9293
:109900009F92AF92BF92CF92DF92EF92FF920F930E
:109910001F93CF93DF93B6EAEB2EB7E0FB2E09E659
:109920001CE0C4E3DCE08FE7C82E8CE0D82EF70102
:1099300081917F0150DF882311F139DF4B015C01F8
:10994000F6018081811103C06091130C01C061E0B8
:1099500070E080E090E00E9417C9F8012081318119
:10996000428153810E944ACB9B01AC01C501B401E5
:109970000E949CC7688379838A839B8309C0F8010E
:1099800080819181A281B38188839983AA83BB83DB
:109990000C5F1F4F2496FFEFCF1ADF0A8AEAE81602
:1099A00087E0F80621F686E416DF8823D1F0FFDE93
:1099B0006B017C016093240C7093250C8093260C22
:1099C0009093270C20E030E0A9010E9478CA181675
:1099D00044F4C092A105D092A205E092A305F092B2
:1099E000A405DF91CF911F910F91FF90EF90DF9031
:1099F000CF90BF90AF909F908F90089580DF89E4C3
:109A0000EADE882351F0D3DE6093280C7093290C92
:109A100080932A0C90932B0C08C01092280C109263
:109A2000290C10922A0C10922B0C8AE4D4DE882385
:109A300051F0BDDE60932C0C70932D0C80932E0C96
:109A400090932F0C089510922C0C10922D0C1092C4
:109A50002E0C10922F0C0895CF92DF92EF92FF926E
:109A6000CF93DF93EC01C090C305D090C405E09084
:109A7000C505F090C605A7019601688179818A81A4
:109A80009B810E9475C887FF04C0C882D982EA8280
:109A9000FB82C090C705D090C805E090C905F09042
:109AA000CA05A70196016C817D818E819F810E94EC
:109AB00075C887FF04C0CC82DD82EE82FF8220E081
:109AC00030E0A9016091CB057091CC058091CD0566
:109AD0009091CE050E949CC76B017C019B01AC015B
:109AE000688579858A859B850E9475C887FF04C033
:109AF000C886D986EA86FB86C090B705D090B8059F
:109B0000E090B905F090BA05A701960168817981C6
:109B10008A819B810E9478CA181624F4C882D9824F
:109B2000EA82FB82C090BB05D090BC05E090BD05E9
:109B3000F090BE05A70196016C817D818E819F8189
:109B40000E9478CA181624F4CC82DD82EE82FF824D
:109B5000C090BF05D090C005E090C105F090C2054F
:109B6000A7019601688579858A859B850E9478CAB8
:109B7000181624F4C886D986EA86FB86DF91CF9131
:109B8000FF90EF90DF90CF900895CF92DF92EF9209
:109B9000FF920F931F9384E39CE05EDF0E9406C355
:109BA00060937F0A7093800A8093810A9093820A5F
:109BB0002091340C3091350C4091360C5091370C7B
:109BC0006091690C70916A0C80916B0C90916C0C97
:109BD0000E9475C8811179C02091380C3091390CE0
:109BE00040913A0C50913B0C60916D0C70916E0C51
:109BF00080916F0C9091700C0E9475C8811165C0A6
:109C000020E030E040E752E46091A1057091A205A8
:109C10008091A3059091A4050E947CC825E5C22EE1
:109C20002CE0D22E7B018C0120E43CE04CE35CE094
:109C300068E37CE084E39CE00E9431B48091340CC2
:109C40009091350CA091360CB091370C8093690C33
:109C500090936A0CA0936B0CB0936C0C8091380CB1
:109C60009091390CA0913A0CB0913B0C80936D0C03
:109C700090936E0CA0936F0CB093700C80913C0C81
:109C800090913D0CA0913E0CB0913F0C8093710CD3
:109C90009093720CA093730CB093740C8091400C51
:109CA0009091410CA091420CB091430C8093750CA3
:109CB0009093760CA093770CB093780C1F910F9132
:109CC000FF90EF90DF90CF9008956091DD05709147
:109CD000DE05882777FD8095982F0E9417C920916F
:109CE000A1053091A2054091A3055091A4050E94C1
:109CF0004ACB20E030E040E752E40E947CC820E0FC
:109D000030E048EC52E488CFCF92DF92EF92FF929E
:109D1000CF93C62FE091550CF0E0882309F4C2C020
:109D2000DF01AF5AB34F8C91811196C18091690CBC
:109D300090916A0CA0916B0CB0916C0C8093340CD8
:109D40009093350CA093360CB093370C80916D0C2A
:109D500090916E0CA0916F0CB091700C8093380CA8
:109D60009093390CA0933A0CB0933B0C8091710CFA
:109D70009091720CA091730CB091740C80933C0C78
:109D800090933D0CA0933E0CB0933F0CC090750C8B
:109D9000D090760CE090770CF090780CC092400C4C
:109DA000D092410CE092420CF092430CEE0FFF1F58
:109DB000EE0FFF1FE153FA4F208131814281538121
:109DC000662349F06091AF057091B0058091B105AF
:109DD0009091B20508C06091B3057091B40580916F
:109DE000B5059091B6050E947CC89B01AC01C701E6
:109DF000B6010E949CC76093750C7093760C80939B
:109E0000770C9093780C85E79CE00E94B8BEC090D8
:109E1000A105D090A205E090A305F090A40520E054
:109E200030E040E752E46091AB057091AC05809161
:109E3000AD059091AE050E944ACB6093A105709349
:109E4000A2058093A3059093A405E091550CF0E042
:109E5000EF5AF34F81E0808398DE20914D0C3091D2
:109E60004E0C40914F0C5091500C6091710C7091C0
:109E7000720C8091730C9091740C0E949BC760933C
:109E8000710C7093720C8093730C9093740C25E793
:109E90003CE041E75CE06DE67CE089E69CE00E9406
:109EA00013BED1C0EF5AF34F8081882309F4D4C088
:109EB0008091690C90916A0CA0916B0CB0916C0C24
:109EC0008093340C9093350CA093360CB093370CE0
:109ED00080916D0C90916E0CA0916F0CB091700CF4
:109EE0008093380C9093390CA0933A0CB0933B0CB0
:109EF0006091710C7091720C8091730C9091740C44
:109F000060933C0C70933D0C80933E0C90933F0CFF
:109F1000C090750CD090760CE090770CF090780C97
:109F2000C092400CD092410CE092420CF092430C53
:109F300020914D0C30914E0C40914F0C5091500C93
:109F40000E949CC76093710C7093720C8093730C89
:109F50009093740C25E73CE041E75CE06DE67CE023
:109F600089E69CE00E9413BEF090550CCC2389F04A
:109F70002091450C3091460C4091470C5091480C73
:109F80006091AF057091B0058091B1059091B205D7
:109F900010C02091490C30914A0C40914B0C5091CB
:109FA0004C0C6091B3057091B4058091B50590910A
:109FB000B6050E949CC724E0F29EF0011124E153F3
:109FC000FA4F20813181428153810E947CC89B01DC
:109FD000AC016091750C7091760C8091770C90912A
:109FE000780C0E949BC76093750C7093760C8093DD
:109FF000770C9093780C85E79CE00E94B8BEC090E7
:10A00000A105D090A205E090A305F090A40520E062
:10A0100030E040E752E46091A7057091A805809177
:10A02000A9059091AA050E944ACB6093A10570935F
:10A03000A2058093A3059093A405E091550CF0E050
:10A04000EF5AF34F1082A1DDC092A105D092A20574
:10A05000E092A305F092A405CF91FF90EF90DF90DE
:10A06000CF900895AF92BF92CF92DF92EF92FF927E
:10A070000F931F93CF93DF93D82F20912C0C309107
:10A080002D0C40912E0C50912F0C6091280C70914A
:10A09000290C80912A0C90912B0C0E9485CAC62F06
:10A0A000172F082FF92E6091DD057091DE058827A6
:10A0B00077FD8095982F0E9417C92091A1053091B6
:10A0C000A2054091A3055091A4050E944ACB20E02F
:10A0D00030E040E752E40E947CC820E030E048ECE9
:10A0E00052E40E947CC82091550C2F93DF93FF927D
:10A0F0000F931F93CF935B016C0142E0E42E01E0CC
:10A1000020E048E25CE064E37CE089E69CE00E94B9
:10A11000F4338091340C9091350CA091360CB091B1
:10A12000370C8093690C90936A0CA0936B0CB093DE
:10A130006C0C8091380C9091390CA0913A0CB09134
:10A140003B0C80936D0C90936E0CA0936F0CB093AE
:10A15000700C80913C0C90913D0CA0913E0CB09104
:10A160003F0C8093710C9093720CA093730CB0937E
:10A17000740C8091400C9091410CA091420CB091D4
:10A18000430C8093750C9093760CA093770CB0934E
:10A19000780C0E9406C360937F0A7093800A8093B4
:10A1A000810A9093820A0F900F900F900F900F905A
:10A1B0000F90DF91CF911F910F91FF90EF90DF9063
:10A1C000CF90BF90AF900895F8940E946E2A179A8E
:10A1D00010925A0C169A10925B0C159A10925C0C05
:10A1E000149A60E087E40E9426C2EBEBF2E28491CD
:10A1F000882341F09091C00095FFFCCF8093C6006A
:10A200003196F5CFE0917A0CF0E0EE0FFF1FE45E9F
:10A21000FD4F0190F081E02DEA59FE4F0190F08151
:10A22000E02D8491882341F09091C00095FFFCCFF0
:10A230008093C6003196F5CF8091C00085FFFCCF9A
:10A240008AE08093C600E0917A0CF0E0EE0FFF1FE9
:10A25000E45EFD4F0190F081E02DE653FF4F8081D9
:10A2600091810E94F6837894C6E0D0E021972097F0
:10A2700049F068EC70E080E090E00E9435C30E94F5
:10A280008584F4CFF894FFCF2F923F924F925F9244
:10A290006F927F928F929F92AF92BF92CF92DF92F6
:10A2A000EF92FF920F931F93CF93DF93CDB7DEB75B
:10A2B0006E970FB6F894DEBF0FBECDBF30E6D32E3B
:10A2C00044E0E42EF12C5AE0C52EBB24B3948091D7
:10A2D0006610909167102091681030916910821B70
:10A2E000930B8F779927892B09F467C28091890A8C
:10A2F00090918A0A04970CF060C285EE9FE00E945C
:10A3000064A28093880A2091860A3091870A8A3055
:10A3100061F08D3051F08A3321F49091850A9923B0
:10A3200021F02F3531050CF442C12115310509F416
:10A330005CC180918B0A90918C0AD89E4001D99E75
:10A34000900C1124F401E20FF31FED56F54F10822B
:10A350002091850A211126C11092850AFC01E1573E
:10A36000F54F108284010D56154F6EE470E0C80160
:10A370000E9401D00097F1F19093840A8093830AA0
:10A38000801B910B880D991D4AE050E060E070E061
:10A390008C56954F0E9434CE60931C0C70931D0C0C
:10A3A00080931E0C90931F0C4090180C5090190C29
:10A3B00060901A0C70901B0C2FEF421A520A620A1E
:10A3C000720A00918B0A10918C0A64157505860536
:10A3D000970509F40DC1D09EC001D19E900D1124A6
:10A3E00060E272E28D56954F0E94ACCF892B09F046
:10A3F000FFC0A9C16AE270E0C8010E9401D0892BA8
:10A4000009F451C0EBEBF2E28491882341F0909182
:10A41000C00095FFFCCF8093C6003196F5CFE09148
:10A420007A0CF0E0EE0FFF1FE45EFD4F0190F0812B
:10A43000E02DEC5BFE4F0190F081E02D84918823AC
:10A4400041F09091C00095FFFCCF8093C6003196FB
:10A45000F5CF4091180C5091190C60911A0C709125
:10A460001B0C2AE030E085EE9FE00E941FA3809144
:10A47000C00085FFFCCF8AE08093C6001092870A57
:10A480001092860A0DC380911C0C90911D0CA09116
:10A490001E0CB0911F0C8093180C9093190CA09374
:10A4A0001A0CB0931B0C80918B0A90918C0AD89E49
:10A4B0008001D99E100D1124C8018D56954F4C0175
:10A4C00067E470E00E9401D0009709F447C09093C0
:10A4D000840A8093830A88199909800F911F60E08C
:10A4E00070E08C56954F0E94CCCC0E94E4C864303A
:10A4F0007105A0F58091710A882381F1E0917A0CB1
:10A50000F0E0EE0FFF1FE45EFD4F0190F081E02DC3
:10A51000E859FE4F0190F081E02D8491882341F0AD
:10A520009091C00095FFFCCF8093C6003196F5CF87
:10A530008091C00085FFFCCFC092C600E0917A0CEC
:10A54000F0E0EE0FFF1FE45EFD4F0190F081E02D83
:10A55000E453FF4F808191810E94E98300918B0A2F
:10A5600010918C0AD09EC001D19E900D11246EE2F4
:10A5700077E08D56954F0E940CD0892B09F424DE8C
:10A58000C8010196B7010E9440CC90938C0A809339
:10A590008B0A8091890A90918A0A019690938A0A7F
:10A5A0008093890A1092870A1092860A90CE8B3384
:10A5B00011F4B092850A9091850A911188CE40914C
:10A5C0008B0A50918C0AB9016F5F7F4F7093870A95
:10A5D0006093860AD49EF001D59EF00D1124E20FFF
:10A5E000F31FED56F54F808372CE1092850A58C244
:10A5F000D09E4001D19E900C1124C4018D56954FE0
:10A600003C016AE270E00E9401D0009709F03EC070
:10A61000EBEBF2E28491882341F09091C00095FF2A
:10A62000FCCF8093C6003196F5CFE0917A0CF0E034
:10A63000EE0FFF1FE45EFD4F0190F081E02DEE5B19
:10A64000FE4F0190F081E02D8491882341F090919C
:10A65000C00095FFFCCF8093C6003196F5CF4091A6
:10A66000180C5091190C60911A0C70911B0C2AE077
:10A6700030E085EE9FE00E941FA38091C00085FF1F
:10A68000FCCF8AE08093C60002D9F8CE20E010E02B
:10A69000F401E20FF11DED56F54F30813A3219F019
:10A6A0002F5F1327F5CF9093840A8093830A86192E
:10A6B0009709880D991D60E070E08C56954F0E94B7
:10A6C000CCCC0E94E4C8212F30E02617370709F4CC
:10A6D000DACEEBEBF2E28491882341F09091C00056
:10A6E00095FFFCCF8093C6003196F5CFE0917A0CB0
:10A6F000F0E0EE0FFF1FE45EFD4F0190F081E02DD2
:10A70000E05CFE4F0190F081E02D8491882341F0C0
:10A710009091C00095FFFCCF8093C6003196F5CF95
:10A720004091180C5091190C60911A0C70911B0CEF
:10A730002AE030E085EE9FE00E941FA38091C000D8
:10A7400085FFFCCF9ECFEBEBF2E28491882341F0B2
:10A750009091C00095FFFCCF8093C6003196F5CF55
:10A76000E0917A0CF0E0EE0FFF1FE45EFD4F0190E8
:10A77000F081E02DE25CFE4F0190F081E02D8491AC
:10A78000882341F09091C00095FFFCCF8093C600D4
:10A790003196F5CF4091180C5091190C60911A0C1C
:10A7A00070911B0C2AE030E085EE9FE00E941FA311
:10A7B0008091C00085FFFCCF64CF80918B0C8823F3
:10A7C00009F46EC18091860A9091870A892B09F05D
:10A7D00067C18091890A90918A0A892B11F410929D
:10A7E0006F0AF8EE2F2EF3E03F2E412C512CACE3F4
:10A7F000CA2ED12CE12CF12C8E010F5F1F4FE0E609
:10A800006E2E772473944091260F5091270F6091FC
:10A81000280F7091290F80911E0F90911F0FA0910A
:10A82000200FB091210F481759076A077B0708F0DE
:10A8300037C18091890A90918A0A04970CF030C13F
:10A8400080916F0A81112CC18091790E90917A0EBE
:10A85000A0917B0EB0917C0E8093260F9093270FD2
:10A86000A093280FB093290F81E79EE00E94091B57
:10A87000482F8093880A8A30B9F04D30A9F04332CE
:10A8800029F42091850A222379F002C04A33C9F3C2
:10A890002091860A3091870A2F3531052CF48F3F9D
:10A8A000AFEF9A0709F0DEC04091260F5091270FB5
:10A8B0006091280F7091290F80911E0F90911F0FAA
:10A8C000A091200FB091210F481759076A077B0705
:10A8D00008F48EC0E0917A0CF0E0EE0FFF1FE45E0A
:10A8E000FD4F0190F081E02DEA5BFE4F0190F08179
:10A8F000E02D8491882341F09091C00095FFFCCF1A
:10A900008093C6003196F5CF8091C00085FFFCCFC3
:10A91000BAE0B093C6000E9406C36093730A7093B6
:10A92000740A8093750A9093760A8090770A9090C3
:10A93000780AA090790AB0907A0A681979098A0988
:10A940009B09A20191010E9453CC49015A01CA01FD
:10A95000B901A70196010E9453CCCA01B901A70110
:10A9600096010E9453CC7F936F93C501B40120E1FF
:10A970003EE040E050E00E9453CC3F932F93ACE088
:10A98000B2E2BF93AF931F930F930E9439D0E5EBD0
:10A99000F2E284910FB6F894DEBF0FBECDBF8823DC
:10A9A00049F09091C00095FFFCCF8093C60031968E
:10A9B0008491F5CFF8018191882339F09091C000FE
:10A9C00095FFFCCF8093C600F6CF8091C00085FF35
:10A9D000FCCF3AE03093C600C8010E94B98389E8F1
:10A9E0009CE00E94664461E089E89CE00E94293E68
:10A9F0008091880A833211F470926F0A2091860A3E
:10AA00003091870A2115310509F4EFCD80918B0A29
:10AA100090918C0A689EF001699EF00D1124E20F5E
:10AA2000F31FED56F54F1082FC01E157F54F708290
:10AA30002091890A30918A0A2F5F3F4F30938A0A0A
:10AA40002093890A019664E070E00E9440CC9093C4
:10AA50008C0A80938B0A1092850A1092870A1092B2
:10AA6000860AD1CE4B3311F47092850A4091850A43
:10AA70004111C5CE40918B0A50918C0AB9016F5F8C
:10AA80007F4F7093870A6093860A649EF001659EEB
:10AA9000F00D1124E20FF31FED56F54F8083B3CE76
:10AAA0006E960FB6F894DEBF0FBECDBFDF91CF918B
:10AAB0001F910F91FF90EF90DF90CF90BF90AF90DC
:10AAC0009F908F907F906F905F904F903F902F90CE
:10AAD0000895CF92DF92EF92FF920F931F93CF933F
:10AAE000C82F8091890A90918A0A03970CF4CCDBD5
:10AAF0000E9406C300917B0A10917C0A20917D0A76
:10AB000030917E0AC0907F0AD090800AE090810A3E
:10AB1000F090820A6C197D098E099F0906171707A4
:10AB20002807390728F4012B022B032B09F04CDBF3
:10AB300040919D0550919E0560919F057091A005E3
:10AB4000452B462B472B19F10E9406C300917F0A23
:10AB50001091800A2091810A3091820A601B710B4A
:10AB6000820B930B00919D0510919E0520919F05EE
:10AB70003091A005061717072807390740F4909170
:10AB8000B7108091B610981302C0CC2349F0CF9132
:10AB90001F910F91FF90EF90DF90CF900C9415B420
:10ABA000179A10925A0C169A10925B0C159A1092E2
:10ABB0005C0C149AECCF0E946E2A8091710A81116C
:10ABC00051C081E08093710A8091180C9091190C0A
:10ABD000A0911A0CB0911B0C8093140C9093150C3F
:10ABE000A093160CB093170CEBEBF2E28491882340
:10ABF00041F09091C00095FFFCCF8093C600319644
:10AC0000F5CFE0917A0CF0E0EE0FFF1FE45EFD4F10
:10AC10000190F081E02DE859FE4F0190F081E02D88
:10AC20008491882341F09091C00095FFFCCF8093E0
:10AC3000C6003196F5CF8091C00085FFFCCF8AE039
:10AC40008093C600E0917A0CF0E0EE0FFF1FE45E07
:10AC5000FD4F0190F081E02DE453FF4F8081918101
:10AC60000C94E98308958091710A0895CF93DF933E
:10AC7000EC018091550C8093720A84E50E94EB4BA5
:10AC8000811102C080E0B8C00E94D74B0E94E9C881
:10AC90006093720A6623B1F3E5EBF2E284918823B4
:10ACA00041F09091C00095FFFCCF8093C600319693
:10ACB000F5CFCD36D10509F454C0BCF4C836D10562
:10ACC00061F1C936D10509F087C0E0917A0CF0E056
:10ACD000EE0FFF1FE45EFD4F0190F081E02DE25B7F
:10ACE000FE4F0190F081E02D38C0CA3DD10509F436
:10ACF00051C0CD3DD10509F06FC0E0917A0CF0E074
:10AD0000EE0FFF1FE45EFD4F0190F081E02DEC5A45
:10AD1000FE4F0190F081E02D5CC0E0917A0CF0E0F4
:10AD2000EE0FFF1FE45EFD4F0190F081E02DE45B2C
:10AD3000FE4F0190F081E02D8191882309F44CC0F1
:10AD40009091C00095FFFCCF8093C600F5CF909105
:10AD5000C00095FFFCCF8093C60081918111F7CF91
:10AD60003BC0E0917A0CF0E0EE0FFF1FE45EFD4F78
:10AD70000190F081E02DE85AFE4F0190F081E02D26
:10AD80008191882349F19091C00095FFFCCF809379
:10AD9000C600F6CFE0917A0CF0E0EE0FFF1FE45E04
:10ADA000FD4F0190F081E02DEE5AFE4F0190F081B1
:10ADB000E02D8191882381F09091C00095FFFCCF18
:10ADC0008093C600F6CF9091C00095FFFCCF809392
:10ADD000C60081918111F7CF40E050E06091720A86
:10ADE00085EE9FE00E9481A38091C00085FFFCCF8B
:10ADF0008AE08093C60081E0DF91CF910895CF92E1
:10AE0000DF92EF92FF922091790C2223F1F020E063
:10AE100030E040E05FE30E944ACB6B017C0120E020
:10AE200030E0A9010E9475C8882379F0A701960136
:10AE3000C701B6010E944ACB2BED3FE049E450E444
:10AE40000E944ACB9B01AC0104C020E030E040E806
:10AE50005FE360E070E080E89FE30E947CC8FF90C1
:10AE6000EF90DF90CF9008956091D3057091D40555
:10AE70008091D5059091D605C2DF6093CF05709380
:10AE8000D0058093D1059093D20508953F924F92BB
:10AE90005F926F927F928F929F92AF92BF92CF926A
:10AEA000DF92EF92FF920F931F93CF93DF93CDB773
:10AEB000DEB7E9970FB6F894DEBF0FBECDBF81E4D1
:10AEC0000E94EB4B882309F43FC082E70E94EB4BC2
:10AED0008823A9F0E3E3F7E08191882339F090918A
:10AEE000C00095FFFCCF8093C600F6CF8091C000D4
:10AEF00085FFFCCF8AE08093C6000C94B66F86E78E
:10AF00000E94EB4B8823A9F0E9E3F7E081918823C5
:10AF100039F09091C00095FFFCCF8093C600F6CF2A
:10AF20008091C00085FFFCCF8AE08093C6000C941E
:10AF3000B66F87E60E94EB4B882311F40C94B66F32
:10AF40000E9494830C94B66F87E40E94EB4B882395
:10AF500009F46EC20E94D74B0E94E4C86A307105A2
:10AF600009F4BBC09CF46230710509F44CC024F4B0
:10AF700077FF25C00C94B66F6330710509F44EC09D
:10AF80006430710509F455C00C94B66F6A357105CB
:10AF900009F4FAC154F46B30710509F4A4C06C31A2
:10AFA000710509F4A6C00C94B66F6B35710509F4F0
:10AFB000EFC16C35710509F4F0C10C94B66F809146
:10AFC000710A81110C94B66F0E947F4C8091520CD3
:10AFD0008823A9F088E50E94EB4B811110C089E518
:10AFE0000E94EB4B81110BC08AE50E94EB4B811153
:10AFF00006C085E40E94EB4B81110C94B96F0E944E
:10B00000C54D0C94B66F8091710A81110C94B66F86
:10B010000E94FE4C81E026D80C94B66F8091710A94
:10B0200081110C94B66F0E94FE4C80E01BD80C94EA
:10B03000B66FE0917A0CF0E0EE0FFF1FE45EFD4F7B
:10B040000190F081E02DE054FF4F808191810E94BA
:10B05000E98380E50E94EB4B882339F00E94D74BAF
:10B060000E94E9C84B015C0103C0812C912C540162
:10B0700083E50E94EB4B882361F00E94D74B20E0D0
:10B0800030E04AE754E40E944ACB0E94E9C84B01F1
:10B090005C010E949EAC0E9406C36B017C01C80C3F
:10B0A000D91CEA1CFB1C0E9406C360937F0A7093A4
:10B0B000800A8093810A9093820A0E9406C36C15CD
:10B0C0007D058E059F0510F00C94B66F0E949B279E
:10B0D00080E0FFDC0E948584F0CF60E081E00E9488
:10B0E000844E0C94B66F60E080E00E94844E0C9415
:10B0F000B66F8091A1059091A205A091A305B09192
:10B10000A4058093200C9093210CA093220CB09363
:10B11000230C8091DD059091DE0590937E0C809349
:10B120007D0C84E690E09093DE058093DD050E941F
:10B1300006C360937F0A7093800A8093810A90937C
:10B14000820A81E00E941EA58091690C90916A0C90
:10B15000A0916B0CB0916C0C8093340C9093350CD7
:10B16000A093360CB093370C80916D0C90916E0CBF
:10B17000A0916F0CB091700C8093380C9093390CA7
:10B18000A0933A0CB0933B0C8091710C9091720C8F
:10B19000A091730CB091740C80933C0C90933D0C77
:10B1A000A0933E0CB0933F0C8091750C9091760C5F
:10B1B000A091770CB091780C8093400C9093410C47
:10B1C000A093420CB093430C1092A1051092A205DB
:10B1D0001092A3051092A40588E50E94EB4B8823EA
:10B1E00011F090E00AC089E50E94EB4B8111F9CF84
:10B1F0008AE50E94EB4B91E098279093A505911169
:10B200000C94E86F88E50E94EB4B81110C94E86F79
:10B210008091A50581110C94EE6F89E50E94EB4B9E
:10B2200081110C94EE6F88E50E94EB4B8823D1F0DE
:10B230000E94E04B672B682B692BA1F00E94D74B33
:10B2400020915D0C30915E0C40915F0C5091600C30
:10B250000E949CC76093690C70936A0C80936B0C7E
:10B2600090936C0C89E50E94EB4B8823D1F00E94EF
:10B27000E04B672B682B692BA1F00E94D74B2091E4
:10B28000610C3091620C4091630C5091640C0E94EF
:10B290009CC760936D0C70936E0C80936F0C9093B1
:10B2A000700C8091A50581110C94F46F8AE50E94C1
:10B2B000EB4B81110C94F46F8AE50E94EB4B8823D1
:10B2C000D1F00E94E04B672B682B692BA1F00E9404
:10B2D000D74B2091650C3091660C4091670C5091D2
:10B2E000680C0E949CC76093710C7093720C8093E1
:10B2F000730C9093740C25E73CE041E75CE06DE64D
:10B300007CE089E69CE00E9413BE80E00E941EA5BE
:10B310008091200C9091210CA091220CB091230CD3
:10B320008093A1059093A205A093A305B093A405D3
:10B3300080917D0C90917E0C9093DE058093DD05CD
:10B340000E9406C360937F0A7093800A8093810AEB
:10B350009093820A0E9417A580918B0C882311F488
:10B360000C94B66F67E87CE089EF9FE00E945D80F7
:10B370008091870C9091880C892B11F40C94B66FF6
:10B380000E94F9960C94B66F1092130C0C94B66F41
:10B3900081E08093130C0C94B66F85E40E94EB4B14
:10B3A000811102C00E949EAC96EAC92E97E0D92E68
:10B3B0002DE5E22E2CE0F22E09E61CE0B12CF60180
:10B3C00081916F010E94EB4B882339F1F3E0BF12AA
:10B3D0000CC00E94D74BF8016083718382839383F2
:10B3E00085E79CE00E94B8BE18C00E94D74BF701C9
:10B3F00020813181428153810E949CC7F801608382
:10B4000071838283938325E73CE041E75CE06DE64E
:10B410007CE089E69CE00E9413BEB394F4E0EF0E5A
:10B42000F11C0C5F1F4F24E0B212C9CF0C94B66F11
:10B430008DE40E94EB4B882311F40C94BD6E0E94A6
:10B44000D74B0E94E4C86537710511F40C94296349
:10B450000CF0D0C06032710509F453C30CF071C018
:10B460006731710509F4A8C20CF044C0623171055E
:10B4700011F40C9448621CF577FF02C00C94B66F6F
:10B48000623071050CF498C16131710511F00C94B2
:10B49000B66FE0917A0CF0E0EE0FFF1FE45EFD4F17
:10B4A0000190F081E02DE853FF4F808191810E944F
:10B4B000E98317981698159814980C94B66F65310F
:10B4C000710509F46DC20CF071C26431710511F09F
:10B4D0000C94B66FE0917A0CF0E0EE0FFF1FE45E83
:10B4E000FD4F0190F081E02DE85BFE4F0190F0816F
:10B4F000E02D25C26B31710509F48AC2B4F46931BB
:10B50000710509F471C20CF075C289E89CE00E94D3
:10B51000113B0E9406C36093770A7093780A809368
:10B52000790A90937A0A0C94B66F6E31710509F41A
:10B53000AAC20CF082C36C31710509F46FC20C947D
:10B54000B66F6C35710509F4F6C7ECF46235710518
:10B5500009F495C764F46035710509F448C70CF027
:10B560005DC76A32710509F4C6C30C94B66F6435C1
:10B57000710509F48DC70CF486C76535710509F4AA
:10B58000BFC70C94B66F6B36710509F42AC764F413
:10B590006936710509F427C40CF0F3C668367105E5
:10B5A00009F4F0C30C94B66F6037710509F408C450
:10B5B00034F46D36710509F423C50C94B66F623707
:10B5C000710511F40C943D636337710511F00C940F
:10B5D000B66FE0917A0CF0E0EE0FFF1FE45EFD4FD6
:10B5E0000190F081E02DEE59FE4F0190F081E02DA9
:10B5F0000C942463623E710511F40C943C680CF0C9
:10B600005FC06B3C710511F40C947B66ACF56C3833
:10B61000710509F4D7C304F56837710511F40C946A
:10B620002A646937710511F40C942F64673771052A
:10B6300011F00C94B66FE0917A0CF0E0EE0FFF1F62
:10B64000E45EFD4F0190F081E02DE258FE4F019045
:10B65000F081E02D0C943A64683C710511F40C946F
:10B66000D865693C710511F40C945A666E3B7105FE
:10B6700011F00C94B66F5AC56F3C710511F40C941F
:10B68000386754F46D3C710511F40C94BA6614F4E7
:10B690000C9498660C941A67613D710511F40C9432
:10B6A000976714F40C946F676C3D710511F40C945A
:10B6B00007686D3D710511F40C9416680C94B66F13
:10B6C000653F31E0730711F40C94E96954F56F326A
:10B6D00091E0790711F40C94AE6984F46D32F1E0D5
:10B6E0007F0711F40C94CD6814F00C94A0696C32AF
:10B6F000714011F40C9497680C94B66F6F3581E02B
:10B70000780711F40C94616E603991E0790711F4B7
:10B710000C94E6696E35714011F00C94B66F0C9480
:10B720002A6E6835F2E07F0711F40C94316BA4F4B3
:10B73000673F31E0730711F40C94F16914F40C9431
:10B74000EE696D3F714011F00C94B66F0E949483C6
:10B75000E5EBF2E20C94FB696B38E3E07E0711F451
:10B760000C94046E3CF46335734011F40C940C6A31
:10B770000C94B66F603A33E0730709F42BC2673E4E
:10B78000734011F00C94B66F1092710A0E94FC8302
:10B790008091140C9091150CA091160CB091170C7F
:10B7A0008093180C9093190CA0931A0CB0931B0C57
:10B7B0000E94474C0C94B66F0091830A1091840A42
:10B7C0000E5F1F4F80E50E94EB4B882379F00E94AB
:10B7D000D74B0E94E9C86B017C01BB24B39461156F
:10B7E00071058105910531F4B12C04C0B12CC12C37
:10B7F000D12C760183E50E94EB4B882399F00E94BF
:10B80000D74B20E030E04AE754E40E944ACB0E9444
:10B81000E9C86B017C01AA24A39461157105810517
:10B82000910509F4A12C6AE270E0C8010E9401D0E0
:10B83000009711F0FC011082F801CF012191203214
:10B84000E1F3B11007C0A11005C0222319F00E9436
:10B85000B98310C0E0917A0CF0E0EE0FFF1FE45EB8
:10B86000FD4F0190F081E02DEE53FF4F80819181DB
:10B870000E94E98381E00E9499830E949EAC0E940D
:10B8800006C360937F0A7093800A8093810A909325
:10B89000820AC114D104E104F104D1F00E9406C36C
:10B8A0004B015C018C0C9D1CAE1CBF1C0E9406C38E
:10B8B000681579058A059B05E0F40E946D85811164
:10B8C00018C00E949B2780E004D90E948584EECF97
:10B8D0000E946B85882311F40C94B66F0E946D85CD
:10B8E00081110AC00E949B2780E0F3D80E948584C2
:10B8F000F5CF80E00E94998380918B0CE0917A0CC7
:10B90000F0E0EE0FFF1FE45EFD4F0190F081E02DAF
:10B91000882341F0EC53FF4F808191810E94E9839D
:10B920000C94B66F808191810E94E9830C94B66F6C
:10B930009091C00095FFFCCF8093C6003196849112
:10B940008111F6CF8091C00085FFFCCF8AE0809303
:10B95000C60089E89CE00E94B939E0917A0CF0E0D9
:10B96000EE0FFF1FE45EFD4F0190F081E02DE65BDE
:10B97000FE4F0190F081E02D8491882341F0909159
:10B98000C00095FFFCCF8093C6003196F5CF809123
:10B99000C00085FFFCCF8AE08093C6000C94B66F90
:10B9A00089E89CE00E940E3A0C94B66F89E89CE00E
:10B9B0000E940D3B0C94B66F0091830A1091840A8B
:10B9C0000C5F1F4F6AE270E0C8010E9401D000972F
:10B9D00011F0FC01108221E041E0B80189E89CE00F
:10B9E0000E948F3F0C94B66F89E89CE00E94183B40
:10B9F0000C94B66F80918C0C882311F40C94B66F64
:10BA000083E50E94EB4B81110C94FA6F0C94B66F96
:10BA100089E89CE00E94BC3C0C94B66F8091830A3C
:10BA20009091840A6AE270E004960E9401D08C0131
:10BA30000097D9F020918D0A30918E0A40E6429FFE
:10BA4000C001439F900D11246EE470E08D56954F18
:10BA50000E9401D060E270E00E9401D001969093B4
:10BA6000840A8093830AF80110826091830A70919E
:10BA7000840A6C5F7F4F21E040E089E89CE00E94EF
:10BA80008F3F0C94B66F80918C0C882311F40C942A
:10BA9000B66F60E089E89CE00E941F3F8091830AB6
:10BAA0009091840A6AE270E004960E9401D08C01B1
:10BAB0000097D9F020918D0A30918E0A40E6429F7E
:10BAC000C001439F900D11246EE470E08D56954F98
:10BAD0000E9401D060E270E00E9401D00196909334
:10BAE000840A8093830AF80110826091830A70911E
:10BAF000840A6C5F7F4F89E89CE00E947C3B0C9439
:10BB0000B66F80918B0C81110E949EAC0091830ACC
:10BB10001091840A0C5F1F4F6AE270E0C8010E9416
:10BB200001D07C0161E270E0C8010E9401D0009761
:10BB300019F08C010F5F1F4FE114F10411F0F701B0
:10BB4000108280E50E94EB4BF82E2091830A309101
:10BB5000840A0217130708F4F12C80918C0C8823B7
:10BB600011F40C94B66F21E02F2541E0B80189E86B
:10BB70009CE00E948F3F83E50E94EB4B8823B9F045
:10BB80002091830A3091840A2017310780F40E94A3
:10BB9000E04BAB01BC014093260F5093270F6093FD
:10BBA000280F7093290F81E79EE00E94D21B89E83D
:10BBB0009CE00E94113BF1100C94B66F0E9406C3EA
:10BBC0006093770A7093780A8093790A90937A0A3F
:10BBD0000C94B66F8091830A9091840A6AE270E0B7
:10BBE00005960E9401D08C010097D9F020918D0A12
:10BBF00030918E0A40E6429FC001439F900D112470
:10BC00006EE470E08D56954F0E9401D060E270E0C6
:10BC10000E9401D001969093840A8093830AF801D0
:10BC200010826091830A7091840A6B5F7F4F89E86C
:10BC30009CE00E9414430C94B66F0E9406C360936C
:10BC4000730A7093740A8093750A9093760A009130
:10BC5000770A1091780A2091790A30917A0A601B4C
:10BC6000710B820B930B28EE33E040E050E00E9412
:10BC700053CCCA01B9012CE330E040E050E00E940F
:10BC800053CC7F936F933F932F938DEF91E29F93CC
:10BC90008F93CE0101969F938F930E9439D0E5EB4D
:10BCA000F2E284910FB6F894DEBF0FBECDBF8823B9
:10BCB00049F09091C00095FFFCCF8093C60031966B
:10BCC0008491F5CFFE0131968191882339F09091CE
:10BCD000C00095FFFCCF8093C600F6CF8091C000D6
:10BCE00085FFFCCF8AE08093C600CE0101960E94BA
:10BCF000B9830C94B66F83E50E94EB4B882311F453
:10BD00000C94B66F0E94D74B0E94E4C8F62EE72E23
:10BD1000862F9E2D8C0180E50E94EB4B882331F00D
:10BD20000F3F110509F010F40C940B700DE010E0BA
:10BD3000EEE6F7E0819191918017910711F40C9450
:10BD4000B66F37E0E63AF307A9F70630110539F484
:10BD50008F2D9E2D9093540C8093530C04C017FF8D
:10BD600002C00C94B66F61E0802F0E9426C26F2D36
:10BD7000802F0E945FC26F2D7E2D802F0E941CC1DC
:10BD80000C94B66F88E690E00E94365681110C94B0
:10BD9000B66F83E50E94EB4B882371F00091720A25
:10BDA0000E94D74B10E0000F111F085A154F0E9438
:10BDB000E4C8F801718360830E946D2A0C94B66F09
:10BDC0000E94E45083E50E94EB4B882311F40C940D
:10BDD000B66F0E94D74B0E94E4C87093570A6093D5
:10BDE000560A0C94B66F89E690E00E94365681118F
:10BDF0000C94B66FE7EFF1E28491882341F09091C3
:10BE0000C00095FFFCCF8093C6003196F5CFE0913E
:10BE1000720A24E0E29FF0011124E05BF54F4081BB
:10BE200051816281738121E030E085EE9FE00E94C4
:10BE300020A4E4EFF1E28491882341F09091C000C6
:10BE400095FFFCCF8093C6003196F5CFE091720A42
:10BE5000F0E0EE0FFF1FE85AF54F608171818827EF
:10BE600077FD8095982F0E9417C9AB01BC0121E096
:10BE700030E085EE9FE00E9420A4E0EFF1E28491A3
:10BE8000882341F09091C00095FFFCCF8093C600BD
:10BE90003196F5CF40914A0A50914B0A60914C0A75
:10BEA00070914D0A21E030E085EE9FE00E9420A4D1
:10BEB000EDEEF1E28491882341F09091C00095FF6E
:10BEC000FCCF8093C6003196F5CF6091560A7091F1
:10BED000570A882777FD8095982F0E9417C9AB01D4
:10BEE000BC0121E030E085EE9FE00E9420A4EAEE54
:10BEF000F1E28491882341F09091C00095FFFCCF3E
:10BF00008093C6003196F5CF4AE050E060E070E0E3
:10BF100085EE9FE00E944AA3E8EEF1E28491882337
:10BF200041F09091C00095FFFCCF8093C600319600
:10BF3000F5CF4091500A5091510A6091520A709188
:10BF4000530A21E030E085EE9FE00E9420A4E5EE58
:10BF5000F1E28491882341F09091C00095FFFCCFDD
:10BF60008093C6003196F5CF6091580A7091590AB6
:10BF7000882777FD8095982F0E9417C9AB01BC01D7
:10BF800021E030E085EE9FE00E9420A4E1EEF1E2A6
:10BF90008491882341F09091C00095FFFCCF80935D
:10BFA000C6003196F5CF8091720A90E00E94652715
:10BFB0004AE050E0BC0185EE9FE00E944AA3ECED10
:10BFC000F1E28491882341F09091C00095FFFCCF6D
:10BFD0008093C6003196F5CF8FEF9FEF0E946527C3
:10BFE0004AE050E0BC0185EE9FE00E944AA38091A8
:10BFF000C00085FFFCCF8AE08093C6000C94757169
:10C000008DE690E00E94365681110C94B66FE09157
:10C010007A0CF0E0EE0FFF1FE45EFD4F0190F0811F
:10C02000E02DE65AFE4F808191810E94E98383E5ED
:10C030000E94EB4B882391F00091720A0E94D74B2B
:10C0400010E0000F111F085A154F0E94E4C8F801B4
:10C050007183608381E080939C0515C082E50E9416
:10C06000EB4B882381F00091720A0E94D74B10E0BD
:10C07000000F111F085A154F0E94E4C8F801718380
:10C08000608310929C050E946D2A0E9406C34B019A
:10C090005C010091720A10E0F801EE0FFF1FE85AF0
:10C0A000F54F60817181882777FD8095982F0E94D8
:10C0B00017C9F801EE0FFF1FEE0FFF1FE05BF54FF2
:10C0C00011E020813181428153810E9478CA181683
:10C0D0000CF010E01093700A1092440CCC24CA9417
:10C0E000DC2C7601F8EE4F2EF3E05F2E612C712CE4
:10C0F000AAE03A2E8091440C81110C941270FFEF4B
:10C10000CF16DF06EF06FF0611F40C943F70F7FE22
:10C1100002C00C9412700E9406C36C197D09683B22
:10C120007B4010F40C943F700C941270E0917A0CE8
:10C13000F0E0EE0FFF1FE45EFD4F0190F081E02D77
:10C14000E25AFE4F808191810E94E98383E50E943B
:10C15000EB4B882361F00E94D74B0E94E4C8709398
:10C16000570A6093560A81E080939C050FC082E5D0
:10C170000E94EB4B882351F00E94D74B0E94E4C8E9
:10C180007093570A6093560A10929C050E9406C34A
:10C190004B015C011092440C6091560A7091570A51
:10C1A000882777FD8095982F0E9417C911E020916C
:10C1B0004A0A30914B0A40914C0A50914D0A0E9414
:10C1C00078CA18160CF010E01093700A0EEC11E209
:10C1D0008AECE82E81E2F82E96ECC92E91E2D92E57
:10C1E0002AE0722E8091700A6091560A7091570A67
:10C1F000882309F48BC08091440C811187C0882763
:10C2000077FD8095982F0E9417C920914A0A309196
:10C210004B0A40914C0A50914D0A0E9478CA181658
:10C220000CF08BC00E9406C3681979098A099B0922
:10C23000693E73408105910508F460C0E091550C9A
:10C2400084E0E89FF0011124E05BF54F40815181CB
:10C2500062817381F8018491EEECF1E2882349F068
:10C260009091C00095FFFCCF8093C60031968491D9
:10C27000F5CF22E030E085EE9FE00E9420A4F70198
:10C280008491EAECF1E2882349F09091C00095FF97
:10C29000FCCF8093C60031968491F5CF6091550C08
:10C2A00070E04AE050E085EE9FE00E944AA3F6016C
:10C2B0008491E6ECF1E2882349F09091C00095FF6B
:10C2C000FCCF8093C60031968491F5CF40914A0A05
:10C2D00050914B0A60914C0A70914D0A21E030E078
:10C2E00085EE9FE00E9420A48091C00085FFFCCFD6
:10C2F0007092C6000E9406C34B015C010E949B27FE
:10C3000080E00E9469550E9485846CCF882777FD64
:10C310008095982F0E9417C920914A0A30914B0AA4
:10C3200040914C0A50914D0A0E9475C887FF05C084
:10C3300080919C05882309F475CFE0917A0CF0E098
:10C34000EE0FFF1FE45EFD4F0190F081E02DE05AFB
:10C35000FE4F808191810E94E98380918B0C88231C
:10C3600021F08CE097E00E94B9830E9406C360939D
:10C370007F0A7093800A8093810A9093820A0C94BA
:10C38000B66F83E50E94EB4B882319F10E94D74BCF
:10C3900020E030E0A9010E9475C887FD0FC00E940F
:10C3A000D74B20E030E04FE753E40E9478CA1816DC
:10C3B00044F00E94D74B0E94E4C805C060E070E0E2
:10C3C00002C06FEF70E07093540C6093530C0C94A8
:10C3D000B66F8FEF90E09093540C8093530C0C94B5
:10C3E000B66F1092540C1092530C0C94B66F9B9A2B
:10C3F000A39881E08093A605E0917A0CF0E0EE0F1F
:10C40000FF1FE45EFD4F0190F081E02D808191815E
:10C410000E94E9830E9485840C94B66F0E946E2A64
:10C420000E949EAC149A0E9408AD1092540C109277
:10C43000530C68EE73E080E090E00E9435C39B9A55
:10C44000A39A1092A605E0917A0CF0E0EE0FFF1F80
:10C45000E45EFD4F0190F081E02DE459FF4F4081F3
:10C46000518124EC31E262EC71E283E597E00E94B5
:10C47000A5330E94E9830E9485840C94B66F1092C4
:10C48000820C0C94B66F81E08093820C0C94B66F92
:10C4900083E50E94EB4B8823A1F00E94D74B20E05C
:10C4A00030E04AE754E40E944ACB0E94E9C8609316
:10C4B0009D0570939E0580939F059093A0050C9415
:10C4C000B66F88E50E94EB4B81110C94537189E59E
:10C4D0000E94EB4B81110C9453718AE50E94EB4B47
:10C4E00081110C94537185E40E94EB4B81110C94E3
:10C4F00053710E949EAC149A0E9408AD0C94B66FC2
:10C5000083E50E94EB4B882311F40C94B66F0E94D4
:10C51000D74B20E030E04AE754E40E944ACB0E9427
:10C52000E9C860937B0A70937C0A80937D0A90939C
:10C530007E0A0C94B66F26EA37E039AF28AF0BEECF
:10C5400015E1EBEF8E2EE5E19E2EFFEAAF2EF5E131
:10C55000BF2E312CE8ADF9AD8191F9AFE8AF0E9463
:10C56000EB4B882309F45BC0F3E03F1251C00E94FB
:10C57000D74B6B017C0120E030E040EA51E40E949F
:10C5800075C887FF3FC0A7019601F80160817181DE
:10C59000828193810E947CC82B013C019B01AC01EC
:10C5A0006091C3157091C4158091C5159091C61501
:10C5B0000E944ACB6093C3157093C4158093C51530
:10C5C0009093C615A3019201F4016081718182816B
:10C5D00093810E944ACBF4016083718382839383A9
:10C5E000F50160817181828193810E9415C9A30147
:10C5F00092010E944ACB0E94E9C8F50160837183D1
:10C6000082839383F801C082D182E282F38207C0E1
:10C610000E94D74BF80160837183828393833394A4
:10C620000C5F1F4FF4E08F0E911C24E0A20EB11C92
:10C6300034E033128FCF0C94B66F9091C00095FF09
:10C64000FCCF8093C600319684918111F6CF0C9473
:10C65000B66F0091830A1091840A0B5F1F4F6AE244
:10C6600070E0C8010E9401D0009711F0FC01108217
:10C67000C8010E94B9830C94B66FEFEBF1E284918C
:10C68000882341F09091C00095FFFCCF8093C600B5
:10C690003196F5CF4091690C50916A0C60916B0C0A
:10C6A00070916C0C22E030E085EE9FE00E9420A4A7
:10C6B000EBEBF1E28491882341F09091C00095FF6B
:10C6C000FCCF8093C6003196F5CF40916D0C509110
:10C6D0006E0C60916F0C7091700C22E030E085EE72
:10C6E0009FE00E9420A4E7EBF1E28491882341F0CF
:10C6F0009091C00095FFFCCF8093C6003196F5CF96
:10C700004091710C5091720C6091730C7091740C8B
:10C7100022E030E085EE9FE00E9420A4E3EBF1E20E
:10C720008491882341F09091C00095FFFCCF8093C5
:10C73000C6003196F5CF4091750C5091760C609102
:10C74000770C7091780C22E030E085EE9FE00E943B
:10C7500020A4E0917A0CF0E0EE0FFF1FE45EFD4FA5
:10C760000190F081E02DEC59FE4F0190F081E02D19
:10C770008491882341F09091C00095FFFCCF809375
:10C78000C6003196F5CF0E94FAAC0E9417C92091DD
:10C79000EB153091EC154091ED155091EE150E947E
:10C7A0007CC8AB01BC0122E030E085EE9FE00E9436
:10C7B00020A4EFEAF1E28491882341F09091C00037
:10C7C00095FFFCCF8093C6003196F5CF81E00E94A3
:10C7D000FAAC0E9417C92091EF153091F0154091E5
:10C7E000F1155091F2150E947CC8AB01BC0122E00A
:10C7F00030E085EE9FE00E9420A4EBEAF1E2849114
:10C80000882341F09091C00095FFFCCF8093C60033
:10C810003196F5CF82E00E94FAAC0E9417C92091B0
:10C82000F3153091F4154091F5155091F6150E94CD
:10C830007CC8AB01BC0122E030E085EE9FE00E94A5
:10C8400020A48091C00085FFFCCF8AE08093C600C1
:10C850000C94B66F80E00E941EA50C94B66F81E028
:10C860000E941EA50C94B66F9091C00095FFFCCF5E
:10C870008093C60081918111F7CF8091C00085FF20
:10C88000FCCF8AE08093C600E0917A0CF0E0EE0FD6
:10C89000FF1FE45EFD4F0190F081E02DEE58FE4F4A
:10C8A0000190F081E02D8491882341F09091C000A7
:10C8B00095FFFCCF8093C6003196F5CFE0917A0CBE
:10C8C000F0E0EE0FFF1FE45EFD4F1E9B06C00190DF
:10C8D000F081E02DE058FE4F05C00190F081E02D81
:10C8E000EE57FE4F90818181E92FF82F81918823A7
:10C8F00039F09091C00095FFFCCF8093C600F6CF31
:10C900008091C00085FFFCCF8AE08093C600E09153
:10C910007A0CF0E0EE0FFF1FE45EFD4F0190F08116
:10C92000E02DEC58FE4F0190F081E02D849188239A
:10C9300041F09091C00095FFFCCF8093C6003196E6
:10C94000F5CFE0917A0CF0E0EE0FFF1FE45EFD4FB3
:10C95000029906C00190F081E02DE058FE4F05C01D
:10C960000190F081E02DEE57FE4F90818181E92FFB
:10C97000F82F8191882339F09091C00095FFFCCF6A
:10C980008093C600F6CF8091C00085FFFCCF8AE07F
:10C990008093C600E0917A0CF0E0EE0FFF1FE45E9A
:10C9A000FD4F0190F081E02DEA58FE4F0190F0819B
:10C9B000E02D8491882341F09091C00095FFFCCF39
:10C9C0008093C6003196F5CFE0917A0CF0E0EE0F3F
:10C9D000FF1FE45EFD4F1D9B06C00190F081E02D1E
:10C9E000E058FE4F05C00190F081E02DEE57FE4F5C
:10C9F00090818181E92FF82F8191882339F09091DE
:10CA0000C00095FFFCCF8093C600F6CF8091C00098
:10CA100085FFFCCF8AE08093C600E0917A0CF0E0BD
:10CA2000EE0FFF1FE45EFD4F0190F081E02DE8580E
:10CA3000FE4F0190F081E02D8491882341F0909188
:10CA4000C00095FFFCCF8093C6003196F5CFE091F2
:10CA50007A0CF0E0EE0FFF1FE45EFD4F019906C077
:10CA60000190F081E02DE058FE4F05C00190F0816B
:10CA7000E02DEE57FE4F90818181E92FF82F8191B3
:10CA8000882339F09091C00095FFFCCF8093C600B9
:10CA9000F6CF8091C00085FFFCCF8AE08093C6006E
:10CAA000E0917A0CF0E0EE0FFF1FE45EFD4F019085
:10CAB000F081E02DE658FE4F0190F081E02D849149
:10CAC000882341F09091C00095FFFCCF8093C60071
:10CAD0003196F5CFE0917A0CF0E0EE0FFF1FE45EA7
:10CAE000FD4F1C9B06C00190F081E02DE058FE4FE9
:10CAF00005C00190F081E02DEE57FE4F90818181BD
:10CB0000E92FF82F8191882339F09091C00095FF8B
:10CB1000FCCF8093C600F6CF8091C00085FFFCCF8C
:10CB20008AE08093C600E0917A0CF0E0EE0FFF1FE0
:10CB3000E45EFD4F0190F081E02DE458FE4F01903E
:10CB4000F081E02D8491882341F09091C00095FF01
:10CB5000FCCF8093C6003196F5CFE0917A0CF0E0DF
:10CB6000EE0FFF1FE45EFD4F379906C00190F08184
:10CB7000E02DE058FE4F05C00190F081E02DEE570A
:10CB8000FE4F90818181E92FF82F8191882339F020
:10CB90009091C00095FFFCCF8093C600F6CF8091A6
:10CBA000C00085FFFCCF8AE08093C6000C94B66F6E
:10CBB0008091550C8093720A84E50E94EB4B882388
:10CBC00081F10E94D74B0E94E9C86093720A6623E4
:10CBD00041F1E5EBF2E28491882341F09091C000AD
:10CBE00095FFFCCF8093C6003196F5CFE0917A0C8B
:10CBF000F0E0EE0FFF1FE45EFD4F0190F081E02DAD
:10CC0000E05BFE4F0190F081E02D8191882311F4CB
:10CC10000C94B66F9091C00095FFFCCF8093C60036
:10CC2000F4CF84E40E94EB4B882311F40C94B66F8C
:10CC30000E94D74B20E030E0A9010E9475C8811105
:10CC400003C01092790C32C00091720A10E00E9469
:10CC5000D74BF801EE0FFF1FEE0FFF1FED52FA4FFB
:10CC60006083718382839383E090D305F090D40531
:10CC70000091D5051091D60520E030E0A901B7015B
:10CC8000C8010E9475C8811104C0E12CF12C00E498
:10CC900010E4C701D8018093D3059093D405A093E5
:10CCA000D505B093D60581E08093790C0E94345766
:10CCB0000C94B66F06EA17E02BEDE22E25E1F22E7A
:10CCC000F80181918F010E94EB4B882349F00E946B
:10CCD000D74B0E94E9C8F7016083718382839383F5
:10CCE000F4E0EF0EF11C27E00A3A120749F70E9420
:10CCF000E5BE0C94B66F06EA17E09BEFE92E95E1CE
:10CD0000F92EF80181918F010E94EB4B882339F0B5
:10CD10000E94D74BF7016083718382839383F4E091
:10CD2000EF0EF11C27E00A3A120759F70C94B66F80
:10CD300083E50E94EB4B882351F00E94D74B609310
:10CD4000D3157093D4158093D5159093D61584E59B
:10CD50000E94EB4B882311F40C94B66F0E94D74BC2
:10CD60006093CF157093D0158093D1159093D21501
:10CD70000C94B66F83E50E94EB4B882351F00E9420
:10CD8000D74B6093D7157093D8158093D91590938E
:10CD9000DA1584E50E94EB4B882351F00E94D74BB3
:10CDA0006093BF157093C0158093C1159093C21501
:10CDB00082E40E94EB4B882361F00E94D74B0E94D3
:10CDC000E9C860930B1670930C1680930D16909320
:10CDD0000E1688E50E94EB4B882351F00E94D74B3A
:10CDE0006093CB157093CC158093CD159093CE1591
:10CDF0008AE50E94EB4B882351F00E94D74B609349
:10CE0000C7157093C8158093C9159093CA1585E40A
:10CE10000E94EB4B882311F40C94B66F0E94D74B01
:10CE20006093C3157093C4158093C5159093C61570
:10CE30000C94B66F06EA17E08DE5E82E8CE0F82E2C
:10CE4000F80181918F010E94EB4B882339F00E94F9
:10CE5000D74BF7016083718382839383F4E0EF0EF5
:10CE6000F11C27E0093A120711F40C94B66FE8CFD1
:10CE700083E50E94EB4B882351F00E94D74B6093CF
:10CE8000B3057093B4058093B5059093B60586E419
:10CE90000E94EB4B882381F00E94D74B20E030E0CA
:10CEA00040E752E40E947CC86093AB057093AC05E8
:10CEB0008093AD059093AE058AE50E94EB4B8823E5
:10CEC00011F40C94B66F0E94D74B60934D0C709385
:10CED0004E0C80934F0C9093500C0C94B66F83E5DE
:10CEE0000E94EB4B882351F00E94D74B6093490C72
:10CEF00070934A0C80934B0C90934C0C86E40E94E8
:10CF0000EB4B882311F40C94B66F0E94D74B20E0B2
:10CF100030E040E752E40E947CC86093A70570931C
:10CF2000A8058093A9059093AA050C94B66F83E594
:10CF30000E94EB4B882311F40C94B66F0E94D74BE0
:10CF40000E94E4C86115710551F06130710569F402
:10CF500081E08093520C1092510C0C94B66F109299
:10CF6000520C1092510C0C94B66FE5EBF2E28491E6
:10CF7000882341F09091C00095FFFCCF8093C600BC
:10CF80003196F5CFE0917A0CF0E0EE0FFF1FE45EF2
:10CF9000FD4F0190F081E02DE459FE4F0190F081AA
:10CFA000E02D8491882341F09091C00095FFFCCF43
:10CFB0008093C6003196F5CF80918D0A90918E0AAC
:10CFC00020E6289FF001299FF00D1124ED56F54F22
:10CFD0008191882339F09091C00095FFFCCF809318
:10CFE000C600F6CFE9EAF1E28491882341F09091FE
:10CFF000C00095FFFCCF8093C6003196F5CF80919D
:10D00000C00085FFFCCF8AE08093C600AFC783E5F0
:10D010000E94EB4B882309F4A9C70E94D74B0E94BA
:10D02000E4C87093DE056093DD05A0C783E50E9428
:10D03000EB4B882309F49AC70E94D74B0E94E4C89F
:10D040006B017C0184E50E94EB4B882381F08DED20
:10D0500090E00E943656811189C7E091720AF0E093
:10D06000EE0FFF1FE752FA4FD182C0827FC7D092E6
:10D07000DC05C092DB057AC780E50E94EB4B882374
:10D0800009F474C70E94D74B0E94E4C8D62E062F1D
:10D09000172F83E50E94EB4B882331F00E94D74B7A
:10D0A0000E94E4C87B0103C0EE24EA94FE2CC70171
:10D0B0000196039708F05AC7EEE6F7E08191919147
:10D0C0008017910709F452C737E0E63AF307B1F742
:10D0D00017FD4CC70E949EACCD2C60E08D2D0E94A8
:10D0E00026C28FEFE816F80631F0EA94EF2871F0C7
:10D0F00000E010E00DC08D2D0E9494C231E020E0D0
:10D10000892B09F030E0032F122F02C001E010E05C
:10D110008C2D0E9494C28017910709F427C70E94A2
:10D120009B2780E00E9469550E948584F1CF83E5AA
:10D130000E94EB4B882331F00E94D74B0E94E4C839
:10D140008B0102C00EE610E080E50E94EB4B8823C5
:10D1500031F00E94D74B0E94E4C8CB0102C088EE98
:10D1600093E06C01EE24D7FCE094FE2C101611061F
:10D170007CF420E030E0A901B8018EE40E94D2C323
:10D18000C701B6010E9435C38EE40E94E3C6EEC615
:10D19000C701B6010E9435C3E9C680E50E94EB4B8A
:10D1A000882351F00E94D74B6093180270931902A4
:10D1B00080931A0290931B0289E40E94EB4B882310
:10D1C00061F00E94D74B0E94E0306093140270938C
:10D1D0001502809316029093170284E40E94EB4B91
:10D1E000882361F00E94D74B0E94EC3060931002BC
:10D1F00070931102809312029093130283E40E94B1
:10D20000EB4B882351F00E94D74B60930C02709334
:10D210000D0280930E0290930F020E944E27E09120
:10D220007A0CF0E0EE0FFF1FE45EFD4F0190F081FD
:10D23000E02DE65CFE4F0190F081E02D8191882386
:10D2400039F09091C00095FFFCCF8093C600F6CFD7
:10D25000ECE5F7E08191882339F09091C00095FFCB
:10D26000FCCF8093C600F6CF40911802509119026E
:10D2700060911A0270911B0222E030E085EE9FE07F
:10D280000E9420A4E0E6F7E08191882339F0909194
:10D29000C00095FFFCCF8093C600F6CF60911402CA
:10D2A0007091150280911602909117020E94E6304B
:10D2B000AB01BC0122E030E085EE9FE00E9420A49B
:10D2C000E4E6F7E08191882339F09091C00095FF62
:10D2D000FCCF8093C600F6CF6091100270911102CE
:10D2E00080911202909113020E94F230AB01BC01B6
:10D2F00022E030E085EE9FE00E9420A4E8E6F7E01F
:10D300008191882339F09091C00095FFFCCF8093E4
:10D31000C600F6CF40910C0250910D0260910E02B2
:10D3200070910F0222E030E085EE9FE00E9420A481
:10D330008091C00085FFFCCF8AE08093C60016C6AE
:10D3400083E50E94EB4B882319F00E94D74B03C062
:10D3500060E070E0CB010E94DCBE08C685E40E945C
:10D36000EB4B882341F00E94D74B0E94E4C88B010D
:10D3700077FF03C009C000E010E0C12CD12CF6E11A
:10D38000EF2EF3E4FF2E06C0C12CD12CECE8EE2EDC
:10D39000E2E4FE2E83E50E94EB4B882321F00E94FD
:10D3A000D74B6B017C0183E40E94EB4B882331F067
:10D3B0000E94D74B0E94E4C89B0102C025E030E0E8
:10D3C000A801C701B6010E94812AD0C50E949EAC67
:10D3D000CDC50E9451A00E94239CC8C50E9451A0A7
:10D3E000C5C50E94239CC2C59091C00095FFFCCF8B
:10D3F0008093C600319684918111F6CFE9E9F1E27C
:10D400008491882309F4B2C59091C00095FFFCCFA8
:10D410008093C6003196F4CF8AE50E94EB4B8823B7
:10D4200009F4D6C00E94D74B6B017C0120E030E0AC
:10D4300040E751EC0E9478CA87FD57C020E030E0F9
:10D4400040EA50ECC701B6010E9475C818160CF4EA
:10D450004CC0F7FAF094F7F8F094C092560CD092C2
:10D46000570CE092580CF092590CE5EBF2E28491E3
:10D47000882341F09091C00095FFFCCF8093C600B7
:10D480003196F5CFE0917A0CF0E0EE0FFF1FE45EED
:10D49000FD4F80819181FC01E65CFE4F408151810E
:10D4A000E255F10928E931E263EC77E0808191816E
:10D4B0000E94A533FC012491222341F03091C00049
:10D4C00035FFFCCF2093C6000196F4CF8091C000B9
:10D4D00085FFFCCF8AE08093C6008091C00085FF65
:10D4E000FCCF8AE08093C60041C5E5EBF2E284916F
:10D4F000882341F09091C00095FFFCCF8093C60037
:10D500003196F5CFE0917A0CF0E0EE0FFF1FE45E6C
:10D51000FD4F0190F081E02DE851FF4F0190F08127
:10D52000E02D8491882341F09091C00095FFFCCFBD
:10D530008093C6003196F5CFE0917A0CF0E0EE0FC3
:10D54000FF1FE45EFD4F0190F081E02DE658FE4F95
:10D550000190F081E02D8491882341F09091C000EA
:10D5600095FFFCCF8093C6003196F5CF4AE050E09E
:10D5700061EF7FEF85EE9FE00E944AA3E0917A0C75
:10D58000F0E0EE0FFF1FE45EFD4F0190F081E02D13
:10D59000E458FE4F0190F081E02D8491882341F002
:10D5A0009091C00095FFFCCF8093C6003196F5CFD7
:10D5B0004AE050E06BEF7FEF85EE9FE00E944AA3C8
:10D5C0008091C00085FFFCCF8AE08093C600CEC466
:10D5D000E5EBF2E28491882341F09091C00095FF41
:10D5E000FCCF8093C6003196F5CFE0917A0CF0E045
:10D5F000EE0FFF1FE45EFD4F0190F081E02DE8513A
:10D60000FF4F64E971E2808191810E948433FC01C3
:10D610002491222341F03091C00035FFFCCF2093AC
:10D62000C6000196F4CF8091C00085FFFCCF8AE050
:10D630008093C6004091560C5091570C6091580C45
:10D640007091590C705822E030E085EE9FE00E9406
:10D6500020A48091C00085FFFCCF8AE08093C600A3
:10D6600085C48091DD059091DE059093D805809367
:10D67000D705C090690CD0906A0CE0906B0CF090CC
:10D680006C0CCF8ED8A2E9A2FAA200916D0C109179
:10D690006E0C20916F0C3091700C0BA31CA32DA36A
:10D6A0003EA34091710C5091720C6091730C70917B
:10D6B000740C4FA358A769A77AA78091750C909115
:10D6C000760CA091770CB091780C8BA79CA7ADA796
:10D6D000BEA7C982DA82EB82FC820D831E832F8370
:10D6E000388749875A876B877C878D879E87AF8766
:10D6F000B88B85E40E94EB4B882359F00E94D74BEE
:10D700009B01AC016BA57CA58DA59EA50E949CC725
:10D710000AC020E030E040E050E46BA57CA58DA578
:10D720009EA50E949BC76BA77CA78DA79EA795E58A
:10D73000C92E9CE0D92EE12CF12C08EC13E49E01BB
:10D74000255D3F4FAE01495D5F4FBE016D5D7F4F6F
:10D75000CE014F960E9431B48AE50E94EB4B88239C
:10D7600049F00E94D74B9B01AC016FA178A589A518
:10D770009AA51EC020E030E040E050E46FA178A5FB
:10D7800089A59AA50E949CC76B017C016FA378A70D
:10D7900089A79AA720E030E040E251E40E9475C8D2
:10D7A00087FF0CC020E030E040E251E4C701B60141
:10D7B0000E949CC76FA378A789A79AA7B5E5CB2E2F
:10D7C000BCE0DB2EE12CF12C06E913E49E01255D83
:10D7D0003F4FAE01495D5F4FBE016D5D7F4FCE0192
:10D7E0004F960E9431B488E50E94EB4B882379F074
:10D7F0000E94D74B9B01AC016F8D78A189A19AA1A2
:10D800000E949CC76F8F78A389A39AA308C080E069
:10D8100090E0A3E5B3E48F8F98A3A9A3BAA389E509
:10D820000E94EB4B882339F00E94D74B6BA37CA35B
:10D830008DA39EA304C01BA21CA21DA21EA2F5E5DF
:10D84000CF2EFCE0DF2EE12CF12C0CE812E49E013F
:10D85000255D3F4FAE01495D5F4FBE016D5D7F4F5E
:10D86000CE014F960E9431B48CE40E94EB4B88238A
:10D8700059F00E94D74B9B01AC016BA57CA58DA5EF
:10D880009EA50E949CC70AC020E030E040EA52E416
:10D890006BA57CA58DA59EA50E949BC76BA77CA7A9
:10D8A0008DA79EA775E5C72E7CE0D72EE12CF12C25
:10D8B00008EC13E49E01255D3F4FAE01495D5F4FCB
:10D8C000BE016D5D7F4FCE014F960E9431B40E9424
:10D8D0009EAC149A64E670E080E090E00E9435C34C
:10D8E0000E94119000E010E0F12C0E946D858111E2
:10D8F0001BC0F3940E949B2781E00E946955F110A0
:10D90000F4CF043FF1E01F0711F400E010E06A9A41
:10D910000115110511F4729A04C00431110509F4BE
:10D9200072980F5F1F4FE1CF729820E030E04CE813
:10D9300052E46BA57CA58DA59EA50E949CC76BA7F4
:10D940007CA78DA79EA745E5C42E4CE0D42EE12CE4
:10D95000F12C00EA11E49E01255D3F4FAE01495DC7
:10D960005F4FBE016D5D7F4FCE014F960E9431B477
:10D9700020E030E048E452E46BA57CA58DA59EA58F
:10D980000E949CC76BA77CA78DA79EA7E12CF12CBA
:10D9900000E010E49E01255D3F4FAE01495D5F4F01
:10D9A000BE016D5D7F4FCE014F960E9431B4109243
:10D9B0007C0C10927B0C0E94A79080917B0C909124
:10D9C0007C0C019709F47CC010927C0C10927B0CAB
:10D9D0000E94FA9080917B0C90917C0C8230910592
:10D9E00049F1039709F069C020E030E048E452E4CF
:10D9F0006BA57CA58DA59EA50E949CC76BA77CA747
:10DA00008DA79EA7B5E5CB2EBCE0DB2EE12CF12C3B
:10DA100000E010E49E01255D3F4FAE01495D5F4F80
:10DA2000BE016D5D7F4FCE014F960E9431B40E94C2
:10DA30005490C3CF20E030E04CE852E46BA57CA5C5
:10DA40008DA59EA50E949CC76BA77CA78DA79EA7AE
:10DA500095E5C92E9CE0D92EE12CF12C00EA11E4C9
:10DA60009E01255D3F4FAE01495D5F4FBE016D5D7B
:10DA70007F4FCE014F960E9431B420E030E048E461
:10DA800052E46BA57CA58DA59EA50E949CC76BA7A3
:10DA90007CA78DA79EA7E12CF12C00E010E49E014D
:10DAA000255D3F4FAE01495D5F4FBE016D5D7F4F0C
:10DAB000CE014F960E9431B47ECF0E943D907DCF23
:10DAC00020E030E040EA50E46BA57CA58DA59EA542
:10DAD0000E949CC76BA77CA78DA79EA755E5C52E66
:10DAE0005CE0D52EE12CF12C00E010E49E01255DD8
:10DAF0003F4FAE01495D5F4FBE016D5D7F4FCE016F
:10DB00004F960E9431B4A80197016BA57CA58DA505
:10DB10009EA50E949BC76BA77CA78DA79EA7E12C03
:10DB2000F12C08EC13E49E01255D3F4FAE01495DE9
:10DB30005F4FBE016D5D7F4FCE014F960E9431B4A5
:10DB4000E12CF12C0CE812E49E01255D3F4FAE0163
:10DB5000495D5F4FBE016B5F7F4FCE0101960E9412
:10DB600031B4E12CF12C06E913E49E01255D3F4F11
:10DB7000AE01475F5F4FBE016B5F7F4FCE010196E5
:10DB80000E9431B420E030E040E050E46BA57CA579
:10DB90008DA59EA50E949CC76BA77CA78DA79EA75D
:10DBA000E12CF12C08EC13E49E01255D3F4FAE0102
:10DBB000475F5F4FBE016B5F7F4FCE0101960E94B2
:10DBC00031B4CE010D960E94B8BE8091D7059091D8
:10DBD000D8058093DD059093DE059F938F938BE8A6
:10DBE00091E29F938F938E01015D1F4F1F930F93BF
:10DBF0000E9439D0C8010E94CB480F900F900F901F
:10DC00000F900F900F90B2C188E50E94EB4B8823D4
:10DC100039F00E94D74B0E94E4C880E00E94C8AD52
:10DC20008AE50E94EB4B882339F00E94D74B0E9473
:10DC3000E4C881E00E94C8AD85E40E94EB4B8823D4
:10DC400009F494C10E94D74B0E94E4C882E00E946C
:10DC5000C8AD8CC183E50E94EB4B811104C006EA7C
:10DC600017E0F12C10C010E00E94D74B0E94E9C8C9
:10DC7000812F0E949EAE1F5F1530B1F7F0CFF39455
:10DC8000F4E0FF1679F0F80181918F010E94EB4BCF
:10DC90008823A9F30E94D74B0E94E9C88F2D0E94C8
:10DCA0009EAEEDCF82E40E94EB4B882339F00E94B8
:10DCB000D74B0E94E9C884E00E949EAE0E9464AFE8
:10DCC00055C183E50E94EB4B882309F453C00E94A1
:10DCD000D74B0E94E4C86130710541F06230710594
:10DCE00009F048C006EA17E0F12C25C006EA17E063
:10DCF000F12CF80181918F010E94EB4B882341F0B8
:10DD00000E94D74B0E94E4C84FEF8F2D0E9460AE57
:10DD1000F394F4E0FF12EDCF82E40E94EB4B8823F2
:10DD200049F10E94D74B0E94E4C84FEF20C0F39402
:10DD3000F4E0FF1689F0F80181918F010E94EB4B0E
:10DD40008823A9F30E94D74B0E94E4C8462F6FEFA7
:10DD50008F2D0E9460AEEBCF82E40E94EB4B8823B4
:10DD600049F00E94D74B0E94E4C8462F6FEF84E031
:10DD70000E9460AE0E9464AFF9C084E50E94EB4B44
:10DD8000882309F4A2C00E94D74B0E94E9C860937F
:10DD9000720A662309F442C0E5EBF2E2849188231B
:10DDA00041F09091C00095FFFCCF8093C600319662
:10DDB000F5CFECE6F7E08191882339F09091C0002F
:10DDC00095FFFCCF8093C600F6CF40E050E0609115
:10DDD000720A85EE9FE00E9481A3E0917A0CF0E048
:10DDE000EE0FFF1FE45EFD4F0190F081E02DE05942
:10DDF000FE4F0190F081E02D8191882339F09091C0
:10DE0000C00095FFFCCF8093C600F6CF8091C00084
:10DE100085FFFCCF8AE08093C600A8C086E40E94FC
:10DE2000EB4B8823D9F00E94D74B6B017C016093A8
:10DE3000240C7093250C8093260C9093270C20E0E3
:10DE400030E0A9010E9478CA181644F4C092A105D6
:10DE5000D092A205E092A305F092A405E5EBF2E2D0
:10DE60008491882341F09091C00095FFFCCF80936E
:10DE7000C6003196F5CFE0917A0CF0E0EE0FFF1F6F
:10DE8000E45EFD4F0190F081E02DE259FE4F0190DC
:10DE9000F081E02D8191882339F09091C00095FFA9
:10DEA000FCCF8093C600F6CF6091550C70E04AE03D
:10DEB00050E085EE9FE00E944AA38091C00085FF5C
:10DEC000FCCF8AE08093C60051C0E5EBF2E284917A
:10DED000882341F09091C00095FFFCCF8093C6004D
:10DEE0003196F5CFE0917A0CF0E0EE0FFF1FE45E83
:10DEF000FD4F0190F081E02DE459FE4F0190F0813B
:10DF0000E02D8491882341F09091C00095FFFCCFD3
:10DF10008093C6003196F5CF80918D0A90918E0A3C
:10DF200020E6289FF001299FF00D1124ED56F54FB2
:10DF30008191882339F09091C00095FFFCCF8093A8
:10DF4000C600F6CFE9E8F1E28491882341F0909190
:10DF5000C00095FFFCCF8093C6003196F5CF80912D
:10DF6000C00085FFFCCF8AE08093C6000E94124C5F
:10DF7000BCC1C090400CD090410CE090420CF0909D
:10DF8000430C2091750C3091760C4091770C509198
:10DF9000780CC701B6010E949BC72DEC3CEC4CEC01
:10DFA0005DE30E9478CA181614F00C94FF57C092D3
:10DFB000750CD092760CE092770CF092780C85E795
:10DFC0009CE00E94B8BE60E080E00E94844E8DC15B
:10DFD00080E090E00E9439470C94085981E090E07D
:10DFE0000E9439470C94135982E090E00E9439470F
:10DFF0000C945C590E94E04BAB01BC014093260F8E
:10E000005093270F6093280F7093290F81E79EE0AC
:10E010000E94D21BABCF0E94D74B0E94E4C88B0159
:10E020000C94985EE0917A0CF0E0EE0FFF1FE45E36
:10E03000FD4F0190F081E02DE45AFE4F80819181E7
:10E040000E94E98380918B0C882321F08CE097E07B
:10E050000E94B9830E9406C36093770A7093780A7E
:10E060008093790A90937A0A0E9406C360937F0A8C
:10E070007093800A8093810A9093820A77CF0E94DE
:10E0800006C3681979098A099B09693E73408105AD
:10E09000910508F479C0E9EDF1E28491882341F01B
:10E0A0009091C00095FFFCCF8093C6003196F5CFCC
:10E0B000E091720A24E0E29FF0011124E05BF54F49
:10E0C000408151816281738121E030E085EE9FE0E3
:10E0D0000E9420A4E5EDF1E28491882341F0909123
:10E0E000C00095FFFCCF8093C6003196F5CF6091BC
:10E0F000720A70E04AE050E085EE9FE00E944AA379
:10E10000E1EDF1E28491882341F09091C00095FF08
:10E11000FCCF8093C6003196F5CFF7FE03C0E1E552
:10E12000F7E025C00E9406C38B019C01C701B60120
:10E130006854744F8F4F9F4F601B710B820B930B72
:10E14000A30192010E9453CCBA01A9012AE030E058
:10E1500085EE9FE00E9476A38091C00085FFFCCFF2
:10E160000DC09091C00095FFFCCF8093C6008191B7
:10E170008111F7CF8091C00085FFFCCF3092C6009F
:10E180000E9406C34B015C010E949B2780E00E9415
:10E1900069550E948584FFEFCF16DF06EF06FF0664
:10E1A00009F046C08091700AE091720AF0E08F0198
:10E1B000000F111F000F111F005B154FEE0FFF1F07
:10E1C000E85AF54F608171818823C9F0882777FD6F
:10E1D0008095982F0E9417C920E030E040E85FE367
:10E1E0000E949BC79B01AC01F80160817181828113
:10E1F00093810E9478CA87FF50C00C947A60882768
:10E2000077FD8095982F0E9417C920E030E040E804
:10E210005FE30E949CC79B01AC01F80160817181A2
:10E22000828193810E9475C81816BCF50C947A609F
:10E23000F7FE02C00C947A60E091720AF0E08F0160
:10E24000000F111F000F111F005B154FEE0FFF1F76
:10E25000E85AF54F60817181882777FD8095982F66
:10E260000E9417C99B01AC01F80160817181828114
:10E2700093810E949BC70E94E4C897FF07C09095B6
:10E280008095709561957F4F8F4F9F4F66307105D8
:10E290008105910514F40C947A600E9406C36B0109
:10E2A0007C010C947A600E949EAC88E50E94EB4B46
:10E2B000882319F0179A10925A0C89E50E94EB4BAB
:10E2C000882319F0169A10925B0C8AE50E94EB4B9A
:10E2D000882319F0159A10925C0C85E40E94EB4B90
:10E2E000882309F443CE149A41CEE9960FB6F894E8
:10E2F000DEBF0FBECDBFDF91CF911F910F91FF9079
:10E30000EF90DF90CF90BF90AF909F908F907F90D5
:10E310006F905F904F903F900895CF93DF938091DF
:10E32000890A90918A0A039714F40E94445160E08C
:10E3300089E89CE00E94293E8091890A90918A0A8E
:10E34000892B09F47EC08091890C8823E1F08091AB
:10E350008D0A90918E0A20E6289FE001299FD00D1A
:10E360001124CD56D54F65E272E2CE010E94ACCFAA
:10E37000892B59F5BE0189E89CE00E94AB3D809154
:10E380008A0C882319F00E94465745C0E0917A0C08
:10E39000F0E0EE0FFF1FE45EFD4F0190F081E02DF5
:10E3A000E65CFE4F0190F081E02D8491882341F0DE
:10E3B0009091C00095FFFCCF8093C6003196F5CFB9
:10E3C0008091C00085FFFCCF23C060E089E89CE01D
:10E3D0000E941F3FE0917A0CF0E0EE0FFF1FE45E19
:10E3E000FD4F0190F081E02DE45CFE4F0190F08143
:10E3F000E02D8491882341F09091C00095FFFCCFDF
:10E400008093C6003196F5CF8091C00085FFFCCF88
:10E410008AE08093C6008091890A90918A0A0197C8
:10E4200090938A0A8093890A80918D0A90918E0A2E
:10E43000019664E070E00E9440CC90938E0A809335
:10E440008D0A0E949B2780E00E9469550E943FA48C
:10E45000DF91CF910C9485848F929F92AF92BF925F
:10E46000CF92DF92EF92FF920F931F93CF93DF93A0
:10E470008C018C519E4F0E947037680189E8C80E4C
:10E48000D11C21F1780181E4E81A8EEFF80AE70146
:10E4900057018FE1A81AB1086DED862E67E0962E20
:10E4A000CC15DD0599F0FE01EE19FF09EA0DFB1D03
:10E4B00091828082FE0178978081811102C06F97DE
:10E4C000EFCFCE014B970E94B51CF9CFC8018659FA
:10E4D0009F4F0E947037C801875B9F4FDF91CF919C
:10E4E0001F910F91FF90EF90DF90CF90BF90AF9072
:10E4F0009F908F900C94703789E89CE00C947C3747
:10E5000089E89CE0A9CFFB016091F0057091F105CD
:10E510007093590F6093580F6091620F7091630F61
:10E520007093570F6093560F62E06093EF0565EBB1
:10E530007DE87093F1056093F0059093550F8093FB
:10E54000540FF093530FE093520F662757FD6095D9
:10E55000762F40934E0F50934F0F6093500F709350
:10E56000510FC901AA2797FDA095BA2F841B950BBF
:10E57000A60BB70B80934A0F90934B0FA0934C0FB1
:10E58000B0934D0F80819181AA2797FDA095BA2F56
:10E59000841B950BA60BB70B8093620F9093630FB0
:10E5A000A093640FB093650F0895CF93DF93CDB719
:10E5B000DEB7C054D1090FB6F894DEBF0FBECDBF91
:10E5C00088E0E7E2F6E0DE01D99601900D928A95A7
:10E5D000E1F788E0EFE2F6E0DE01D19601900D92DE
:10E5E0008A95E1F788E0E7E3F6E0DE01999601908D
:10E5F0000D928A95E1F788E0EFE3F6E0DE0191966F
:10E6000001900D928A95E1F788E0E7E4F6E0DE01FB
:10E61000599601900D928A95E1F788E0EFE4F6E0D3
:10E62000DE01519601900D928A95E1F788E0E7E5C9
:10E63000F6E0DE01199601900D928A95E1F788E0E7
:10E64000EFE5F6E0DE01119601900D928A95E1F773
:10E65000AE01475C5F4F60E08DE69FE00E9445336E
:10E66000AE014F5C5F4F61E08DE69FE00E94453355
:10E67000AE01475D5F4F62E08DE69FE00E9445334B
:10E68000AE014F5D5F4F63E08DE69FE00E94453332
:10E69000AE01475E5F4F64E08DE69FE00E94453328
:10E6A000AE014F5E5F4F65E08DE69FE00E9445330F
:10E6B000AE01475F5F4F66E08DE69FE00E94453305
:10E6C000AE014F5F5F4F67E08DE69FE00E944533EC
:10E6D000C05CDF4F0FB6F894DEBF0FBECDBFDF9139
:10E6E000CF9108950F931F93CF93DF93EB01142FD6
:10E6F000022F482F60E08DE69FE00E94A731612F36
:10E700008DE69FE00E9494C711E1FE0164916623AB
:10E7100011F0111117C0112339F060E28DE69FE06E
:10E720000E9494C71150F7CF602F8DE69FE00E94A2
:10E7300094C760E28DE69FE0DF91CF911F910F912A
:10E740000C9494C78DE69FE00E9494C721961150C7
:10E75000DCCFEF92FF920F931F93CF93DF93EB01E8
:10E76000E42E8901F90101900020E9F7F22EFE1A4A
:10E7700092E1F90E482F60E08DE69FE00E94A731FC
:10E780006E2D8DE69FE00E9494C7FE016491662382
:10E7900011F0F11019C06AE38DE69FE00E9494C762
:10E7A000FF2039F060E28DE69FE00E9494C7FA9462
:10E7B000F7CFB8018DE69FE0DF91CF911F910F91C8
:10E7C000FF90EF900C9493C78DE69FE00E9494C752
:10E7D0002196FA94DACF80937A0C91E09093F20527
:10E7E000682F88EF9FE00E945DD28091410F8130B9
:10E7F00019F482E08093410F08951092DC0F89E8AC
:10E800009CE00E94324410926B0F089589E89CE0CE
:10E810000C94113B89E89CE00C94183BCF9382E068
:10E820008093EF050E9406C36C507E4F8F4F9F4F21
:10E830006093670F7093680F8093690F90936A0FCE
:10E840006A9ACAE0729A84E690E00E9459C372986C
:10E8500084E690E00E9459C3C150A1F7CF9108957A
:10E86000E091F005F091F105E817F90771F0909348
:10E87000F1058093F0054093620F5093630F60930E
:10E88000640F7093650F2111C9CF089521E040E016
:10E8900050E0BA01E5CF21E040E050E0BA01E0CF1E
:10E8A000CF92DF92EF92FF920F931F93CF93DF935C
:10E8B0008091620F9091630FA091640FB091650FEA
:10E8C00081309048A105B10540F01092620F10927E
:10E8D000630F1092640F1092650F8091620F9091F8
:10E8E000630FA091640FB091650FB695A7959795AA
:10E8F000879540916B0F50E060E070E084179507BA
:10E90000A607B70710F480936B0FD0916B0F10918F
:10E910006C0F12FB112710F9C0E0B1E1CB2ED12C06
:10E92000E12CF12C01E04091620F5091630F609156
:10E93000640F7091650FD11138C08091EF05882365
:10E94000C1F0E0917A0CF0E0EE0FFF1FE45EFD4FA6
:10E950000190F081E02D8681978123E042305105BE
:10E960006105710510F443E001C040E2BC018C2F49
:10E97000B9DE112309F49CC18091620F9091630F5D
:10E98000A091640FB091650F0297A105B10508F041
:10E990008FC144DF8AE392E9DF91CF911F910F91FC
:10E9A000FF90EF90DF90CF9071CFD13051F58091F3
:10E9B000EF05882389F0769567955795479523E06D
:10E9C000413051056105710511F443E001C040E299
:10E9D00061EC73E28C2F86DE112309F469C180910A
:10E9E000620F9091630FA091640FB091650FB6957F
:10E9F000A795979587950197A105B10509F058C18D
:10EA0000C8CFD230B9F58091EF058823F1F0E091BD
:10EA10007A0CF0E0EE0FFF1FE45EFD4F0190F081F5
:10EA2000E02DE854FE4F808191817695679557954A
:10EA3000479523E0423051056105710511F443E02B
:10EA400001C040E2BC018C2F4DDE112309F430C11E
:10EA50008091620F9091630FA091640FB091650F48
:10EA6000B695A795979587950297A105B10509F0E9
:10EA70001FC18FCFD330B9F58091EF058823F1F016
:10EA8000E0917A0CF0E0EE0FFF1FE45EFD4F019085
:10EA9000F081E02DE654FE4F808191817695679557
:10EAA0005795479523E0433051056105710511F4F1
:10EAB00043E001C040E2BC018C2F14DE112309F4B5
:10EAC000F7C08091620F9091630FA091640FB09195
:10EAD000650FB695A795979587950397A105B105FD
:10EAE00009F0E6C056CFD430B9F58091EF05882300
:10EAF000F1F0E0917A0CF0E0EE0FFF1FE45EFD4FC5
:10EB00000190F081E02DE454FE4F80819181769553
:10EB100067955795479523E0443051056105710588
:10EB200011F443E001C040E2BC018C2FDBDD112376
:10EB300009F4BEC08091620F9091630FA091640FA1
:10EB4000B091650FB695A795979587950497A10500
:10EB5000B10509F0ADC01DCFD53051F58091EF055D
:10EB6000882389F0769567955795479523E045303A
:10EB700051056105710511F443E001C040E264EB09
:10EB800073E28C2FAFDD112309F492C08091620FE4
:10EB90009091630FA091640FB091650FB695A79502
:10EBA000979587950597A105B10509F081C0F1CE2C
:10EBB000D63051F58091EF05882389F076956795D9
:10EBC0005795479523E0463051056105710511F4CD
:10EBD00043E001C040E26DEA73E28C2F83DD112334
:10EBE00009F466C08091620F9091630FA091640F49
:10EBF000B091650FB695A795979587950697A1054E
:10EC0000B10509F055C0C5CED73041F58091EF056B
:10EC1000882389F0769567955795479523E0473087
:10EC200051056105710511F443E001C040E263EA5A
:10EC300073E28C2F57DD1123D9F18091620F9091EF
:10EC4000630FA091640FB091650FB695A795979546
:10EC500087950797A105B10559F59BCED83041F5A9
:10EC60008091EF05882389F07695679557954795AC
:10EC700023E0483051056105710511F443E001C0FE
:10EC800040E26CE973E28C2F2DDD112389F0809135
:10EC9000620F9091630FA091640FB091650FB695CC
:10ECA000A795979587950897A105B10509F471CEA9
:10ECB0008091620F9091630FA091640FB091650FE6
:10ECC0004297A105B10540F0C092620FD092630F48
:10ECD000E092640FF092650F4091620F5091630FC4
:10ECE0006091640F7091650F76956795579547957C
:10ECF00080916B0F90E00396242F30E082179307EA
:10ED00004CF48DEF840F80936B0F0093EF05DCEFD5
:10ED1000D40FCFEFCF5FDF5FC43008F404CEDF91B4
:10ED2000CF911F910F91FF90EF90DF90CF900895BA
:10ED30007F928F929F92AF92BF92CF92DF92EF928B
:10ED4000FF920F931F93CF93DF938091620F909167
:10ED5000630FA091640FB091650F81309048A105B9
:10ED6000B10540F01092620F1092630F1092640F81
:10ED70001092650F8091620F9091630FA091640FC4
:10ED8000B091650FB695A7959795879540916B0FB4
:10ED900050E060E070E084179507A607B70710F40D
:10EDA00080936B0FE0906B0FD0906C0FD2FADD2444
:10EDB000D0F8F12CCC24C3948091410F81113BC039
:10EDC000EE2019F07724739437C08091EF058823E3
:10EDD00001F1E0917A0CF0E0EE0FFF1FE45EFD4FD1
:10EDE0000190F081E02DEA50FF4F608171818091A8
:10EDF000620F9091630FA091640FB091650F23E0B3
:10EE00000297A105B10510F443E001C040E28F2D47
:10EE100069DCDD20B9F28091620F9091630FA091BF
:10EE2000640FB091650F0297A105B10558F6F6DCA5
:10EE300087EE90E851C0712C8091410F823009F02B
:10EE40005AC07E1057C08091EF05882359F1E09198
:10EE50007A0CF0E0EE0FFF1FE45EFD4F0190F081B1
:10EE6000E02DE055FF4F0190F081E02D8091620F81
:10EE70009091630FA091640FB091650FB695A7951F
:10EE800097958795472D50E060E070E023E0841768
:10EE90009507A607B70711F443E001C040E2BF01A0
:10EEA0008F2D20DCDD2031F18091620F9091630F76
:10EEB000A091640FB091650FB695A795979587952A
:10EEC000472D50E060E070E084179507A607B7076C
:10EED00089F4A4DC86EE98E9DF91CF911F910F9120
:10EEE000FF90EF90DF90CF90BF90AF909F908F906A
:10EEF0007F90CCCC73940CE112E0C0E0D0E08E2C7B
:10EF0000912CA12CB12C7E104AC08091EF05882352
:10EF100019F1D801ED91FC91EC54FE4F60817181A3
:10EF20008091620F9091630FA091640FB091650F73
:10EF3000B695A79597958795272D30E040E050E04E
:10EF400082179307A407B50719F420E24EE302C025
:10EF500020E240E28F2DC6DBDD2009F18091620FB7
:10EF60009091630FA091640FB091650FB695A7952E
:10EF70009795879588159905AA05BB0581F44EDC00
:10EF80008C2FDF91CF911F910F91FF90EF90DF9029
:10EF9000CF90BF90AF909F908F907F901CCC739438
:10EFA00021960E5F1F4FC230D10509F0ACCF4091C2
:10EFB000620F5091630F6091640F7091650F7695A9
:10EFC000679557954795872D90E0A0E0B0E04817EA
:10EFD00059076A077B0788F0872D90E0880F991FF3
:10EFE0000197AA2797FDA095BA2F8093620F90935F
:10EFF000630FA093640FB093650F4091620F50911F
:10F00000630F6091640F7091650F769567955795C2
:10F01000479580916B0F90E00396242F30E0821784
:10F0200093075CF48DEF840F80936B0FC092EF0514
:10F03000DCEFED2EE40EFF24FA94F394E394B3E0B6
:10F04000BF1508F0B9CEDF91CF911F910F91FF90BE
:10F05000EF90DF90CF90BF90AF909F908F907F9078
:10F0600008950F931F93CF93DF938091620F909138
:10F07000630FA091640FB091650F81309048A10596
:10F08000B10540F01092620F1092630F1092640F5E
:10F090001092650F8091620F9091630FA091640FA1
:10F0A000B091650FB695A7959795879540916B0F91
:10F0B00050E060E070E084179507A607B70710F4EA
:10F0C00080936B0FD0916B0F10916C0F12FB112777
:10F0D00010F9C0E001E08091620F9091630FA09160
:10F0E000640FB091650FD11134C02091EF05222338
:10F0F000C1F0E0917A0CF0E0EE0FFF1FE45EFD4FEF
:10F100000190F081E02DEA50FF4F6081718123E092
:10F110000297A105B10510F443E001C040E28C2F35
:10F12000E1DA112309F482C08091620F9091630F9C
:10F13000A091640FB091650F0297A105B10508F089
:10F1400075C06CDB87EE90E8DF91CF911F910F9136
:10F150009DCBD130A9F52091EF052223D1F0E0918C
:10F160007A0CF0E0EE0FFF1FE45EFD4F0190F0819E
:10F17000E02D62AD73ADB695A795979587952EE76F
:10F180000197A105B10511F44EE301C040E28C2FB7
:10F19000A9DA112309F44AC08091620F9091630F9C
:10F1A000A091640FB091650FB695A7959795879537
:10F1B0000197A105B105D1F531DB81E09FE8BFC022
:10F1C000D230A1F52091EF052223D1F0E0917A0C05
:10F1D000F0E0EE0FFF1FE45EFD4F0190F081E02DA7
:10F1E00064AD75ADB695A795979587952EE702976F
:10F1F000A105B10511F44EE301C040E28C2F72DA93
:10F200001123A1F08091620F9091630FA091640F80
:10F21000B091650FB695A795979587950297A1052B
:10F22000B10521F4FBDA88E09FE889C020E030E0F6
:10F2300040E251E460913D0F70913E0F80913F0F8D
:10F240009091400F0E9475C887FF7EC08091620F29
:10F250009091630FA091640FB091650FD330B1F519
:10F260002091EF052223D1F0E0917A0CF0E0EE0F2F
:10F27000FF1FE45EFD4F0190F081E02D66AD77AD9C
:10F28000B695A795979587952EE70397A105B105A4
:10F2900011F44EE301C040E28C2F24DA111102C0B8
:10F2A00025E053C08091620F9091630FA091640F8D
:10F2B000B091650FB695A795979587950397A1058A
:10F2C000B10571F7ABDA8FE09FE839C0D43041F770
:10F2D0002091EF052223E1F0E0917A0CF0E0EE0FAF
:10F2E000FF1FE45EFD4F0190F081E02DE05CFF4FD9
:10F2F00060817181B695A795979587952EE70497BC
:10F30000A105B10511F44EE301C040E28C2FEAD90A
:10F31000112331F24091620F5091630F6091640F9D
:10F320007091650F769567955795479544305105CF
:10F330006105710509F0B4CF71DA8BE39DE8DF91C7
:10F34000CF911F910F91A7CA23E04091620F509176
:10F35000630F6091640F7091650F7695679557956F
:10F360004795822F90E0A0E0B0E0481759076A0760
:10F370007B0788F0822F90E0880F991F0197AA27BA
:10F3800097FDA095BA2F8093620F9093630FA0937F
:10F39000640FB093650F4091620F5091630F6091BD
:10F3A000640F7091650F7695679557954795809195
:10F3B0006B0F90E00396242F30E0821793074CF4F4
:10F3C0008DEF840F80936B0F0093EF05DCEFD40F6C
:10F3D000CFEFCF5FDF5FC43008F47DCEDF91CF91F8
:10F3E0001F910F91089580E090E0A0E8BFE3809323
:10F3F0003D0F90933E0FA0933F0FB093400F31CE3F
:10F4000020E044E064E18DE69FE00E94DA31CDD84F
:10F410008DE69FE00C949B31F3DF20E040E050E06C
:10F42000BA0186EE98E91CCA1092590A1092580A3D
:10F430001092570A1092560A1092540C1092530CC4
:10F44000EBCF8DE69FE00C949B318091D90F90918A
:10F45000DA0F9093590A8093580A8091D70F9091B0
:10F46000D80F9093570A8093560A1092540C10921A
:10F47000530CD2DF0C946D2A8091D30F9091D40F4E
:10F480009093590A8093580A8091D10F9091D20F8E
:10F490009093570A8093560A1092540C1092530C72
:10F4A000BBDF0C946D2A8091010690910206909327
:10F4B000590A8093580A8091FF0590910006909315
:10F4C000570A8093560A1092540C1092530CA4DFE2
:10F4D0000C946D2A8091FD059091FE059093590A38
:10F4E0008093580A8091FB059091FC059093570AF0
:10F4F0008093560A1092540C1092530C8DDF0C948A
:10F500006D2A8091F9059091FA059093590A80939C
:10F51000580A8091F7059091F8059093570A8093C7
:10F52000560A1092540C1092530C76DF0C946D2AEC
:10F530008091F5059091F6059093590A8093580AA9
:10F540008091F3059091F4059093570A8093560AA1
:10F550001092540C1092530C5FDF0C946D2A2F9272
:10F560003F924F925F926F927F928F929F92AF9253
:10F57000BF92CF92DF92EF92FF920F931F93CF93A0
:10F58000DF93CDB7DEB7A2970FB6F894DEBF0FBEFC
:10F59000CDBF8091EF05811104C080916C0F82FF77
:10F5A000B6C289E89CE00E9419434091620F5091D5
:10F5B000630F6091640F7091650F41305048610591
:10F5C000710540F01092620F1092630F1092640F59
:10F5D0001092650F4091620F5091630F6091640F1C
:10F5E0007091650F769567955795479500916B0FCC
:10F5F00010E020E030E0401751076207730710F475
:10F6000040936B0F40906B0F30906C0F32FA3324A5
:10F6100030F8512C9C012150310939A328A3411005
:10F6200035C08091EF058823F1F0E0917A0CF0E08D
:10F63000EE0FFF1FE45EFD4F0190F081E02D66812B
:10F6400077818091620F9091630FA091640FB091C8
:10F65000650F23E00297A105B10510F443E001C056
:10F6600040E2852D3FD8332089F08091620F909140
:10F67000630FA091640FB091650F0297A105B105CA
:10F6800028F4CCD88AE392E901D941C26DE87CE044
:10F6900087EF9CE00E94691980918D0C8F3229F0D0
:10F6A00031E0431669F022E001C021E0A8A0B9A032
:10F6B000C42CD12CE12CF12C22242394240C4AC0FC
:10F6C0008091EF058823C9F08091620F9091630FBC
:10F6D000A091640FB091650FB695A7959795879502
:10F6E00020E20197A105B10511F44EE301C040E20B
:10F6F0006AEA77E0852D0E9472733320A1F280912F
:10F70000620F9091630FA091640FB091650FB69551
:10F71000A795979587950197A105B10521F67ED804
:10F720006CD8F5C1241161C140E050E0B50189E811
:10F730009CE00E94343F9091CF0C8091EF0599237B
:10F7400009F49BC081110BC0311074C0222DF1E06F
:10F75000AF1AB1083FEFA316B30621F748C1809155
:10F76000620F9091630FA091640FB091650FB695F1
:10F77000A79597958795452D60E08C159D05AE055D
:10F78000BF0561F58DE69FE00E94A7316EE38DE62F
:10F790009FE00E9494C765E08DE69FE00E9494C7B9
:10F7A00080919A0C882329F01092AC0C0AE91CE095
:10F7B00002C00DE81CE092E1992EF80161918F01E1
:10F7C000662311F0911062C1992009F4BDCF60E267
:10F7D0008DE69FE00E9494C79A94F6CF8DE69FE055
:10F7E0000E94A73160E28DE69FE00E9494C765E029
:10F7F0008DE69FE00E9494C780919A0C882329F09F
:10F800001092AC0C0AE91CE002C00DE81CE082E199
:10F81000982EF80161918F01662311F091103CC17F
:10F82000992009F491CF60E28DE69FE00E9494C791
:10F830009A94F6CF8091620F9091630FA091640F1C
:10F84000B091650FB695A795979587958C159D05F1
:10F85000AE05BF0509F07ACF0E940E746DE87CE01A
:10F8600089E89CE00E947C431092620F1092630F23
:10F870001092640F1092650F4AC1811103C03110BC
:10F8800071C064CF8091620F9091630FA091640F5B
:10F89000B091650FB695A795979587958C159D05A1
:10F8A000AE05BF05B1F52091E40F2F8F10E0412F79
:10F8B00060E08DE69FE00E94A73160E28DE69FE068
:10F8C0000E9494C71F5F143091F7452D60E08DE6CC
:10F8D0009FE00E94A7316EE38DE69FE00E9494C7EF
:10F8E000ABE98A2EACE09A2EBAE96B2EBCE07B2EF7
:10F8F00001E010E0F30121913F012111D3C014E197
:10F90000101B60E28DE69FE00E9494C71150C9F77A
:10F91000B6CF452D60E08DE69FE00E94A73160E202
:10F920008DE69FE00E9494C780919A0C882329F06D
:10F930001092AD0C0AE91CE002C00DE81CE0F3E1F6
:10F940009F2EF80161918F01662311F09110D9C0AB
:10F95000992009F494CF60E28DE69FE00E9494C75D
:10F960009A94F6CF8091620F9091630FA091640FEB
:10F97000B091650FB695A795979587958C159D05C0
:10F98000AE05BF0509F0E2CE0E940E748DE89CE042
:10F990009F938F9388E793E29F938F938E010F5FDE
:10F9A0001F4F1F930F930E9439D00F900F900F900D
:10F9B0000F900F900F907E01F5E0EF0EF11CF70114
:10F9C0008081882349F0992787FD90950E946DCF0B
:10F9D000F70181937F01F3CFC8010E94CB4884E7F0
:10F9E00093E20E944B4918DD92C02F5FB0CE809108
:10F9F000620F9091630FA091640FB091650FB6955F
:10FA0000A79597958795422F50E060E070E08417A6
:10FA10009507A607B70788F0822F90E0880F991FF7
:10FA20000197AA2797FDA095BA2F8093620F909314
:10FA3000630FA093640FB093650F8091620F909154
:10FA4000630FA091640FB091650FB695A795979538
:10FA5000879520916B0F30E02D5F3F4F482F50E08E
:10FA60002417350764F42DEF280F20936B0F21E046
:10FA70002093EF054CEF442E480E55245A9453948E
:10FA8000439483E0851508F0CACD41C08DE69FE020
:10FA90000E9494C79A9491CE8DE69FE00E9494C7ED
:10FAA0009A94B7CE452D602F8DE69FE02AA30E9441
:10FAB000A7312AA1622F8DE69FE00E9494C70F5FB5
:10FAC0001F4F0431110509F015CF34010CE211E08C
:10FAD00080916C0F82FD05C08091E40F3F8D381737
:10FAE00049F0015011090115110591F78FEF881A9E
:10FAF000980AFECE61E070E080E090E00E9435C39D
:10FB0000F0CF8DE69FE00E9494C79A941ACFA296F8
:10FB10000FB6F894DEBF0FBECDBFDF91CF911F911E
:10FB20000F91FF90EF90DF90CF90BF90AF909F909C
:10FB30008F907F906F905F904F903F902F9008959F
:10FB4000CF92DF92EF92FF920F931F93CF93DF93A9
:10FB50008091620F9091630FA091640FB091650F37
:10FB600081309048A105B10540F01092620F1092CB
:10FB7000630F1092640F1092650F8091620F909145
:10FB8000630FA091640FB091650FB695A7959795F7
:10FB9000879540916B0F50E060E070E08417950707
:10FBA000A607B70710F480936B0FD0916B0F1091DD
:10FBB0006C0F12FB112710F9C0E0BFE0CB2ED12C47
:10FBC000E12CF12C01E04091620F5091630F6091A4
:10FBD000640F7091650FD1113BC08091EF058823B0
:10FBE000C9F0E0917A0CF0E0EE0FFF1FE45EFD4FEC
:10FBF0000190F081E02D8681978123E0423051050C
:10FC00006105710510F443E001C040E2BC018C2F96
:10FC10000E947273112309F4A6C18091620F909122
:10FC2000630FA091640FB091650F0297A105B10514
:10FC300008F099C10E940E748AE392E9DF91CF9196
:10FC40001F910F91FF90EF90DF90CF900C9446742E
:10FC5000D130A9F58091EF05882391F076956795CD
:10FC60005795479520E2413051056105710511F422
:10FC70004EE301C040E264E573E28C2F0E94727390
:10FC8000112309F470C18091620F9091630FA091CC
:10FC9000640FB091650FB695A795979587950197D5
:10FCA000A105B10509F05FC10E940E74DF91CF91EB
:10FCB0001F910F91FF90EF90DF90CF90DDCBD2306E
:10FCC000A9F58091EF05882391F076956795579572
:10FCD000479520E2423051056105710511F44EE36C
:10FCE00001C040E265E473E28C2F0E94727311231D
:10FCF00009F439C18091620F9091630FA091640F54
:10FD0000B091650FB695A795979587950297A10530
:10FD1000B10509F028C10E940E74DF91CF911F91A7
:10FD20000F91FF90EF90DF90CF908FCBD330A9F55C
:10FD30008091EF05882391F07695679557954795C3
:10FD400020E2433051056105710511F44EE301C015
:10FD500040E266E373E28C2F0E947273112309F470
:10FD600002C18091620F9091630FA091640FB091D6
:10FD7000650FB695A795979587950397A105B1054A
:10FD800009F0F1C00E940E74DF91CF911F910F9185
:10FD9000FF90EF90DF90CF909DCBD430A9F580916C
:10FDA000EF05882391F0769567955795479520E262
:10FDB000443051056105710511F44EE301C040E284
:10FDC00066E273E28C2F0E947273112309F4CBC098
:10FDD0008091620F9091630FA091640FB091650FB5
:10FDE000B695A795979587950497A105B10509F054
:10FDF000BAC00E940E74DF91CF911F910F91FF90B6
:10FE0000EF90DF90CF907DCBD530A9F58091EF05B5
:10FE1000882391F0769567955795479520E2453070
:10FE200051056105710511F44EE301C040E266E140
:10FE300073E28C2F0E947273112309F494C0809195
:10FE4000620F9091630FA091640FB091650FB6950A
:10FE5000A795979587950597A105B10509F083C0EA
:10FE60000E940E74DF91CF911F910F91FF90EF9040
:10FE7000DF90CF9018CBD630A9F58091EF0588237D
:10FE800091F0769567955795479520E24630510554
:10FE90006105710511F44EE301C040E267E073E2D1
:10FEA0008C2F0E947273112309F45DC08091620F40
:10FEB0009091630FA091640FB091650FB695A795CF
:10FEC000979587950697A105B10509F04CC00E944A
:10FED0000E74DF91CF911F910F91FF90EF90DF9003
:10FEE000CF9026CBD73009F03EC08091EF05882314
:10FEF000E9F0E0917A0CF0E0EE0FFF1FE45EFD4FB9
:10FF00000190F081E02D86A597A576956795579588
:10FF1000479520E2473051056105710511F44EE324
:10FF200001C040E2BC018C2F0E9472731123D9F0F2
:10FF30008091620F9091630FA091640FB091650F53
:10FF4000B695A795979587950797A105B10559F49B
:10FF50000E940E74DF91CF911F910F91FF90EF904F
:10FF6000DF90CF9061CA8091620F9091630FA09152
:10FF7000640FB091650F4097A105B10540F0C092A4
:10FF8000620FD092630FE092640FF092650F409180
:10FF9000620F5091630F6091640F7091650F7695B9
:10FFA00067955795479580916B0F90E00396242FA6
:10FFB00030E0821793074CF48DEF840F80936B0F22
:10FFC0000093EF05DCEFD40FCFEFCF5FDF5FC430DE
:10FFD00008F4F9CDDF91CF911F910F91FF90EF9031
:10FFE000DF90CF900895CF93DF93CDB7DEB72897FA
:10FFF0000FB6F894DEBF0FBECDBF88E0E7E6F6E0AF
:020000021000EC
:10000000DE01119601900D928A95E1F7AE014F5FE6
:100010005F4F61E08DE69FE00E94453328960FB662
:10002000F894DEBF0FBECDBFDF91CF910895CF937F
:10003000DF93CDB7DEB728970FB6F894DEBF0FBEBB
:10004000CDBF88E0EFE2F6E0DE01119601900D925F
:100050008A95E1F7AE014F5F5F4F61E08DE69FE06B
:100060000E94453328960FB6F894DEBF0FBECDBF71
:10007000DF91CF91089588EF9FE00E9455D28230A2
:1000800028F480937A0C1092410F089581E08093B8
:100090007A0C8093410F08951F93CF93DF93EC0167
:1000A000FB01608111810E945DD2612FCE0101961A
:1000B000DF91CF911F910C945DD2FF920F931F930C
:1000C000CF93DF938C01EB010E9455D2F82EC8012B
:1000D00001960E9455D2F8828983DF91CF911F91BA
:1000E0000F91FF900895EF92FF920F931F93CF937C
:1000F000DF931F92CDB7DEB77B018C01061B170B78
:10010000460FC701800F911FF70161917F0149835D
:100110000E945DD249814E11F4CF0F90DF91CF91B3
:100120001F910F91FF90EF90089581E09091DB0F68
:10013000911180E08093DB0F41E06BED7FE08FEF6A
:100140009FE0D1DF0E94F8AD21E047E050E060E0A1
:1001500070E087EE90E80C94307481E09091DB0FB2
:10016000911180E08093DB0F41E06BED7FE08FEF3A
:100170009FE0B9DF0E94F8AD21E049E050E060E087
:1001800070E085EE98E80C943074EF92FF920F9334
:100190001F93CF93DF931F92CDB7DEB77B018C0106
:1001A000061B170B460FC701800F911F49830E9442
:1001B00055D2F70181937F0149814E13F4CF0F90FF
:1001C000DF91CF911F910F91FF90EF900895CF9203
:1001D000DF92EF92FF920F931F93CF93DF9341E053
:1001E0006BED7FE08FEF9FE0D0DF8091620F909109
:1001F000630FA091640FB091650F81309048A10505
:10020000B10540F01092620F1092630F1092640FCC
:100210001092650F8091620F9091630FA091640F0F
:10022000B091650FB695A7959795879540916B0FFF
:1002300050E060E070E084179507A607B70710F458
:1002400080936B0FD0916B0F10916C0F12FB1127E5
:1002500010F9C0E09FE0C92ED12CE12CF12C01E077
:100260004091620F5091630F6091640F7091650F20
:10027000D1113BC08091EF058823C9F0E0917A0C41
:10028000F0E0EE0FFF1FE45EFD4F0190F081E02DE6
:100290008681978123E0423051056105710510F494
:1002A00043E001C040E2BC018C2F0E947273112315
:1002B00009F453C18091620F9091630FA091640F74
:1002C000B091650F0297A105B10508F046C10E94E3
:1002D0000E748AE392E9DF91CF911F910F91FF9005
:1002E000EF90DF90CF900C944674D130E1F580917F
:1002F000EF058823F9F0E0917A0CF0E0EE0FFF1F94
:10030000E45EFD4F0190F081E02DE856FF4F8081C3
:10031000918176956795579547952EE74130510520
:100320006105710511F44EE301C040E2BC018C2F60
:100330000E947273112309F410C18091620F909191
:10034000630FA091640FB091650FB695A79597952F
:1003500087950197A105B10509F0FFC00E940E74B1
:1003600088EE96E897C1D230D1F58091EF058823C9
:10037000E9F0E0917A0CF0E0EE0FFF1FE45EFD4F34
:100380000190F081E02D80AD91AD76956795579500
:1003900047952EE7423051056105710511F44EE392
:1003A00001C040E2BC018C2F0E947273112309F43A
:1003B000D4C08091620F9091630FA091640FB091AF
:1003C000650FB695A795979587950297A105B105F5
:1003D00009F0C3C00E940E7483EF99E75BC1D3306C
:1003E000E1F58091EF058823F9F0E0917A0CF0E0D7
:1003F000EE0FFF1FE45EFD4F0190F081E02DEC5009
:10040000FF4F80819181769567955795479520E2BA
:10041000433051056105710511F44EE301C040E21E
:10042000BC018C2F0E947273112309F496C0809135
:10043000620F9091630FA091640FB091650FB69514
:10044000A795979587950397A105B10509F085C0F4
:100450000E940E7486E993E23CC0D43009F043C098
:100460008091EF058823E9F0E0917A0CF0E0EE0F3F
:10047000FF1FE45EFD4F0190F081E02D82859385A2
:10048000769567955795479520E24430510561056B
:10049000710511F44EE301C040E2BC018C2F0E94B3
:1004A0007273112309F459C08091620F9091630F08
:1004B000A091640FB091650FB695A7959795879514
:1004C0000497A105B10509F048C00E940E7482E9A5
:1004D00093E2DF91CF911F910F91FF90EF90DF900A
:1004E000CF900C944B49D530C1F58091EF0588230E
:1004F000E9F0E0917A0CF0E0EE0FFF1FE45EFD4FB3
:100500000190F081E02D84859585769567955795C6
:10051000479520E2453051056105710511F44EE320
:1005200001C040E2BC018C2F0E9472731123A9F01C
:100530008091620F9091630FA091640FB091650F4D
:10054000B695A795979587950597A105B10529F4C7
:100550000E940E748EE893E2BCCF2091DB0F809155
:10056000620F9091630FA091640FB091650F2111FC
:1005700014C0D63009F054C02091EF05222379F140
:10058000E0917A0CF0E0EE0FFF1FE45EFD4F01906A
:10059000F081E02DE05EFE4F13C0D63009F040C080
:1005A0002091EF052223D9F0E0917A0CF0E0EE0FD4
:1005B000FF1FE45EFD4F0190F081E02DE25EFE4FF3
:1005C00060817181B695A7959795879520E20697EA
:1005D000A105B10519F140E28C2F0E94727311231D
:1005E00009F462C08091620F9091630FA091640F33
:1005F000B091650FB695A795979587950697A10534
:10060000B10509F051C00E940E74DF91CF911F9186
:100610000F91FF90EF90DF90CF9087CD4EE3DCCF2E
:10062000D73009F041C02091EF052223E9F0E09195
:100630007A0CF0E0EE0FFF1FE45EFD4F0190F081B9
:10064000E02DEA54FE4F60817181B695A79597958C
:1006500087952EE70797A105B10511F44EE301C078
:1006600040E28C2F0E9472731123F1F08091620F8F
:100670009091630FA091640FB091650FB695A79507
:10068000979587950797A105B10571F40E940E749F
:1006900088E996E7DF91CF911F910F91FF90EF903E
:1006A000DF90CF900C944B748091620F9091630F08
:1006B000A091640FB091650F4097A105B10540F07E
:1006C000C092620FD092630FE092640FF092650FB8
:1006D0004091620F5091630F6091640F7091650FAC
:1006E000769567955795479580916B0F90E00396A7
:1006F000242F30E0821793074CF48DEF840F809302
:100700006B0F0093EF05DCEFD40FCFEFCF5FDF5F10
:10071000C43008F4A5CDDF91CF911F910F91FF90C8
:10072000EF90DF90CF9008956FEF88EF9FE00C94EB
:100730005DD280935B0F10925A0F0895E9EBFFE0B2
:1007400001900020E9F73197E95BFF401E161F0674
:1007500034F01092CD0F82E08093EF05089580E28F
:10076000E431F105B4F7DF01A754B04F8C93319613
:10077000F7CF2091CE0F211108C044E150E0BC0119
:1007800089EB9FE00E942AD0D9CF089510928B0C5C
:1007900060E089E89CE00E941F3F0E9414AD88E65B
:1007A00093E20E944B4981E08093440CE0917A0CE3
:1007B000F0E0EE0FFF1FE45EFD4F0190F081E02DB1
:1007C000EA53FF4F80819181D4DF84E693E20C9459
:1007D0004B492091CE0F211108C044E150E0BC01EB
:1007E00089EB9FE00E949DCFA9CF0895F2DF81E0C1
:1007F0008093CE0F0C940C7A1092CE0F0895CF9266
:10080000DF92EF92FF92CF93CCB1C095CC1FCC2753
:10081000CC1F8091030183FFC260C090670FD0900E
:10082000680FE090690FF0906A0F0E9406C3C61629
:10083000D706E806F90610F4489B39C0C0936C0F40
:1008400080916C0F817090916C0F91FD82609091FE
:10085000660F891721F18130F1F028F0823089F09C
:100860008330A1F01CC0913021F49091E40F9F5F80
:1008700005C09230A1F49091E40F91509093E40F51
:100880000EC0992391F3933051F4F5CF923069F370
:10089000913029F4F0CF933041F3992361F38093A1
:1008A000660FCF91FF90EF90DF90CF900895C460D6
:1008B000C5CF0E94007A6F98E4E0F1E08081877FE5
:1008C0008083779A9FB7F894E5E0F1E080818860B3
:1008D00080839FBF5098589A60E088E40E9426C2A7
:1008E0009FB7F894E5E0F1E08081846080839FBF4A
:1008F0008091030182FB882780F991E0892780930A
:10090000610F7DDF1092E40F0895CF92DF92EF9296
:10091000FF9275DF8091030191E082FB882780F9C7
:1009200089272091610F821719F182E08093EF05EA
:100930008091030182FB882780F989278093610FCA
:100940000E94007A8091610F882309F4A8C089E889
:100950009CE00E940E3AE0917A0CF0E0EE0FFF1F4F
:10096000E45EFD4F0190F081E02D8281938131DFC3
:10097000C0905D0FD0905E0FE0905F0FF090600F21
:100980000E9406C3C616D706E806F90608F09EC000
:100990008091E40F482F552747FD509557FF03C01E
:1009A0005195419551094230510584F191E0909360
:1009B000EF0587FD8F5F482F4595552747FD5095DB
:1009C000652F752F8091620F9091630FA091640F36
:1009D000B091650F840F951FA61FB71F8093620FFC
:1009E0009093630FA093640FB093650F1092E40F80
:1009F0000E9406C36856754C8F4F9F4F6093310F0E
:100A00007093320F8093330F9093340F80916C0F5B
:100A100082FF0EC00E9406C36856754C8F4F9F4FD1
:100A20006093310F7093320F8093330F9093340F94
:100A3000E091F005F091F1051995C090310FD0903B
:100A4000320FE090330FF090340F0E9406C3C616A9
:100A5000D706E806F90638F48091F0059091F10583
:100A6000865E984969F58091EF05823011F40E9405
:100A7000217A8091EF05882319F081508093EF054A
:100A80000E9406C36C597F4F8F4F9F4F60935D0F3D
:100A900070935E0F80935F0F9093600F17C089E88B
:100AA0009CE00E940D3BE0917A0CF0E0EE0FFF1FFE
:100AB000E45EFD4F0190F081E02D8481958157CF58
:100AC0000E940C7A82E08093EF05CDCFFF90EF90EB
:100AD000DF90CF90089581E0089580916C0F82FBA4
:100AE000882780F90895FC01808190E02AE030E0B9
:100AF000B9010E9440CC482FCB01B9010E9440CCE3
:100B0000805D8093350F405D4093360F1092370F14
:100B100085E39FE0089520E030E040E251E4FC01ED
:100B200060817181828193810E944ACB0E94E4C8D6
:100B300077FD02C02BE201C02DE22093350F9B010F
:100B400077FF04C022273327261B370BC90168EE25
:100B500073E00E9440CCCB01EAE0F0E0BF010E94CC
:100B600040CC805D8093360FC90164E670E00E943E
:100B700040CCCB01BF010E9440CC805D8093370FF9
:100B8000C901BF010E9440CC282FCB01BF010E94A8
:100B900040CC805D8093380F8EE28093390F205DCA
:100BA00020933A0F10923B0F85E39FE008958F92B8
:100BB0009F92AF92BF92CF92DF92EF92FF92FC0191
:100BC00080809180A280B38020E030E048EC52E445
:100BD000C501B4010E944ACB6B017C0120E030E0EA
:100BE000A9010E9478CA18161CF4C701B60103C0F7
:100BF000C701B60190580E94E4C86B017C0120E057
:100C000030E0A901C501B4010E9475C887FF12C078
:100C10008DE28093350FC701B60128EE33E040E046
:100C200050E00E9475CCCA01B9012AE030E040E0F2
:100C300050E036C0C701B60120E137E240E050E0A5
:100C40000E9475CCAAE08A2E912CA12CB12CCA014D
:100C5000B901A50194010E9475CC662391F0605DF5
:100C60006093350FC701B60128EE33E040E050E055
:100C70000E9475CCCA01B901A50194010E9475CCEE
:100C800013C080E28093350FC701B60128EE33E030
:100C900040E050E00E9475CCCA01B901A501940161
:100CA0000E9475CC662311F0605D01C060E2609324
:100CB000360FC701B60124E630E040E050E00E9464
:100CC00075CCFAE08F2E912CA12CB12CCA01B90160
:100CD000A50194010E9475CC605D6093370FC70138
:100CE000B601A50194010E9475CC662381F0605D78
:100CF00060933A0FCA01B901A50194010E9475CC15
:100D0000605D6093390F8EE28093380F15C0CA0181
:100D1000B901A50194010E9475CC662329F0605D9C
:100D20006093390F8EE203C080E28093390F809385
:100D3000380F80E280933A0F10923B0F85E39FE0DB
:100D4000FF90EF90DF90CF90BF90AF909F908F90EB
:100D50000895FC012081318137FF07C08DE2809327
:100D6000350F31952195310914C02436310574F0C1
:100D7000C90164E670E00E9440CCCB016AE070E0FB
:100D80000E9440CC805D8093350F06C080E2809346
:100D9000350F2A30310564F0EAE0F0E0C901BF0107
:100DA0000E9440CCCB01BF010E9440CC805D01C0BD
:100DB00080E28093360FC9016AE070E00E9440CC67
:100DC000805D8093370F1092380F85E39FE0089580
:100DD000AF92BF92CF92DF92EF92FF920F931F9349
:100DE000CF93DF93609114027091150280911602E7
:100DF000909117020E94E6306093460F7093470F60
:100E00008093480F9093490F6091100270911102E6
:100E100080911202909113020E94F2306093420F6F
:100E20007093430F8093440F9093450F8091620F0E
:100E30009091630FA091640FB091650F813090483D
:100E4000A105B10540F01092620F1092630F10924D
:100E5000640F1092650F8091620F9091630FA091C3
:100E6000640FB091650FB695A795979587954091BA
:100E70006B0F50E060E070E084179507A607B70796
:100E800010F480936B0F00916B0FB0906C0FB2FA5F
:100E9000BB24B0F810E047E0C42ED12CE12CF12C9B
:100EA000AA24A3948091620F9091630FA091640F84
:100EB000B091650F01113DC02091EF052223C9F0CB
:100EC000E0917A0CF0E0EE0FFF1FE45EFD4F019021
:100ED000F081E02DEA50FF4F6081718123E002979D
:100EE000A105B10510F443E001C040E2812F0E944A
:100EF0007273BB2009F427C18091620F9091630F38
:100F0000A091640FB091650F0297A105B10508F09B
:100F10001AC10E940E7487EE90E8DF91CF911F9165
:100F20000F91FF90EF90DF90CF90BF90AF900C9417
:100F30004674013009F052C02091EF05222329F1B7
:100F4000E0917A0CF0E0EE0FFF1FE45EFD4F0190A0
:100F5000F081E02DE25BFF4FC081D181B695A7956E
:100F6000979587950197A105B10531F488E59AE039
:100F7000F0DE9C014EE305C088E59AE0EADE9C01C4
:100F800040E2BE01812F0E94A973BB2009F4DBC09F
:100F90008091620F9091630FA091640FB091650FE3
:100FA000B695A795979587950197A105B10509F085
:100FB000CAC00E940E74E0917A0CF0E0EE0FFF1FA1
:100FC000E45EFD4F0190F081E02DE25BFF4F2CE2EB
:100FD00031E040E050E068E57AE0A7C0023009F077
:100FE00052C02091EF05222329F1E0917A0CF0E024
:100FF000EE0FFF1FE45EFD4F0190F081E02DEC5AF3
:10100000FF4FC081D181B695A79597958795029797
:10101000A105B10531F486E59AE09BDE9C014EE323
:1010200005C086E59AE095DE9C0140E2BE01812F75
:101030000E94A973BB2009F486C08091620F909131
:10104000630FA091640FB091650FB695A795979522
:1010500087950297A105B10509F075C00E940E742D
:10106000E0917A0CF0E0EE0FFF1FE45EFD4F01907F
:10107000F081E02DEC5AFF4F23E930E040E050E0F2
:1010800066E57AE052C0033009F05DC02091EF05BB
:10109000222329F1E0917A0CF0E0EE0FFF1FE45ECD
:1010A000FD4F0190F081E02DEA5AFF4FC081D181C0
:1010B000B695A795979587950397A105B10531F446
:1010C00083E59CE046DE9C014EE305C083E59CE0A1
:1010D00040DE9C0140E2BE01812F0E94A973BB202B
:1010E00091F18091620F9091630FA091640FB09184
:1010F000650FB695A795979587950397A105B105B7
:1011000011F50E940E74E0917A0CF0E0EE0FFF1FD3
:10111000E45EFD4F0190F081E02DEA5AFF4F2FEF82
:1011200030E040E050E063E57CE080819181DF9138
:10113000CF911F910F91FF90EF90DF90CF90BF90D4
:10114000AF900C9483728091620F9091630FA09185
:10115000640FB091650F0897A105B10540F0C092EA
:10116000620FD092630FE092640FF092650F40918E
:10117000620F5091630F6091640F7091650F7695C7
:1011800067955795479580916B0F90E00396242FB4
:1011900030E0821793074CF48DEF840F80936B0F30
:1011A000A092EF050CEF040F1FEF1F5F0F5F1430CD
:1011B00008F478CEDF91CF911F910F91FF90EF90BF
:1011C000DF90CF90BF90AF900895AF92BF92CF9233
:1011D000DF92EF92FF920F931F93CF93DF9341E043
:1011E0006BED7FE08FEF9FE00E94C5808091620FE2
:1011F0009091630FA091640FB091650F813090487A
:10120000A105B10540F01092620F1092630F109289
:10121000640F1092650F8091620F9091630FA091FF
:10122000640FB091650FB695A795979587954091F6
:101230006B0F50E060E070E084179507A607B707D2
:1012400010F480936B0F00916B0FB0906C0FB2FA9B
:10125000BB24B0F810E04FE0C42ED12CE12CF12CCF
:10126000AA24A3948091620F9091630FA091640FC0
:10127000B091650F01113BC02091EF052223B9F019
:10128000E0917A0CF0E0EE0FFF1FE45EFD4F01905D
:10129000F081E02D6681778123E00297A105B105F9
:1012A00010F443E001C040E2812F0E947273BB2022
:1012B00009F419C28091620F9091630FA091640F9D
:1012C000B091650F0297A105B10508F00CC20E940C
:1012D0000E748AE392E9DF91CF911F910F91FF90F5
:1012E000EF90DF90CF90BF90AF900C944674013098
:1012F00009F052C02091EF05222329F1E0917A0CE8
:10130000F0E0EE0FFF1FE45EFD4F0190F081E02D55
:10131000E45BFF4FC081D181B695A79597958795DE
:101320000197A105B10531F48DED95E012DD9C0129
:101330004EE305C08DED95E00CDD9C0140E2BE0161
:10134000812F0E94A973BB2009F4CDC18091620F47
:101350009091630FA091640FB091650FB695A7951A
:10136000979587950197A105B10509F0BCC10E9429
:101370000E74E0917A0CF0E0EE0FFF1FE45EFD4F7B
:101380000190F081E02DE45BFF4F27EE33E04AE06F
:1013900050E06DED75E054C0023009F05FC020915F
:1013A000EF05222329F1E0917A0CF0E0EE0FFF1F08
:1013B000E45EFD4F0190F081E02DE25BFF4FC081C4
:1013C000D181B695A795979587950297A105B10507
:1013D00031F488E59AE0BDDC9C014EE305C088E568
:1013E0009AE0B7DC9C0140E2BE01812F0E94A97304
:1013F000BB2009F478C18091620F9091630FA09196
:10140000640FB091650FB695A7959795879502974C
:10141000A105B10509F067C10E940E74E0917A0C34
:10142000F0E0EE0FFF1FE45EFD4F0190F081E02D34
:10143000E25BFF4F2CE231E040E050E068E57AE00B
:1014400080819181DF91CF911F910F91FF90EF905B
:10145000DF90CF90BF90AF900C948372033009F06F
:1014600052C02091EF05222329F1E0917A0CF0E09F
:10147000EE0FFF1FE45EFD4F0190F081E02DEC5A6E
:10148000FF4FC081D181B695A79597958795039712
:10149000A105B10531F486E59AE05BDC9C014EE3E1
:1014A00005C086E59AE055DC9C0140E2BE01812F33
:1014B0000E94A973BB2009F416C18091620F90911C
:1014C000630FA091640FB091650FB695A79597959E
:1014D00087950397A105B10509F005C10E940E7417
:1014E000E0917A0CF0E0EE0FFF1FE45EFD4F0190FB
:1014F000F081E02DEC5AFF4F2CE830E040E050E066
:1015000066E57AE09DCF043009F052C02091EF05E6
:10151000222329F1E0917A0CF0E0EE0FFF1FE45E48
:10152000FD4F0190F081E02DEA5AFF4FC081D1813B
:10153000B695A795979587950497A105B10531F4C0
:1015400083E59CE006DC9C014EE305C083E59CE05E
:1015500000DC9C0140E2BE01812F0E94A973BB20E8
:1015600009F4C1C08091620F9091630FA091640F44
:10157000B091650FB695A795979587950497A105A6
:10158000B10509F0B0C00E940E74E0917A0CF0E051
:10159000EE0FFF1FE45EFD4F0190F081E02DEA5A4F
:1015A000FF4F2FEF30E040E050E063E57CE048CFB4
:1015B000053009F052C02091EF05222329F1E09176
:1015C0007A0CF0E0EE0FFF1FE45EFD4F0190F0811A
:1015D000E02DE85AFF4FC081D181B695A795979528
:1015E00087950597A105B10531F48BED95E0B1DB49
:1015F0009C014EE305C08BED95E0ABDB9C0140E226
:10160000BE01812F0E94A973BB2009F46CC0809198
:10161000620F9091630FA091640FB091650FB69522
:10162000A795979587950597A105B10509F05BC02A
:101630000E940E74E0917A0CF0E0EE0FFF1FE45E62
:10164000FD4F0190F081E02DE85AFF4F27EE33E087
:101650004AE050E06BED75E0F3CE063009F043C090
:101660002091EF052223E9F0E0917A0CF0E0EE0FF3
:10167000FF1FE45EFD4F0190F081E02DE252FF4F2D
:1016800060817181B695A7959795879520E2069719
:10169000A105B10511F44EE301C040E2812F0E9483
:1016A0007273BB2001F18091620F9091630FA09142
:1016B000640FB091650FB695A79597958795069796
:1016C000A105B10581F40E940E7482E093E2DF91DE
:1016D000CF911F910F91FF90EF90DF90CF90BF902F
:1016E000AF900C944B492091DB0F8091620F909149
:1016F000630FA091640FB091650F211114C00730E2
:1017000009F055C02091EF05222379F1E0917A0C80
:10171000F0E0EE0FFF1FE45EFD4F0190F081E02D41
:10172000E05EFE4F13C0073009F041C02091EF0585
:101730002223D9F0E0917A0CF0E0EE0FFF1FE45E77
:10174000FD4F0190F081E02DE25EFE4F60817181DE
:10175000B695A7959795879520E20797A105B105BE
:1017600021F140E2812F0E947273BB2001F1809130
:10177000620F9091630FA091640FB091650FB695C1
:10178000A795979587950797A105B10581F40E94C4
:101790000E74DF91CF911F910F91FF90EF90DF902A
:1017A000CF90BF90AF900C94AD804EE3DBCF809193
:1017B000620F9091630FA091640FB091650F4097F5
:1017C000A105B10540F0C092620FD092630FE09284
:1017D000640FF092650F8091620F9091630FA0915A
:1017E000640FB091650FB695A79597958795209151
:1017F0006B0F30E02D5F3F4F482F50E02417350727
:101800004CF42DEF280F20936B0FA092EF050CEFF7
:10181000080F1FEF1F5F0F5F143008F423CDDF9117
:10182000CF911F910F91FF90EF90DF90CF90BF90DD
:10183000AF900895FC01808191818436910524F157
:1018400064E670E00E9440CCCB012AE030E0B901B0
:101850000E9440CC805D8093350F80819181B901D9
:101860000E9440CCCB01B9010E9440CC805D8093A6
:10187000360F80819181B9010E9440CC805D8093B8
:10188000370F1092380F23C08A309105BCF02AE040
:1018900030E0B9010E9440CCCB01B9010E9440CC9C
:1018A000805D8093350F80819181B9010E9440CC89
:1018B000805D8093360F1092370F09C06AE070E0A8
:1018C0000E9440CC805D8093350F1092360F85E3E7
:1018D0009FE008958F929F92AF92BF92CF92DF9236
:1018E000EF92FF92CF9320E030E040E251E4FC0120
:1018F00060817181828193810E944ACB0E94E4C8F9
:1019000097FD02C02BE201C02DE22093350F6B0141
:101910007C0197FF08C0F094E094D094C094C11C5F
:10192000D11CE11CF11CC701B60120E137E240E007
:1019300050E00E9475CC7AE0872E912CA12CB12C1E
:10194000CA01B901A50194010E9475CC605D609344
:10195000360FC701B60128EE33E040E050E00E94A8
:1019600075CCCA01B901A50194010E9475CC605DD6
:101970006093370FC701B60124E630E040E050E045
:101980000E9475CCCA01B901A50194010E9475CCD1
:10199000605D6093380FC701B601A50194010E94F4
:1019A00075CCC62FCA01B901A50194010E9475CC5E
:1019B000605D6093390F8EE280933A0FC05DC093F3
:1019C0003B0F10923C0F85E39FE0CF91FF90EF908B
:1019D000DF90CF90BF90AF909F908F900895CF925F
:1019E000EF920F93FFE1CF2EA0E2EA2E0FE02EE060
:1019F00045E066E28DE69FE00E9492320F91EF9003
:101A0000CF900895CF93DF93FC016491EC01219670
:101A1000662331F08DE69FE00E947F33CE01F4CF44
:101A2000DF91CF9108950F931F93CF93DF938C0194
:101A3000EB0141E061E08DE69FE00E94A731C80123
:101A4000E1DF6AE38DE69FE00E9494C7FE0101900A
:101A50000020E9F76C2F6E1B6C5E41E08DE69FE085
:101A60000E94A731BE018DE69FE0DF91CF911F91CB
:101A70000F910C9493C7CF92DF92EF92FF920F9346
:101A80001F938091620F9091630FA091640FB091AA
:101A9000650F0097A105B10509F442C0BC01882774
:101AA00077FD8095982F0E9417C920913D0F3091A6
:101AB0003E0F40913F0F5091400F0E944ACB9B0137
:101AC000AC016091750C7091760C8091770C9091BF
:101AD000780C0E949CC76093750C7093760C809371
:101AE000770C9093780C1092620F1092630F109203
:101AF000640F1092650FB5E5CB2EBCE0DB2EE12C18
:101B0000F12C00E81FE325E73CE041E75CE06DE6EF
:101B10007CE089E69CE00E9431B481E08093EF058F
:101B20008091EF05882341F085E79CE00E948B853A
:101B3000BC0185E893E277DF80916C0F82FF0EC0D5
:101B400021E040E050E0BA0181E398E71F910F9156
:101B5000FF90EF90DF90CF900C9430741F910F9115
:101B6000FF90EF90DF90CF900895CF93DF931F9277
:101B70001F92CDB7DEB78091620F9091630FA09155
:101B8000640FB091650FB7FF08C01092620F1092FA
:101B9000630F1092640F1092650F80914A0F90911D
:101BA0004B0FA0914C0FB0914D0F4091620F50918F
:101BB000630F6091640F7091650F84179507A607F6
:101BC000B70744F48093620F9093630FA093640F60
:101BD000B093650F8091EF058823A9F080914E0F97
:101BE00090914F0F2091620F3091630F820F931FDE
:101BF0009A838983CE010196ACD8BC018091540FA1
:101C00009091550F10DF80916C0F82FF1DC0E09105
